:100000000C9414290C9485510C945A510C942F5132
:100010000C9404510C94D9500C94AE500C94835011
:100020000C9458500C9445290C9445290C9445295E
:100030000C9445290C949BF00C9445290C9445296B
:100040000C9445290C948BDF0C9445290C9445297C
:100050000C9445290C9445290C9499D10C946C531B
:100060000C9445290C94686A0C94056B0C944529F2
:100070000C9445290C9445290C9445290C94452948
:100080000C9445290C9445290C9445290C94452938
:100090000C9445290C9445290C9445290C94452928
:1000A0000C9445290C9445290C9445290C94452918
:1000B0000C9445290C9445290C9445290C94452908
:1000C0000C9445290C9445290C9445290C944529F8
:1000D0000C9445290C9445290C9445290C944529E8
:1000E0000C94452992489548844888488E48CC48C5
:1000F00099489D48A348A748AB48B148B548B94876
:10010000CC48BF48C348C748305235523A5244528F
:100110004E52C75258526052685272527C528652A6
:1001200095529F52C752A952B352BD528A628A62F7
:10013000916291629162986298629862A5629F62F0
:100140009F629F629E6AA46AB56AC06AC86ADD6AD5
:10015000CC6ADD6AD06AD46ADD6ADA6A39D23DD205
:1001600066D26AD24CD257D226D2084AD73B3BCE6F
:10017000016E84BCBFFDC12F3D6C74319ABD5683A6
:100180003DDA3D00C77F11BED9E4BB4C3E916BAA5E
:10019000AABE000000803F05A84CCDB2D44EB938AD
:1001A00036A9020C50B9918688083CA6AAAA2ABE94
:1001B000000000803F004E414E494E495459494E7F
:1001C00046CDCCCC3D0AD7233C17B7D13877CC2BC2
:1001D000329595E6241FB14F0A000020410000C867
:1001E0004200401C4620BCBE4CCA1B0E5AAEC59DE8
:1001F00074434F4D4D554E49434154494F4E004471
:10020000525952554E004552524F525300494E4694
:100210004F004543484F0020746F6F206C6F6E672E
:1002200020657874727573696F6E2070726576657B
:100230006E7465640A0020636F6C64206578747264
:100240007573696F6E2070726576656E7465640A89
:100250000047322F47332062616420706172616D04
:1002600065746572730A00536C6565702E2E2E00DE
:100270004C756C7A426F742054415A203520726557
:100280006164792E00526573756D696E67207072B6
:10029000696E7400436C69636B20746F20726573C0
:1002A000756D652E2E2E004E6F206D6F76652E00BB
:1002B000456E642066696C65206C6973740A00423F
:1002C0006567696E2066696C65206C6973740A00E5
:1002D0004D313235005344207072696E74696E6717
:1002E000206279746520004E6F7420534420707230
:1002F000696E74696E670A0046696C652064656C96
:10030000657465643A0044656C6574696F6E206657
:1003100061696C65642C2046696C653A20006F70D9
:10032000656E206661696C65642C2046696C653A6F
:1003300020004578747275646572202569202573E4
:10034000004C756C7A426F742054415A20352072EB
:10035000656164792E0012020D020602FF01F101AF
:100360006F66660044454255473A00426564206422
:100370006F6E652E0020573A004265642068656103
:1003800074696E672E0042656420636F6F6C696EDE
:10039000672E004361703A454D455247454E4359DB
:1003A0005F5041525345523A310A004361703A431B
:1003B0004153455F4C494748545F4252494748546E
:1003C0004E4553533A300A004361703A544F474701
:1003D0004C455F4C49474854533A300A00436170DA
:1003E0003A534F4654574152455F504F5745523A42
:1003F000300A004361703A4C4556454C494E475FC0
:10040000444154413A300A004361703A5A5F5052B5
:100410004F42453A300A004361703A4155544F4CBF
:100420004556454C3A300A004361703A5052494EA5
:10043000545F4A4F423A310A004361703A50524F7A
:1004400047524553533A300A004361703A4155547C
:100450004F5245504F52545F54454D503A310A0067
:100460004361703A454550524F4D3A310A00464972
:10047000524D574152455F4E414D453A4D61726C68
:10048000696E20204649524D574152455F564552AC
:1004900053494F4E3A312E312E352E37352045589F
:1004A0005452554445525F545950453A466C65780C
:1004B000794475616C6C7920763220534F555243E4
:1004C000455F434F44455F55524C3A6874747073AE
:1004D0003A2F2F636F64652E616C6570686F626A76
:1004E000656374732E636F6D2F64696666757369D7
:1004F0006F6E2F4D41524C494E2050524F544F4336
:100500004F4C5F56455253494F4E3A312E30204D95
:10051000414348494E455F545950453A4C756C7AB1
:10052000426F742054415A20352045585452554446
:1005300045525F434F554E543A3220555549443A3F
:1005400063333235356339362D343039372D34380D
:1005500038342D386564302D6465643266663962DE
:10056000616536310A007A5F6D696E3A2000795F05
:100570006D696E3A2000785F6D696E3A20005265B1
:10058000706F7274696E6720656E6473746F70202B
:100590007374617475730A004D31343520533C69AE
:1005A0006E6465783E206F7574206F662072616E90
:1005B00067652028302D31290A0020643A0020691F
:1005C0003A0020703A0020643A0020693A00207016
:1005D0003A0043290A0061626C656420286D696EE7
:1005E0002074656D702000436F6C642065787472B0
:1005F000756465732061726520004B64200023647C
:100600006566696E65202044454641554C545F003F
:100610004B69200023646566696E65202044454669
:1006200041554C545F004B70200023646566696E31
:1006300065202044454641554C545F0050494420B4
:100640004175746F74756E652066696E697368654F
:1006500064212050757420746865206C6173742067
:100660004B702C204B6920616E64204B6420636FBB
:100670006E7374616E74732066726F6D2062656C48
:100680006F7720696E746F20436F6E66696775724D
:100690006174696F6E2E680A005049442041757478
:1006A0006F74756E65206661696C6564212074697C
:1006B0006D656F75740A00504944204175746F74FC
:1006C000756E65206661696C6564212054656D7086
:1006D0006572617475726520746F6F2068696768F0
:1006E0000A00204B643A2000204B693A2000204B3E
:1006F000703A20000A20436C61737369632050498B
:1007000044200A002054753A2000204B753A2000FE
:10071000206D61783A2000206D696E3A20002064D7
:100720003A200020626961733A20004F6666736563
:100730007473206170706C696564004572723A2050
:10074000546F6F206661722100546F6F2066617272
:100750002066726F6D207265666572656E636520D6
:10076000706F696E740A004E6F2063617365206C50
:10077000696768740A00556E6B6E6F776E20636FE1
:100780006D6D616E643A2022000000200023002677
:100790000029002C002F0032000001000003010698
:1007A0000109014E6F204C696E65204E756D6265C2
:1007B00072207769746820636865636B73756D2C4C
:1007C000204C617374204C696E653A200053544F7D
:1007D000505045442E20005072696E74657220732B
:1007E000746F707065642064756520746F20657225
:1007F000726F72732E204669782074686520657266
:10080000726F7220616E6420757365204D393939BD
:1008100020746F20726573746172742E2028546581
:100820006D7065726174757265206973207265738D
:1008300065742E2053657420697420616674657236
:100840002072657374617274696E67290A004E6F55
:1008500020436865636B73756D2077697468206CDD
:10086000696E65206E756D6265722C204C617374C3
:10087000204C696E653A2000636865636B73756D23
:10088000206D69736D617463682C204C61737420F2
:100890004C696E653A20004C696E65204E756D623C
:1008A0006572206973206E6F74204C617374204CE4
:1008B000696E65204E756D6265722B312C204C611E
:1008C0007374204C696E653A20004D313130004D13
:1008D0003331004D383420582059205A20450053D8
:1008E000442072656164206572726F720A00446F01
:1008F0006E65207072696E74696E672066696C65DA
:100900000A0025753A2530327500253032753A25B2
:100910003032750025756420253032753A25303225
:10092000750000060900FE00000000000109000833
:10093000FE000005080806000040F0C88888987886
:1009400010050808060000C0F88888888888F8051F
:1009500005050600012030F83020050808060000D3
:100960002070F820202020E00509090600FF2070F3
:10097000A8A8B8888870200509090600FFE080C093
:10098000B0A8283028280509090600FFF8A888889B
:10099000888888A8F8050A0A0600FE2050505050A2
:1009A00088A8A8887003030306000340A04000063F
:1009B0000900FE070192032120FFFF08FF07FF0047
:1009C000000006000001070706020080808080808A
:1009D0000080030202060105A0A00507070600002B
:1009E0005050F850F850500507070600002078A036
:1009F0007028F020050707060000C0C810204098A6
:100A0000180507070600006090A040A89068020340
:100A100003060104C0408003070706010020408050
:100A200080804020030707060100804020202040EE
:100A30008005050506000120A870A820050505060B
:100A400000012020F820200203030602FFC040809E
:100A5000050101060003F8020202060200C0C005FB
:100A60000505060001081020408005070706000064
:100A70007088888888887003070706010040C04096
:100A8000404040E00507070600007088087080803D
:100A9000F8050707060000F81020100808F0050701
:100AA0000706000010305090F810100507070600E8
:100AB00000F880F0080888700507070600007080BD
:100AC00080F0888870050707060000F808102020CD
:100AD0002020050707060000708888708888700548
:100AE0000707060000708888780808700205050668
:100AF0000200C0C000C0C00206060602FFC0C0005F
:100B0000C0408004070706000010204080402010ED
:100B1000050303060002F800F80407070601008039
:100B2000402010204080050707060000708808104C
:100B300020002005070706000070880868A8A87034
:100B4000050707060000708888F888888805070769
:100B5000060000F08888F08888F005070706000086
:100B600070888080808870050707060000F08888FC
:100B7000888888F0050707060000F88080F08080EC
:100B8000F8050707060000F88080F08080800507E0
:100B900007060000708880B888887005070706007F
:100BA00000888888F8888888010707060200808006
:100BB0008080808080050707060000381010101024
:100BC00090600507070600008890A0C0A0908805E7
:100BD0000707060000808080808080F805070706F0
:100BE000000088D8A888888888050707060000883C
:100BF00088C8A89888880507070600007088888834
:100C0000888870050707060000F08888F0808080DB
:100C100005070706000070888888A8906805070700
:100C2000060000F08888F0A09088050707060000FD
:100C3000788080700808F0050707060000F820207B
:100C400020202020050707060000888888888888DB
:100C500070050707060000888888888850200507E7
:100C6000070600008888888888A8500507070600BE
:100C7000008888502050888805070706000088886B
:100C80008850202020050707060000F808102040A3
:100C900080F8030707060100E08080808080E0057F
:100CA0000505060001804020100803070706010023
:100CB000E02020202020E0050303060004205088C7
:100CC000050101060000F802020206020580400547
:100CD00005050600007008788878050707060000FB
:100CE0008080B0C88888F005050506000070808007
:100CF0008870050707060000080868988888780546
:100D000005050600007088F88070050707060000DA
:100D10003048E0404040400506060600FF708888E5
:100D20007808700507070600008080B0C8888888AA
:100D30000107070602008000808080808003080889
:100D40000601FF200020202020A040040707060005
:100D500000808090A0C0A090030707060100C0405B
:100D600040404040E0050505060000D0A8A8A8A81E
:100D7000050505060000B0C8888888050505060039
:100D80000070888888700506060600FFF08888F0E5
:100D900080800506060600FF788888780808050523
:100DA00005060000B0C880808005050506000070BB
:100DB000807008F00407070600004040E040404013
:100DC0003005050506000088888898680505050631
:100DD000000088888850200505050600008888A83E
:100DE000A850050505060000885020508805060615
:100DF0000600FF888888780870050505060000F859
:100E0000102040F8030707060100204040804040C2
:100E10002001070706020080808080808080030711
:100E20000706010080404020404080050202060085
:100E300002689000000006000000000006000000AC
:100E40000000060000000000060000000000060090
:100E50000000000006000000000006000000000086
:100E60000600000000000600000000000600000070
:100E70000000060000000000060000000000060060
:100E80000000000006000000000006000000000056
:100E90000600000000000600000000000600000040
:100EA0000000060000000000060000000000060030
:100EB0000000000006000000000006000000000026
:100EC0000600000000000600000000000600000010
:100ED0000000060000000000060000000000060000
:100EE00000000000060000000000060000000000F6
:100EF00006000000000006000000000006000001DF
:100F000007070602008000808080808005070706B2
:100F100000002070A8A0A870200507070600003078
:100F20004040E04050A8050505060000887050705C
:100F300088050707060000885020F820F8200107E0
:100F40000706020080808000808080050808060077
:100F5000003048205050209060030101060107A096
:100F6000050707060000F888B8B8B888F80507072D
:100F7000060001700878887800F80505050600016C
:100F80002850A05028050303060001F808080202B3
:100F9000020602064080050707060000F888A888B8
:100FA00098A8F8050101060006F8040404060003E9
:100FB000609090600507070600002020F8202000C0
:100FC000F804050506000360902040F003050506BF
:100FD0000003E020E020E002020206020640800555
:100FE00008080600FF8888888898E8808005070739
:100FF0000600007898987818181802020206020273
:10100000C0C00202020602FF40800305050600037D
:1010100040C04040E00507070600017088888870DE
:1010200000F8050505060001A0502850A005070797
:101030000600008890A858B80808050707060000B1
:101040008890B848982038050808060000C040C0BD
:1010500048D838080805070706000020002040800F
:1010600088700508080600004020007088F888880D
:101070000508080600001020007088F88888050818
:10108000080600002050007088F8888805080806C7
:1010900000006890007088F888880508080600003D
:1010A0005000708888F888880508080600002050DD
:1010B000207088F888880507070600003860A0B807
:1010C000E0A0B80508080600FF70888080887020BE
:1010D00060050808060000402000F880F080F80550
:1010E0000808060000081000F880F080F8050808DD
:1010F000060000205000F880F080F8050707060081
:10110000005000F880F080F80308080601008040D5
:1011100000E0404040E0030808060100204000E0F5
:10112000404040E003080806010040A000E04040C5
:1011300040E0030707060100A000E0404040E00552
:101140000707060000704848E84848700508080688
:10115000000068900088C8A8988805080806000064
:1011600040207088888888700508080600001020D4
:101170007088888888700508080600002050007074
:1011800088888870050808060000689000708888C4
:1011900088700508080600005000708888888870EC
:1011A000050505060001885020508805080806003E
:1011B000FF1070A8A8A8A870400508080600004005
:1011C0002088888888887005080806000010208814
:1011D00088888888700508080600002050008888E4
:1011E000888870050808060000500088888888886C
:1011F00070050808060000102088502020202005D7
:1012000009090600FFC040704848704040E00408EB
:10121000080601FF609090A09090E0800508080605
:101220000000402000700878887805080806000053
:101230001020007008788878050808060000205003
:10124000007008788878050808060000689000702B
:10125000087888780507070600005000700878882D
:101260007805080806000020502070087888780566
:101270000606060000D02878A0A85005060606003D
:10128000FF7080887020600508080600004020007C
:101290007088F8807005080806000010200070882B
:1012A000F880700508080600002050007088F8805B
:1012B0007005070706000050007088F8807003086A
:1012C0000806010080400040C04040E003080806D6
:1012D000010020400040C04040E003080806010033
:1012E00040A00040C04040E0030707060100A00006
:1012F00040C04040E0050707060000A040A010786D
:101300008870050808060000689000B0C8888888C2
:1013100005080806000040200070888888700508CD
:1013200008060000102000708888887005080806EC
:1013300000002050007088888870050808060000AA
:1013400068900070888888700507070600005000C4
:1013500070888888700505050600012000F80020C7
:101360000507070600FF1070A8A8A8704005080828
:101370000600004020008888889868050808060054
:10138000001020008888889868050808060000205A
:101390005000888888986805070706000050008874
:1013A000888898680509090600FF10200088888849
:1013B000F808700407070601FFC04060506040E075
:1013C0000508080600FF50008888887808705A00D1
:1013D0005900580009200000000000000000000033
:1013E0000000007FFFE0000000000000000000009F
:1013F00000007000E000000000000000000000009D
:101400000061F86000000000000000000000000023
:1014100041F8200000000000000000000000004033
:10142000F02000000000000000000000000040600C
:10143000200000000000000000000000005801A093
:101440007F80003FC0000000004104005C63A0FBFF
:10145000C00079E0000000002082005EF7A0F3C029
:101460000076E0000000002082005EF7A0EBC000E4
:101470007EE0000000004104005C63A07B80003D32
:10148000C0000000008208005801A07B80003BC023
:1014900000000001041000406020FBC00077E00065
:1014A00000000104100040F020FBC00070E00000CC
:1014B000000082080041F820FFC0007FE00000002B
:1014C0000041040061F8603F00001F800000000040
:1014D0000000007000E01E00000F0000000001FF8F
:1014E000FF807FFFE00C0000060000000001FFFF0E
:1014F000800000000000000000000000000000006C
:101500007FFFE0000000000000000000000000700D
:1015100000E0000000000000000000000000630C7C
:1015200060000000000000000000000000470E20E6
:101530000000000000000000000000004F0F20002D
:1015400000000000000000000000005F0FA000008D
:10155000000000000000000000005E07A07F800087
:101560003FC000000000410400406020FBC0007943
:10157000E00000000020820040F020F3C00076E090
:101580000000000020820040F020EBC0007EE00060
:101590000000004104004060207B80003DC000004E
:1015A00000008208005E07A07B80003BC0000000B6
:1015B000010410005F0FA0FBC00077E000000001F5
:1015C0000410004F0F20FBC00070E00000000082FC
:1015D0000800470E20FFC0007FE00000000041042B
:1015E00000630C603F00001F80000000000000004E
:1015F0007000E01E00000F0000000001FFFF807F70
:10160000FFE00C0000060000000001FFFF8000006A
:101610000000000A0B02090C0D0E0807030401006C
:1016200000000000000000000000000000000000BA
:101630000000000000000000000000000012111077
:10164000000000000000000000000000000000009A
:1016500000000000000000486F6D652025732573B1
:101660002573206669727374002066697273740A48
:10167000005A0059005800486F6D652000534420FF
:1016800063617264206F6B0A006F70656E526F6FDA
:1016900074206661696C65640A00766F6C756D65AF
:1016A0002E696E6974206661696C65640A00534432
:1016B00020696E6974206661696C0A006175746FD7
:1016C00025692E67004D3234004D323320257300DA
:1016D00057726974696E6720746F2066696C653A29
:1016E00020006F70656E206661696C65642C204611
:1016F000696C653A20006F70656E206661696C6583
:10170000642C2046696C653A200046696C6520733C
:10171000656C65637465640A002053697A653A20D4
:101720000046696C65206F70656E65643A20006FD5
:1017300070656E206661696C65642C2046696C6515
:101740003A20002066696C653A20004E6F772000D1
:101750002220706F73002220706172656E743A22CD
:1017600000535542524F5554494E452043414C4C2D
:10177000207461726765743A22004B494C4C4544B1
:101780002E2000747279696E6720746F2063616C1B
:101790006C207375622D67636F64652066696C6584
:1017A00073207769746820746F6F206D616E792083
:1017B0006C6576656C732E204D4158206C6576659E
:1017C0006C2069733A004572726F723A001FFFFF16
:1017D000FFFFFFFF600000000001FF40000000006D
:1017E00000FF8000000000007F83CF00000C303F2E
:1017F00087FF80000C301F867980000C000F8C3032
:10180000C7838C30E78C30CFC7CC31F38C30DCEC25
:10181000EC33B98C30D86C6C33198C30D06C0C3301
:10182000198C30D86C0C33198C30DC6C0E3B198C55
:1018300030CF7C079F198C30C77C038F1940000084
:1018400000000002600000000000061FFFFFFFFF15
:10185000FFF82020506C616E6E6572427566666599
:101860007242797465733A20002046726565204D96
:10187000656D6F72793A2000436F6D70696C6564B5
:101880003A204A616E20333020323031380A00204D
:101890007C20417574686F723A2028416C657068CD
:1018A000204F626A6563747320496E632E2C204C4E
:1018B000756C7A426F7420476974205265706F733B
:1018C00069746F7279290A004A616E2033302032C0
:1018D00030313830393A30353A303100204C61738C
:1018E0007420557064617465643A2000312E312E85
:1018F000350A004D61726C696E0020536F66747713
:101900006172652052657365740A002057617463C3
:1019100068646F672052657365740A002042726FB5
:10192000776E206F75742052657365740A002045C8
:10193000787465726E616C2052657365740A00502C
:101940006F77657255700A0073746172740A00656E
:1019500072726F722077726974696E6720746F207B
:1019600066696C650A00456E6473746F7073202538
:101970006320256320256320256300205A3A002038
:10198000593A0020583A00656E6473746F70732082
:101990006869743A2000446F6E6520736176696EE1
:1019A000672066696C652E0A004D3239004D36306D
:1019B0003020486F74656E6420746F6F20636F6CA5
:1019C0006420746F206368616E67652066696C616E
:1019D0006D656E740A004B494C4C45442E20004501
:1019E000787472756465206D6F72650052657375E9
:1019F0006D65207072696E7400524553554D4520D7
:101A00004F5054494F4E533A0020204E6F7A7A6C13
:101A1000653A20006368616E6765006F66207468D0
:101A2000652066696C616D656E740057616974202C
:101A3000666F72207374617274005052494E542064
:101A40005041555345440020204E6F7A7A6C653AD8
:101A50002000200066696C616D656E7420756E6C87
:101A60006F6164005761697420666F72005052495B
:101A70004E54205041555345440020204E6F7A7AF1
:101A80006C653A20002000506C65617365207761B9
:101A900069742E2E2E0048656174696E67206E6F22
:101AA0007A7A6C65005052494E5420504155534546
:101AB000440020204E6F7A7A6C653A20002000683E
:101AC000656174206E6F7A7A6C652E005072657352
:101AD0007320627574746F6E20746F005052494E9B
:101AE00054205041555345440020204E6F7A7A6C63
:101AF000653A2000746F20636F6E74696E75652E91
:101B00002E2E00616E64207072657373206275748E
:101B1000746F6E00496E736572742066696C616DD6
:101B2000656E74005052494E5420504155534544FF
:101B30000020204E6F7A7A6C653A2000200066699A
:101B40006C616D656E74206C6F61640057616974BF
:101B500020666F72005052494E54205041555345F3
:101B6000440020204E6F7A7A6C653A20002000668F
:101B7000696C616D656E742065787472756465005A
:101B80005761697420666F72005052494E5420505C
:101B9000415553454400746F20726573756D65003F
:101BA0005761697420666F72207072696E7400509C
:101BB00052494E5420504155534544007C3C3E5EB2
:101BC0002B3D3F2F5B5D3B2C2A225C004D6F7665E1
:101BD00020617869730044697361626C6520737475
:101BE000657070657273004D3834004175746F20F4
:101BF000686F6D6500473238004D61696E004D3584
:101C000030320A4D353030004C6F6164207365749A
:101C100074696E677300526573746F7265206661D4
:101C2000696C736166650053746F726520736574C7
:101C300074696E677300416476616E6365642053F6
:101C4000657474696E6773004D61696E004D36305E
:101C500030204230205431004D3630302042302088
:101C6000543000466C6F77203200466C6F7720321C
:101C700000466C6F77203100466C6F77203100464C
:101C8000616E20737065656420310046616E20735B
:101C90007065656420310042656400426564004EF1
:101CA0006F7A7A6C652032004E6F7A7A6C652032DA
:101CB000004E6F7A7A6C652031004E6F7A7A6C65CF
:101CC0002031005370656564005370656564004D94
:101CD00061696E004D6F76652058004D6F76652006
:101CE00059004D6F7665205A0045787472756465A9
:101CF000723200457874727564657231004D6F768A
:101D00006520302E316D6D004D6F766520316D6D23
:101D1000004D6F76652031306D6D004D6F7665201A
:101D200061786973004578747275646572004D6FEF
:101D30007665205A004D6F76652059004D6F7665A7
:101D400020580020496E76616C6964206578747251
:101D5000756465722000000000C0000000000000F3
:101D6000000000008F4300008A4300007A435A209D
:101D700070726F6265206F75742E206265640A0050
:101D80005A2070726F6265206F75742E20626564D0
:101D900000486F6D652058592066697273740A0097
:101DA000486F6D6520585920666972737400256903
:101DB000730025696D2025697300256968202569F0
:101DC0006D202569730025696420256968202569CF
:101DD0006D202569730025697920256964202569AE
:101DE000682025696D20256973005072696E742022
:101DF00074696D653A2000000125301D0CFF243107
:101E00001C0BFF232F1B0AFFFF04030608020222FC
:101E10002B1A4142212A193F40033809FF3607FF98
:101E20003728294527444350726F7465637465648D
:101E30002050696E0A00202F002040002042403AC6
:101E40000020403A0045787472756465723200452E
:101E500078747275646572004D6F7665205A004D16
:101E60006F76652059004D6F76652058004D6F766E
:101E7000656D656E7400436F6F6C646F776E0046BE
:101E8000616E20737065656420310046616E207359
:101E90007065656420310042656400426564004EEF
:101EA0006F7A7A6C652032004E6F7A7A6C652032D8
:101EB000004E6F7A7A6C652031004E6F7A7A6C65CD
:101EC0002031004D61696E005654726176206D6953
:101ED0006E005654726176206D696E0056547261C0
:101EE00076206D696E00566D696E00566D696E00E4
:101EF000566D696E00566D617820453200566D61F1
:101F00007820453200566D617820453200566D616B
:101F10007820453100566D617820453100566D615D
:101F20007820453100566D6178205A00566D6178F1
:101F3000205A00566D6178205A00566D61782059FC
:101F400000566D6178205900566D61782059005611
:101F50006D6178205800566D6178205800566D618B
:101F6000782058004D6F74696F6E00416D61782064
:101F7000453200416D617820453200416D61782025
:101F8000453100416D617820453100416D61782017
:101F90005A00416D6178205A00416D6178205900E6
:101FA000416D6178205900416D6178205800416D84
:101FB0006178205800412D74726176656C00412D66
:101FC00074726176656C00412D7265747261637420
:101FD00000412D7265747261637400416363656CC6
:101FE00000416363656C004D6F74696F6E006F6BC9
:101FF00000436F6F6C696E6720646F6E652E0048DA
:10200000656174696E6720646F6E652E0020573AB3
:102010000045787472756465722025692025730007
:102020004C756C7A426F742054415A203520726589
:102030006164792E004C756C7A426F742054415A59
:102040002035204F66662E00205A3A0020593A006B
:1020500020436F756E7420583A0020453A00205A8C
:102060003A0020593A00583A002F2F200053657447
:1020700074696E672054726176656C204163636594
:102080006C65726174696F6E3A200053657474698F
:102090006E67205265747261637420416363656C7E
:1020A00065726174696F6E3A200053657474696E6D
:1020B00067205072696E7420416363656C6572615C
:1020C00074696F6E3A200053657474696E672050AE
:1020D00072696E7420616E642054726176656C2042
:1020E000416363656C65726174696F6E3A200020AC
:1020F0005A00205900580020204D61783A200020D5
:102100005A00205900580020204D696E3A20004F97
:102110006E20004F666600536F667420656E6473B0
:10212000746F70733A2000486F74656E64206F6638
:1021300066736574733A0020746F6F206C6F6E67FE
:1021400020657874727573696F6E2070726576653C
:102150006E7465640A0020636F6C64206578747225
:102160007573696F6E2070726576656E7465640A4A
:102170000056652D6A65726B0056652D6A65726B37
:102180000056652D6A65726B00567A2D6A65726B12
:1021900000567A2D6A65726B0056792D6A65726BEE
:1021A0000056792D6A65726B0056792D6A65726BDF
:1021B0000056782D6A65726B0056782D6A65726BD1
:1021C0000056782D6A65726B004D6F74696F6E00F2
:1021D000453273746570732F6D6D0045327374658D
:1021E00070732F6D6D00453173746570732F6D6D55
:1021F00000453173746570732F6D6D005A7374658B
:1022000070732F6D6D005A73746570732F6D6D0050
:102210005973746570732F6D6D00597374657073A5
:102220002F6D6D005873746570732F6D6D0058734A
:10223000746570732F6D6D004D6F74696F6E004F14
:102240006666004F6E2000456E6473746F70206187
:10225000626F72740053746570732F6D6D004A6500
:10226000726B00416363656C65726174696F6E00C7
:1022700056656C6F6369747900416476616E63655D
:10228000642053657474696E67730043616E6E6F8A
:102290007420656E746572207375626469723A2089
:1022A00000022E2E004D61696E0020204E6F7A7A5A
:1022B0006C653A200020004261636B004D696E69D5
:1022C0006D756D2054656D70206973203132302E2C
:1022D0000048656174696E67206661696C656400B9
:1022E00043616E6E6F74206F70656E2073756264EB
:1022F000697220006563686F3A00544845524D4149
:102300004C2052554E415741592042454400546893
:1023100065726D616C2052756E6177617900544809
:1023200045524D414C2052554E415741592045315F
:1023300000544845524D414C2052554E4157415949
:102340002045300000002200250028002B002E0030
:102350003100340002010000050108010B010000FA
:102360002100240027002A002D0030003300010145
:102370000000040107010A01050505050705080815
:102380000808020202020A0A0808040404040101FF
:102390000101010101010303030303030303040714
:1023A00007070C0C0C0C0C0C0C0C020202020606AB
:1023B0000606060606060B0B0B0B0B0B0B0B01029E
:1023C0001020200808102040102040800201020147
:1023D00008040201010204081020408080402010FF
:1023E0000804020180040201804020100804020158
:1023F00008040201010204081020408001020408C0
:1024000010204080436172642072656D6F76656450
:10241000004361726420696E7365727465640000C4
:10242000060900FE06018902FE20FFFE07FE06FEE9
:10243000000000060007010606060200808080807A
:102440000080030303060103A0A0A0050707060000
:10245000FF5050F850F850500509090600FE207052
:10246000A8A07028A870200608080600FF40A84809
:1024700010204854080507070600FF6090906098F8
:1024800090680103030602038080800207070602AA
:10249000FF408080808080400207070602FF804066
:1024A00040404040800505050600008850F85088EF
:1024B0000505050600002020F8202002040406027D
:1024C000FEC0404080050101060002F8020202063B
:1024D0000200C0C0040606060100101020408080E3
:1024E00004060606010060909090906003060606C0
:1024F000010040C0404040E0040606060100609034
:10250000102040F0040606060100F020601010E0E4
:1025100005060606000010305090F8100406060666
:102520000100F080E01010E0040606060100608063
:10253000E0909060040606060100F0101020404074
:10254000040606060100609060909060040606068E
:102550000100609090701060020505060200C0C086
:1025600000C0C00207070602FEC0C000C040408095
:1025700005050506000018608060180503030600C5
:1025800001F800F8050505060000C0300830C00459
:10259000070706010060901060400040050606062F
:1025A00000007090A8B0807005060606000020505C
:1025B00088F88888050606060000F088F08888F00C
:1025C00004060606010060908080906004060606FE
:1025D0000100E090909090E0040606060100F08073
:1025E000E08080F0040606060100F080E080808034
:1025F000040606060100609080B09060040606069E
:1026000001009090F0909090030606060100E040D3
:10261000404040E0050606060000381010109060AB
:1026200004060606010090A0C0A0909004060606CD
:1026300001008080808080F005060606000088D8B2
:10264000A8A8888804060606010090D0B090909053
:10265000050606060000708888888870040606064D
:102660000100E09090E080800407070601FF609081
:1026700090D0B06010040606060100E09090E09053
:102680009004060606010060904020906005060652
:10269000060000F8202020202004060606010090F5
:1026A0009090909060040606060100909090F06073
:1026B000600506060600008888A8A8D888050606D2
:1026C0000600008850202050880506060600008875
:1026D0008850202020040606060100F010204080CB
:1026E000F0030606060100E080808080E004060614
:1026F000060100808040201010030606060100E05D
:1027000020202020E0050303060003205088050157
:10271000010600FEF80202020602048040040404DE
:10272000060100709090700406060601008080E0AB
:102730009090E00404040601007080807004060696
:1027400006010010107090907004040406010060EF
:10275000B0C070040606060100205040E04040046E
:1027600006060601FE6090907010600406060601E1
:10277000008080E09090900306060601004000C0B3
:102780004040E00308080601FE200060202020A051
:10279000400406060601008080A0C0A09003060643
:1027A000060100C040404040E0050404060000D09F
:1027B000A8A888040404060100E090909004040492
:1027C000060100609090600406060601FEE090900D
:1027D000E080800406060601FE70909070101004E0
:1027E0000404060100A0D0808004040406010070E7
:1027F000C030E00406060601004040E040502004DE
:1028000004040601009090907004040406010090F6
:1028100090606005040406000088A8A85004040421
:10282000060100906060900406060601FE909090FC
:10283000709060040404060100F02040F0030707D4
:10284000060100204040804040200107070602FFAB
:1028500080808080808080030707060100804040E0
:102860002040408004020206010350A0FFFFFFFF4A
:10287000FFFFFFFFFFFFFFFFFFFFFFFFFFFFFFFF68
:10288000FFFFFFFFFFFFFFFFFFFFFFFFFF00000055
:102890000600070106060602008000808080800492
:1028A00006060601FF2070A0A0702005070706009D
:1028B000FF304840F04040F8050505060000A850EC
:1028C0008850A80506060600008850F820F8200168
:1028D00007070602FF8080800080808004070706CB
:1028E00001FF708060906010E0030101060105A007
:1028F000060707060000788494A4948478030505ED
:1029000006010160A06000E00505050600002850F2
:10291000A05028040303060100F010100401010672
:102920000102F00607070600007884B4A4A48478A6
:10293000040101060105F004030306010260906032
:102940000507070600FF2020F8202000F8030505F2
:1029500006010140A02040E0030505060101C0205A
:102960004020C00202020602044080040505060160
:10297000FF9090B0D08005060606000078E8E86871
:102980002828010101060202800202020602FE401E
:102990008003050506010140C04040E0030505062F
:1029A000010140A04000E0050505060000A05028F8
:1029B00050A00508080600FF40C040507030781055
:1029C0000508080600FF40C0405068081038050898
:1029D000080600FFC0204030F030781004070706DA
:1029E000010020002060809060050707060000407D
:1029F000202050708888050707060000102020500E
:102A000070888805070706000020502050708888CD
:102A10000507070600002850205070888805070722
:102A20000600005000205070888805070706000047
:102A30002050205070888805060606000078A0F017
:102A4000A0A0B80408080601FE6090808090602075
:102A5000400407070601004020F080E080F00407F2
:102A6000070601002040F080E080F004070706011F
:102A7000002050F080E080F00407070601005000BD
:102A8000F080E080F00307070601008040E040404E
:102A900040E00307070601002040E0404040E0031B
:102AA000070706010040A0E0404040E0030707069A
:102AB0000100A000E0404040E0050606060000706E
:102AC00048E848487004070706010050A090D0B0BD
:102AD00090900407070601004020609090906004E9
:102AE00007070601002040609090906004070706E9
:102AF000010020506090909060040707060100508C
:102B0000A06090909060040707060100500060905C
:102B10009090600505050600008850205088040844
:102B2000080601FF1070B0B0D0D0E080040707069F
:102B3000010040209090909060040707060100205B
:102B400040909090906004070706010020509090FC
:102B500090906004070706010050009090909060EC
:102B600005070706000010208850202020040606D4
:102B700006010080E09090E08004060606010060F7
:102B800090A0A090A00407070601004020007090CC
:102B900090700407070601002040007090907004B8
:102BA0000707060100205000709090700407070688
:102BB000010050A0007090907004060606010050BD
:102BC000007090907004070706010020502070905C
:102BD000907005040406000070A8B078040606068C
:102BE00001FE70808070204004070706010040202D
:102BF0000060B0C07004070706010020400060B00C
:102C0000C07004070706010020500060B0C07004C7
:102C10000606060100500060B0C0700307070601F9
:102C200000804000C04040E003070706010020404C
:102C300000C04040E003070706010040A000C0407C
:102C400040E0030606060100A000C04040E0040783
:102C500007060100306010709090600407070601BD
:102C60000050A000E090909004070706010040206B
:102C7000006090906004070706010020400060900B
:102C800090600407070601002050006090906004E7
:102C9000070706010050A000609090600406060639
:102CA00001005000609090600505050600002000BE
:102CB000F8002004040406010070B0D0E004070707
:102CC0000601004020009090907004070706010064
:102CD00020400090909070040707060100205000EB
:102CE000909090700406060601005000909090703D
:102CF0000409090601FE2040009090907090600445
:102D000008080601FE8080E09090E08080040808BA
:102D10000601FE50009090907090601000C9021063
:102D2000012C014001220170011801B0010E01F0D7
:102D30000104015002FA00B002F0003003E600D0B6
:102D400003DC009004D2007005C800A006BE00009D
:102D500008B400B009AA00D00BA000600E96006075
:102D6000118C000015820020197800C01D6E00A093
:102D7000226400B0275A00902C500000314600E039
:102D8000343C0010383200903A2800603C1E00A00D
:102D90003D1400803E0A00203F00006265640A0086
:102DA0002C2073797374656D2073746F7070656413
:102DB00021204865617465725F49443A2000486586
:102DC0006174696E67206661696C65642042454480
:102DD0000048656174696E67206661696C656400AE
:102DE00048656174696E67206661696C6564004856
:102DF000656174696E67206661696C656420453140
:102E00000048656174696E67206661696C6564205D
:102E10004530001000AD0330016A0150022B0170F3
:102E2000030A019004F500B005E500D006D800F0D3
:102E300007CE001009C500300ABE00500BB7007065
:102E40000CB100900DAB00B00EA600D00FA200F0A8
:102E5000109D0010129900301395005014920070CC
:102E6000158E0090168B00B0178700D0188400F0E4
:102E7000198100101B7E00301C7B00501D790070F2
:102E80001E7600901F7300B0207000D0216E00F0FD
:102E9000226B001024690030256600502663007004
:102EA00027610090285E00B0295C00D02A5900F00C
:102EB0002B5600102D5400302E5100502F4E007014
:102EC000304B0090314800B0324500D0334200F022
:102ED000343E0010363B0030373700503833007036
:102EE000392E00903A2900B03B2300D03C1B00F063
:102EF0003D1100103F0100F03F00004572723A2082
:102F00004D494E54454D5020424544004D494E5484
:102F1000454D50207472696767657265640045723B
:102F2000723A204D494E54454D502045310045726E
:102F3000723A204D494E54454D502045300045725F
:102F4000723A204D415854454D5020424544004D61
:102F5000415854454D5020747269676765726564C5
:102F6000004572723A204D415854454D502045312C
:102F7000004572723A204D415854454D502045301D
:102F8000004572726F722077726974696E6720747F
:102F90006F20454550524F4D210A00290A002062FA
:102FA000797465733B2063726320005365747469A0
:102FB0006E67732053746F72656420280020286345
:102FC000616C63756C6174656429210A0020213D80
:102FD0002000454550524F4D20435243206D6973A8
:102FE0006D61746368202D202873746F7265642985
:102FF0002000290A002062797465733B20637263A4
:1030000020002073746F7265642073657474696E38
:103010006773207265747269657665642028002084
:103020004D61726C696E3D563430290A0028454561
:1030300050524F4D3D00454550524F4D20766572E0
:1030400073696F6E206D69736D617463682000240D
:10305000F4D43050C38E20C2A24017828B7011125C
:103060007A910D816CD90AA861E108C75866076199
:103070005143061E4B5D05C145A7041A41110409C1
:103080003D9803713931034036DB0265339102D438
:10309000305402802E1D02632CEE01752AC501B04A
:1030A00028A001102781018F2564012B244B01E00A
:1030B000223401AC211F018D200D01801FFC0084F2
:1030C0001EED00971DDF00B81CD200E61BC60020D5
:1030D0001BBC00641AB200B219A8000A19A0006A49
:1030E000189900D117910040178B00B51684003154
:1030F000167E00B31579003A157300C7146F005897
:10310000146A00EE1366008813630025135E00C77F
:10311000125B006C12570015125400C1115100705F
:10312000114F0021114B00D61049008D1047004669
:1031300010440002104200C00F4000800F3E0042C9
:103140000F3C00060F3B00CB0E3800930E37005C9F
:103150000E3500270E3400F30D3200C10D31009002
:103160000D3000600D2E00320D2D00050D2C00D904
:103170000C2B00AE0C2900850C29005C0C270035B7
:103180000C27000E0C2600E80B2400C40B2400A022
:103190000B23007D0B23005A0B2100390B21001853
:1031A0000B2000F80A1F00D90A1E00BB0A1E009D52
:1031B0000A1D00800A1D00630A1C00470A1B002C20
:1031C0000A1B00110A1A00F7091A00DD091900C4C8
:1031D000091900AB091900920917007B091800634F
:1031E0000917004C09160036091600200916000AB6
:1031F000091500F5081500E0081400CC081400B803
:10320000081400A4081400900813007D0812006B35
:103210000813005808120046081200340811002351
:103220000811001208110001081100F0071000E059
:10323000071000D0071000C0071000B0070F00A152
:1032400007100091070E0083070F0074070F006539
:10325000070E0057070E0049070E003B070D002E12
:10326000070E0020070D0013070D0006070D00F9DB
:10327000060C00ED060D00E0060C00D4060C00C89C
:10328000060C00BC060C00B0060C00A4060B00994E
:10329000060C008D060B0082060B0077060B006CF7
:1032A000060B0061060A0057060B004C060A004296
:1032B000060A0038060A002E060A0024060A001A2A
:1032C000060A001006090007060A00FD050900F4B9
:1032D000050900EB050900E2050900D9050900D040
:1032E000050900C7050900BE050900B5050800ADC0
:1032F000050800A50509009C050800940508008C38
:10330000050800840508007C050800740508006CA9
:10331000050700650508005D050700560508004E15
:10332000050700470507004005080038050700317C
:103330000507002A050700230507001C05060016DF
:103340000507000F0507000805060002050700FB3A
:10335000040600F5040700EE040600E8040600E297
:10336000040700DB040600D5040600CF040600C9EC
:10337000040600C3040600BD040600B7040600B13D
:10338000040500AC040600A6040600A00405009B8A
:1033900004060095040500900406008A04050085D3
:1033A000040500800406007A040500750405007019
:1033B0000405006B04050066040500610405005C5B
:1033C00004050057040500520405004D040500489B
:1033D000040500430405003E0404003A04050035DA
:1033E000040500300404002C040500270404002315
:1033F0000405001E0404001A04040016040500114C
:103400000404000D04040009040500040404000081
:10341000040400FC030400F8030400F4030400F0B7
:10342000030400EC030400E8030400E4030400E0E8
:10343000030400DC030400D8030400D4030400D018
:10344000030400CC030400C8030300C503030024E5
:10345000F404D9201BC40C5C0E9804C4095F0265F7
:10346000077101F405F900FB04B30048048700C1AB
:103470000369005803550003034500BE023A008467
:1034800002310053022A002902250004022000E430
:10349000011C00C8011900AF011700980114008435
:1034A000011300710110006101100051010E004371
:1034B000010D0036010B002B010B0020010B001544
:1034C0000109000C01090003010800FB000800F3DA
:1034D000000800EB000700E4000600DE000600D84C
:1034E000000600D2000600CC000500C7000500C29F
:1034F000000500BD000400B9000400B5000400B1DF
:10350000000400AD000400A9000400A5000300A20F
:103510000003009F0004009B000300980003009537
:1035200000020093000300900003008D0002008B56
:10353000000300880002008600020084000300816E
:103540000002007F0002007D0002007B0002007983
:103550000002007700010076000200740002007291
:10356000000100710002006F0002006D0001006C9C
:103570000002006A000100690002006700010066A5
:1035800000010065000100640002006200010061AA
:10359000000100600001005F0002005D0001005CAE
:1035A0000001005B0001005A0001005900010058B1
:1035B00000010057000100560001005500010054B1
:1035C00000010053000000530001005200010051AF
:1035D000000100500001004F0001004E0000004EAD
:1035E0000001004D0001004C0001004B0000004BA9
:1035F0000001004A000100490001004800000048A5
:10360000000100470001004600000046000100459F
:103610000000004500010044000100430000004399
:103620000001004200000042000100410000004192
:10363000000100400001003F0000003F0001003E8B
:103640000000003E0001003D0000003D0001003C84
:103650000000003C0000003C0001003B0000003B7B
:103660000001003A0000003A000100390000003972
:103670000001003800000038000000380001003769
:103680000000003700010036000000360000003660
:103690000001003500000035000000350001003455
:1036A000000000340000003400010033000000334B
:1036B0000000003300010032000000320000003240
:1036C0000001003100000031000000310001003035
:1036D00000000030000000300001002F0000002F2B
:1036E0000000002F0000002F0001002E0000002E1F
:1036F0000000002E0001002D0000002D0000002D14
:103700000000002D0001002C0000002C0000002C07
:103710000000002C0001002B0000002B0000002BFB
:103720000000002B0001002A0000002A0000002AEF
:103730000000002A000100290000002900000029E3
:1037400000000029000000290001002800000028D6
:1037500000000028000000280000002800010027C9
:1037600000000027000000270000002700000027BD
:1037700000010026000000260000002600000026B0
:1037800000000026000100250000002500000025A3
:103790000000002500000025000000250001002495
:1037A0000000002400000024000000240000002489
:1037B000000100230000002300000023000000237C
:1037C000000000230000002300000023000100226D
:1037D0000000002200000022000000220000002261
:1037E0000000002200010021000000210000002153
:1037F0000000002100000021000000210000002145
:103800000001002000000020000000200000002037
:103810000000002000000020000000200000002028
:103820000001001F0000001F0000001F0000001F1B
:103830000000001F0000001F0000001F0001001E0C
:103840000000001E0000001E0000001E0000004DD1
:10385000383420582059205A204500526573656E2F
:10386000643A20002042002050006F6B004B494C0E
:103870004C45442E20004B494C4C206361757365C8
:1038800064206279204B494C4C20627574746F6ED1
:103890002F70696E0A004B494C4C45442E20004B5A
:1038A000494C4C2063617573656420627920746FA4
:1038B0006F206D75636820696E6163746976652039
:1038C00074696D65202D2063757272656E74206356
:1038D0006F6D6D616E643A2000506C656173652098
:1038E0007265736574005052494E544552204841E8
:1038F0004C544544005072696E7465722068616C66
:103900007465642E206B696C6C28292063616C6C73
:103910006564210A00656E7175657565696E67205D
:103920002200000000C000000000000000000000B5
:10393000484200004842000040400000000057613B
:10394000726E696E673A20486F6D696E67204275C6
:103950006D702044697669736F72203C20310A00D3
:103960000202040000A0400000A04000000040004F
:1039700000904300008A4300007A43FFFFFF416349
:10398000746976652045787472756465723A2000B2
:103990000201050800FF060121023520FFFF07FF95
:1039A00006FF090050221656808080800080153363
:1039B00053A0A0A00257575050F850F8505002574B
:1039C000572070A07028702013355580A040A0208B
:1039D00002475740A0A040A0A050251353808080EC
:1039E00012265640808080804012265680404040FB
:1039F00040800245559060F060900255552020F8B7
:103A00002020113353604080044151F01133534062
:103A1000E04002465610102040808012365640A0EA
:103A2000A0A0A04012365640C0404040E00246569A
:103A30006090106080F0024656F0206010906002A6
:103A400046562060A0F02020024656F080E01090FC
:103A5000600246566080E0909060024656F010206A
:103A6000204040024656609060909060024656604A
:103A70009090701060122555C0C000C0C01136561D
:103A800060600060408012365620408080402003F5
:103A90004353F000F012365680402020408012360A
:103AA0005640A020400040015858304898A8A8909F
:103AB0004030024656609090F09090024656E0905A
:103AC000E09090E0024656609080809060024656FA
:103AD000E090909090E0024656F080E08080F00206
:103AE0004656F080E0808080024656609080B0901C
:103AF000600246569090F0909090123656E040400A
:103B00004040E002465670202020A04002465690D9
:103B1000A0C0A0A0900246568080808080F002461F
:103B20005690F0F090909002465690D0F0B0B09041
:103B3000024656609090909060024656E09090E069
:103B40008080014757609090D0B06010024656E0E8
:103B50009090E0909002465660904020906012361F
:103B600056E0404040404002465690909090906011
:103B7000024656909090906060024656909090F069
:103B8000F090024656909060609090025656888859
:103B900050202020024656F010204080F012365669
:103BA000E080808080E00246568080402010101225
:103BB0003656E020202020E016325240A00141512C
:103BC000F016225280400244547090907002465683
:103BD0008080E09090E0123454608080600246560D
:103BE00010107090907002445460B0C0600246564D
:103BF000205040E040400145556090701060024602
:103C0000568080E09090901236564000C04040E0D0
:103C10001137572000202020A04002465680809077
:103C2000E09090123656C040404040E0025454D0DC
:103C3000A8A8A8024454E090909002445460909048
:103C400060014555E090E08080014555709070100E
:103C500010024454A0D0808012345460C020C002AE
:103C600046564040E04050200244549090907012DC
:103C70003454A0A0A04002545488A8A85002445430
:103C8000906060900145559090709060024454F0AF
:103C90002040F0024757304020C0204030221656C6
:103CA000808080808080024757C02040304020C004
:103CB00006425250A0FFFFFFFFFFFFFFFFFFFFFF85
:103CC000FFFFFFFFFFFFFFFFFFFFFFFFFFFFFFFF04
:103CD000FFFFFFFFFFFF0900502216568000808083
:103CE00080800146562070A0A070200246562050C9
:103CF000E04050A002555588705070880256568892
:103D000050F820F8202217578080800080808002A1
:103D100047577080E0907010E0173151A00256565E
:103D200070A8C8C8A87014355560A06000E00343AF
:103D30005350A050123353E02020143151E002566A
:103D40005670E8D8E8D870173151E015335340A0C9
:103D50004012355540E04000E014355540A0204069
:103D6000E0143555C020C020C016225240800145C5
:103D700055909090E08002565678E8E8682828240C
:103D8000115180112252408014355540C04040E00E
:103D900014355540A04000E0034353A050A0024713
:103DA00057808080A060F0200247578080A0D0100C
:103DB000207002475780408060A0F02012365640A5
:103DC000004080A04002475740206090F090900251
:103DD000475720406090F090900247576090609065
:103DE000F0909002475750A06090F0909002475793
:103DF00090006090F0909002475760906090F09033
:103E00009002465670A0A0F0A0B001475760908085
:103E1000809060400247574020F080E080F00247E9
:103E2000572040F080E080F00247576090F080E03B
:103E300080F00247579000F080E080F01237578002
:103E400040E0404040E01237572040E0404040E032
:103E500012375740A0E0404040E0123757A000E042
:103E6000404040E00256567048E8484870024757C4
:103E700050A090D0B0909002475740206090909012
:103E800060024757204060909090600247576090D2
:103E9000609090906002475750A0609090906002B0
:103EA000475790006090909060123353A040A0025A
:103EB000465670B0B0D0D0E0024757402090909066
:103EC0009060024757204090909090600247576062
:103ED00090909090906002475790009090909060E2
:103EE0000257571020885020202002465680E0902C
:103EF00090E0800246566090A0A090A002475740F4
:103F00002000709090700247572040007090907091
:103F10000247572050007090907002475750A00001
:103F20007090907002465650007090907002475703
:103F300060906070909070025454F068B0781135C1
:103F400055608080604002475740200060B0C060EC
:103F500002475720400060B0C060024757609000A1
:103F600060B0C060024656500060B0C06012375763
:103F7000804000C04040E0123757204000C0404021
:103F8000E012375740A000C04040E0123656A00073
:103F9000C04040E0024757A040A010709060024728
:103FA0005750A000E090909002475740200060904A
:103FB0009060024757204000609090600247576031
:103FC00090006090906002475750A0006090906011
:103FD0000246569000609090601235554000E00017
:103FE0004002445470B0D0E0024757402000909007
:103FF00090700247572040009090907002475760A1
:1040000090009090907002465690009090907001B1
:10401000485820400090907090600147578080E0A1
:1040200090E080800147579000909070906001056B
:104030000700FE0500FB01F220FFFE05FE05FE0263
:1040400000400215258080800080053242A0A00239
:10405000556550F850F8500146562070C030E020A9
:104060000255659010204048025565608068906850
:10407000051222808002253540808080400225354F
:104080008040404080043343A040A003334340E0DD
:10409000400122324080043141E00211218002556A
:1040A0006508102040800245556090909060022580
:1040B00035C040404040024555E0106080F0024568
:1040C00055E0106010E00245552060A0F020024548
:1040D00055F080E010E00245556080E090600245B8
:1040E00055F01020404002455560906090600245B8
:1040F00055609070106003132380008002142480A8
:104100000080800235452040804020033343E0009A
:10411000E00235458040204080024555E0106000B7
:10412000400255657088B8A870024555609090F0BF
:1041300090024555E090E090E00235456080808037
:1041400060024555E0909090E0023545E080E080C7
:10415000E0023545E080E080800245557080B090F7
:10416000700245559090F09090023545E0404040F7
:10417000E0024555301010906002455590A0C0A057
:104180009002354580808080E002556588D8A888F7
:104190008802455590D0B09090024555609090901F
:1041A00060024555E09090E0800146566090909006
:1041B0006010024555E09090E09002455570806097
:1041C00010E0023545E04040404002455590909057
:1041D00090600245559090A0A04002556588A8A81F
:1041E000A85002455590906090900245559090706F
:1041F0001060023545E0204080E0022535C0808017
:1042000080C00255658040201008022535C040401E
:1042100040C005324240A0024151F00522328040A8
:104220000244547090907002455580E09090E002F6
:104230003444608080600245551070909070024454
:104240005460B0C0600235452040E0404000465612
:1042500070909070106002455580E090909002152B
:10426000258000808080002737400040404040800B
:104270000245558090A0E0900215258080808080C6
:10428000025464F0A8A8A8024454E090909002441C
:104290005460909060004656E09090E08080004628
:1042A00056709090701010023444A0C08080024478
:1042B0005470C030E002354540E040402002445494
:1042C000909090700244549090A040025464A8A82A
:1042D0005050023444A04040A00046569090907048
:1042E0001060024454F02040F002354560408040A8
:1042F000600215258080808080023545C0402040C6
:10430000C005425250A0FFFFFFFFFFFFFFFFFFFF6E
:10431000FFFFFFFFFFFFFFFFFFFFFFFFFFFFFFFFAD
:10432000FFFFFFFFFFFFFF020040FFFFFFFFFFFF58
:10433000FFFFFFFFFFFFFFFFFFFFFFFFFFFFFFFF8D
:10434000FFFFFFFFFFFFFFFFFFFFFFFFFFFFFFFF7D
:10435000FFFFFFFFFFFFFFFFFFFFFFFFFFFFFFFF6D
:10436000FFFFFFFFFFFFFFFFFFFFFFFFFFFFFFFF5D
:10437000FFFFFFFFFFFFFFFFFFFFFFFFFFFFFFFF4D
:10438000FFFFFFFFFFFFFFFFFF01060D00FE09011A
:104390006602D620FFFE0BFE0AFE0D0060221969A0
:1043A000808080808080800080183363A0A0A0037C
:1043B00057675050F850F850500259692078A0A023
:1043C000702828F02002596948A85010204050A8B1
:1043D0009002586840A0A040A0989068281363807D
:1043E0008080113B6B204040808080808040402056
:1043F000113B6B804040202020202040408006550B
:104400006520A870A8200455652020F820201133CD
:1044100063604080065161F811336340E040025907
:104420006908081010204040808002596920508897
:104430008888888850200259692060A02020202088
:1044400020F80259697088880810204080F80259C5
:1044500069F8081020700808887002596910103037
:10446000505090F81010025969F88080B0C80808C0
:10447000887002596970888080F088888870025935
:1044800069F808101020204040400259697088885F
:1044900088708888887002596970888888780808C8
:1044A000887011386840E040000040E040113868F2
:1044B00040E04000006040800259690810204080C0
:1044C00040201008045464F80000F8025969804044
:1044D0002010081020408002596970888808102038
:1044E00020002002596970888898A8A8B0807802B6
:1044F00059692050888888F8888888025969F04866
:10450000484870484848F002596970888080808027
:10451000808870025969F048484848484848F00285
:104520005969F8808080F0808080F8025969F880AD
:104530008080F080808080025969708880808098B7
:1045400088887002596988888888F88888888812DD
:104550003969E040404040404040E002596938102D
:1045600010101010109060025969888890A0C0A0A7
:104570009088880259698080808080808080F802DD
:1045800059698888D8A8A88888888802596988C8FD
:10459000C8A8A898988888025969708888888888E7
:1045A000888870025969F0888888F080808080014E
:1045B0005A6A70888888888888A87008025969F0C3
:1045C000888888F0A09088880259697088808070F7
:1045D00008088870025969F8202020202020202017
:1045E000025969888888888888888870025969880B
:1045F000888888505050202002596988888888A867
:10460000A8A8A8500259698888505020505088881E
:10461000025969888850502020202020025969F8CA
:1046200008101020404080F8113B6BE080808080B3
:104630008080808080E00259698080404020101096
:104640000808113B6BE0202020202020202020E0C3
:10465000085363205088015161F82A226280400289
:104660005666700878889868025969808080F0885A
:10467000888888F002566670888080887002596940
:104680000808087888888888780256667088F880D4
:10469000887002596930484040F04040404000581E
:1046A000687088888878088870025969808080B02E
:1046B000C8888888881238684000C040404040E080
:1046C000004A6A1000301010101090906002596972
:1046D00080808090A0C0A09088123969C04040407E
:1046E00040404040E0025666D0A8A8A8A8880256DC
:1046F00066B0C888888888025666708888888870FE
:10470000005868F0888888F0808080005868788831
:10471000888878080808025666B0C88080808002C1
:1047200056667088601088700258684040F04040BB
:10473000404830025666888888889868025666889D
:1047400088885050200256668888A8A8A85002562B
:1047500066885020205088005868888888986808A3
:104760008870025666F810204080F8015B6B1820B4
:10477000202020C0202020201822196980808080DD
:104780008080808080015B6BC0202020201820204A
:104790002020C008536348A890FFFFFFFFFFFFFFE2
:1047A000FFFFFFFFFFFFFFFFFFFFFFFFFFFFFFFF19
:1047B000FFFFFFFFFFFFFFFFFFFF0D0060221969F2
:1047C0008000808080808080800358682070A8A04E
:1047D000A0A8702002596930484040E0404048B0ED
:1047E0000356668870505070880259698888505006
:1047F000F820F82020221969808080800080808045
:1048000080124A6A609080609090601090601A32C6
:1048100062A0A00359697088A8D8C8D8A888700475
:104820005767700878887800F80356662850A0A06B
:104830005028045363F80808163161E00359697081
:1048400088E8D8D8E8D888700A5161F817446460BD
:104850009090600357672020F8202000F807356506
:1048600040A02040E007356540A04020C02A2262D9
:1048700040800058688888888898E8808002596954
:1048800078E8E8E8E868282828262161C020226224
:10489000408007356540C04040E004576770888815
:1048A000887000F8035666A050282850A0025A6A63
:1048B00040C04040E00818283808025A6A40C0400A
:1048C00040E01028081038025A6A40A04020A04852
:1048D00018283808025969200020204080888870F4
:1048E000025A6A40200020508888F88888025A6A54
:1048F00010200020508888F88888025A6A304800C2
:1049000020508888F88888025A6A285000205088E9
:1049100088F88888025A6A50500020508888F888A1
:1049200088025A6A20502020508888F888880259C6
:104930006958A0A0A0B0E0A0A0B8005B6B70888010
:104940008080808088702040025A6A402000F88071
:1049500080F08080F8025A6A102000F88080F08091
:1049600080F8025A6A304800F88080F08080F802AF
:104970005A6A505000F88080F08080F8123A6A80BD
:104980004000E04040404040E0123A6A204000E0F1
:104990004040404040E0124A6A609000E0404040A1
:1049A0004040E0123A6AA0A000E04040404040E0B1
:1049B000025969F0484848E8484848F0025A6A28CD
:1049C00050008888C8A8988888025A6A40200070D9
:1049D000888888888870025A6A10200070888888C1
:1049E000888870025A6A3048007088888888887081
:1049F000025A6A28500070888888888870025A6A2B
:104A000050500070888888888870035565885020C9
:104A10005088015B6B08709898A8A8A8C8C87080D7
:104A2000025A6A40200088888888888870025A6AFA
:104A300010200088888888888870025A6A30480068
:104A400088888888888870025A6A505000888888C8
:104A500088888870025A6A10200088885020202098
:104A60002002596980F0888888F080808002596926
:104A7000609090A0A0908888B00259694020007092
:104A8000087888986802596910200070087888981A
:104A90006802596930480070087888986802596936
:104AA0002850007008788898680259695050007042
:104AB0000878889868025A6A304830007008788808
:104AC0009868025666702870A0A8500058687088D0
:104AD0008080887020400259694020007088F880EA
:104AE00088700259691020007088F8808870025917
:104AF000693048007088F880887002596950500009
:104B00007088F8808870123969804000C040404049
:104B100040E0123969204000C040404040E0124966
:104B200069609000C040404040E0123969A0A00098
:104B3000C040404040E0025A6A50206010708888AF
:104B4000888870025969285000B0C888888888020F
:104B5000596940200070888888887002596910203F
:104B60000070888888887002596930480070888889
:104B70008888700259692850007088888888700277
:104B800059695050007088888888700357672020C2
:104B900000F8002020015868087098A8A8C8708004
:104BA00002596940200088888888986802596910ED
:104BB0002000888888889868025969304800888869
:104BC0008888986802596950500088888888986851
:104BD000005B6B1020008888889868088870005AED
:104BE0006A8080B0C88888C8B08080005B6B5050F5
:104BF000008888889868088870000000000000001D
:104C000000000000000000000000000000000000A4
:104C10000000000000000000000000000C00000088
:104C2000000000000C000000000000001200000066
:104C30000000000023000000000000002100000030
:104C4000000000004C800000000000005E800000BA
:104C5000000000009240000000000000A1400000A1
:104C60000000000121200000000000027F900000F1
:104C7000000000020010000000000007FFF8000024
:104C8000000000040008000000000008000400000C
:104C900000000008000600000000001000020000F4
:104CA000000000301E010000000000207F81000095
:104CB00000000041FFE0800000000043FCF08000A5
:104CC000000000873B7840000000018EDBFC6000A4
:104CD0000000010FEBCC20000000021FEDB6100019
:104CE0000000021FDEB6100000000439CD7F08006E
:104CF00000000436E0FF08000000087EC0BB84000E
:104D00000000187F005D86000000107FC0ED82006B
:104D10000000203CC07301000000203B337F0100F5
:104D20000000701BE77E03800000C81DEEDE04C09B
:104D30000000880FDEDC04400001240FDF3C092066
:104D400000012607DBF8192000027203E7F0139038
:104D500000025101FFE02290000489007F80244876
:104D6000000904801E004824000BFE400000DFF410
:104D70000010004000008002001FFFFFFFFFFFFE49
:104D80000000000000000000000000000000000023
:104D90000000000000000000001022103C3C0E1F2C
:104DA0000010221004221104001022100822110405
:104DB00000102210083C11040010221010221104CF
:104DC0000010221020221104001E1C1E3C3C0E0468
:104DD00000000000000000000000000000000000D3
:104DE00000000000000000000000000000000000C3
:104DF00000000000000000000000000000000000B3
:104E000000000000000000000000000000000000A2
:104E10000000000000000000000000000000000092
:104E20000000000000000000000000000000000082
:104E30000000000000000048617264636F646564F4
:104E40002044656661756C742053657474696E677F
:104E500073204C6F616465640A00282300002823D6
:104E600000006400000010270000000096430000CE
:104E70009643000040400000C8410000C9420000C5
:104E8000C9420000C84400804F4400804F44204481
:104E90000020490020204D333034205000204400B1
:104EA00020490020204D3330312050002044002084
:104EB000490020500020204D33303120450050491A
:104EC000442073657474696E67733A0A0020460063
:104ED00020420020480020204D3134352053004D21
:104EE0006174657269616C206865617475702070A9
:104EF0006172616D65746572733A0A002059002011
:104F0000580020204D323138205400486F74656EAF
:104F100064206F6666736574733A0A00205A002035
:104F2000590020204D323036205800486F6D6520E2
:104F30006F66667365743A0A00204500205A0020A7
:104F4000590020580020420020540020204D3230CB
:104F500035205300416476616E6365643A20533CAA
:104F60006D696E5F66656564726174653E20543C70
:104F70006D696E5F74726176656C5F66656564729B
:104F80006174653E20423C6D696E5F7365676D6557
:104F90006E745F74696D655F6D733E20583C6D6122
:104FA000785F78795F6A65726B3E205A3C6D6178F4
:104FB0005F7A5F6A65726B3E20453C6D61785F6524
:104FC0005F6A65726B3E0A00205400205200202068
:104FD0004D323034205000416363656C65726174FA
:104FE000696F6E2028756E6974732F7332293A20A9
:104FF000503C7072696E745F616363656C3E2052F1
:105000003C726574726163745F616363656C3E20BA
:10501000543C74726176656C5F616363656C3E0AD3
:105020000020450020204D323031205400205A000D
:1050300020590020204D3230312058004D617869D0
:105040006D756D20416363656C65726174696F6E27
:105050002028756E6974732F7332293A0A0020452F
:105060000020204D323033205400205A00205900B7
:1050700020204D3230332058004D6178696D756DB8
:10508000206665656472617465732028756E697445
:10509000732F73293A0A0020450020204D39322011
:1050A0005400205A0020590020204D393220580049
:1050B00053746570732070657220756E69743A0A56
:1050C0000020204D3230302044300A0020204D3264
:1050D000303020543120440020204D3230302044E4
:1050E000002044697361626C65640A0046696C6102
:1050F0006D656E742073657474696E67733A002011
:10510000204D3134392043203B20556E6974732083
:10511000696E2043656C736975730A0020204732FD
:1051200031202020203B20556E69747320696E2049
:105130006D6D0A0045313A200045303A20005A3A58
:105140002000593A2000583A20004D53312C4D533D
:10515000322050696E730A005072696E742070615B
:1051600075736564004D31323500004D32340050A6
:1051700072696E742061626F72746564004E6F2094
:1051800053442063617264005072696E74206672C9
:105190006F6D2053440053746F70207072696E7489
:1051A00000526573756D65207072696E7400506190
:1051B000757365207072696E74004368616E67650F
:1051C0002066696C616D656E742045320041626FC6
:1051D0007574204669726D77617265004368616E0F
:1051E00067652066696C616D656E742045310043AA
:1051F0006F6E66696775726174696F6E0054656D74
:105200007065726174757265004D6F76656D656E5F
:10521000740054756E6500496E666F207363726525
:10522000656E00002DBCC8E911241FBECFEFD1E28E
:10523000DEBFCDBF00E00CBF14E0A0E0B2E0E2E7CB
:10524000F4E102E00BBF02C007900D92AE30B1074F
:10525000D9F725E1AEE0B4E001C01D92A136B20756
:10526000E1F719E2C3E1D9E200E006C021970109A4
:10527000802FFE010F94B509C231D10780E00807E5
:10528000A9F70E9475630D94280A0C9400002F92D0
:105290003F924F925F926F927F928F929F92AF92C6
:1052A000BF92CF92DF92EF92FF920F931F93CF9313
:1052B000DF93CDB7DEB7C35BD1090FB6F894DEBF7D
:1052C0000FBECDBF0091180920E6029F8001112476
:1052D0000856184F8091F00980FF1AC0E4EFF2E2FF
:1052E00084917F013FEFE31AF30A811102C0780134
:1052F00004C00E940669F701F3CFD7018D917D01AB
:10530000882319F00E940669F8CF8AE00E94066996
:1053100010922D0410922C048FE38093420410927B
:105320004104109240041092280410922904109213
:105330002A0410922B04F80180810F5F1F4F8032E6
:10534000D1F38E34B1F4818190ED980F9A3020F032
:105350008D3211F08B3269F43296DF0131962C9147
:1053600020532A30D0F3CD01FC0101962081203258
:10537000D9F3F093E113E093E0137F01BFEFEB1A51
:10538000FB0A10816AE270E0C7010F94F9090097E7
:1053900031F0FC01319780818032E1F311821D34BC
:1053A00029F0143519F0173409F0C9C0F7018081CC
:1053B0002FEFE21AF20A8032C9F380538A3008F0E4
:1053C000BEC01093420420914004309141044AE051
:1053D0003196429FC001439F900D1124DF01119728
:1053E0002C9130E020533109280F391F80818053E0
:1053F0008A3070F33093410420934004DF013196EA
:105400008C918032D9F31D34D1F42E31310591F0D5
:105410003CF42731310571F02C31310581F40AC09B
:105420002537310564F02737310524F0203A43E071
:10543000340729F4B0932D04A0932C0480C010925B
:105440002D0410922C040091E01361E070E0FD0146
:1054500031968C91882309F472C08132A1F41D34F5
:1054600091F42032310579F4F0932D04E0932C046B
:1054700063E270E0CF010F94F909009709F45FC06F
:10548000DC011C925CC04FEBD42ED80E59E1C52E26
:10549000CD14C0F1AF01FA0190814F5F5F4F9032A0
:1054A000D1F340ED490F4A3040F043ED490F42300F
:1054B00020F09B3211F00C941644AF01AD2CB12CAE
:1054C000750193E0F594E7949A95E1F7C701885D3B
:1054D0009B4F7C018D2D8770DB0102C0AA0FBB1F83
:1054E0008A95E2F7CD01D7019C91892B8C934115C8
:1054F000510511F0401B01C040E0D501A25FBB4F38
:105500004C930AC080912C0490912D04892B21F496
:10551000B0932D04A0932C04808181548A3110F41F
:10552000DF0195CFDF0131969C9190539A30D0F3F3
:10553000CD01FC01019640814032D9F3F1CF809139
:1055400042048D3409F4B1C7843511F40C94D0436E
:10555000873411F00C94F9438091400490914104F8
:105560008A31910509F4D0C684F48430910544F45D
:10557000823091050CF001C197FF23C00C941344B5
:10558000049709F47AC60C9413448A35910509F4FA
:105590004DC76CF48B31910509F4BDC64C9711F0E1
:1055A0000C94134480E00E942B8F0C9413448B3591
:1055B000910509F43FC78C35910509F440C70C9457
:1055C000134480917802882311F40C9413440E94B0
:1055D0005F8D8AE199E00E94EDEC0E946253809118
:1055E000F00983FD79C0C0902609D0902709E0908A
:1055F0002809F090290920912D0530912E05409120
:105600002F0550913005C701B6010F9491028823F0
:1056100009F462C0809146050E94F24C882301F192
:10562000C0922D05D0922E05E0922F05F092300504
:10563000E4EFF2E284918F010F5F1F4F882321F086
:105640000E940669F801F6CFE6E3F2E084918F014B
:105650000F5F1F4F882321F00E940669F801F6CFE3
:10566000C0902609D0902709E0902809F0902909D8
:1056700020912D0530912E0540912F055091300538
:10568000C701B6010F94C90620E030E048E453E4B6
:105690000F94F008181604F5C0922D05D0922E052F
:1056A000E0922F05F0923005E4EFF2E284918F0151
:1056B0000F5F1F4F882321F00E940669F801F6CF83
:1056C000E7E1F2E084918F010F5F1F4F882321F003
:1056D0000E940669F801F6CF20911A0930911B0942
:1056E00040911C0950911D0960912105709122057E
:1056F00080912305909124050F94910281111DC082
:1057000020911E0930911F094091200950912109D3
:1057100060912505709126058091270590912805B7
:105720000F949102811109C06091870270918802E3
:105730008091890290918A021AC06091240270912E
:105740002502072E000C880B990B0F9497022091CD
:105750008702309188024091890250918A020F9409
:10576000F6022AE037ED43E25CE30F94F6020E9472
:10577000D9910E94CF910C94134420917802222356
:1057800011F40C94134411E0029709F010E00E9408
:105790005F8D82E50E94E04C882309F45CC10E9481
:1057A0007E4C6B017C014090210550902205609059
:1057B0002305709024052091250530912605409100
:1057C00027055091280563962CAF3DAF4EAF5FAFD4
:1057D000639780911A0990911B09A0911C09B091BF
:1057E0001D0967968CAF9DAFAEAFBFAF6797209195
:1057F0001E0930911F0940912009509121096B9693
:105800002CAF3DAF4EAF5FAF6B9720E030E0A9010A
:10581000C701B6010F949102882309F414C5A301AE
:10582000920167966CAD7DAD8EAD9FAD67970F947D
:105830009102811111C063962CAD3DAD4EAD5FADAF
:1058400063976B966CAD7DAD8EAD9FAD6B970F94EE
:105850009102882309F4F7C420E030E0A901C701D0
:10586000B6010F949102881F8827881F18130BC058
:1058700080E090E0A0E8BFE3AB968CAF9DAFAEAF09
:10588000BFAFAB970AC020E030E040E85FEBAB96DB
:105890002CAF3DAF4EAF5FAFAB97A30192016796C0
:1058A0006CAD7DAD8EAD9FAD67970F94C906A39685
:1058B0006CAF7DAF8EAF9FAFA39763962CAD3DAD20
:1058C0004EAD5FAD63976B966CAD7DAD8EAD9FAD0C
:1058D0006B970F94C906A7966CAF7DAF8EAF9FAF45
:1058E000A797A3962CAD3DAD4EAD5FADA397CA0172
:1058F000B9010F94F6024B015C01A7962CAD3DADAA
:105900004EAD5FADA797CA01B9010F94F6029B0196
:10591000AC01C501B4010F94CA060F9435096F9606
:105920006CAF7DAF8EAF9FAF6F9720E030E040E06F
:105930005FE30F94F6024B015C01A7019601C701DA
:10594000B6010F94F6026B017C01A5019401C5011B
:10595000B4010F94F6029B01AC01C701B6010F948C
:10596000C9060F9435099B01AC01AB966CAD7DADBA
:105970008EAD9FADAB970F94F6024B015C0167961D
:105980002CAD3DAD4EAD5FAD6797C301B2010F9435
:10599000CA0620E030E040E05FE30F94F6026B01BE
:1059A0007C01A7966CAD7DAD8EAD9FADA79790584D
:1059B0006F962CAD3DAD4EAD5FAD6F970F94A607C2
:1059C0009B01AC01C501B4010F94F6029B01AC012F
:1059D000C701B6010F94CA06A30192010F94C9062C
:1059E0006B017C016B962CAD3DAD4EAD5FAD6B9701
:1059F00063966CAD7DAD8EAD9FAD63970F94CA0677
:105A000020E030E040E05FE30F94F6022B013C0120
:105A10006F962CAD3DAD4EAD5FAD6F97A3966CAD5F
:105A20007DAD8EAD9FADA3970F94A6079B01AC01F2
:105A3000C501B4010F94F6029B01AC01C301B20190
:105A40000F94CA0663962CAD3DAD4EAD5FAD639726
:105A50000F94C90614C089E40E94E04C882329F001
:105A60000E947E4C6B017C0103C0C12CD12C7601BD
:105A70008AE40E94E04C8823F9F00E947E4C6B96E9
:105A80006CAF7DAF8EAF9FAF6B9720E030E0A90188
:105A9000C701B6010F94910281111EC020E030E0D1
:105AA000A9016B966CAD7DAD8EAD9FAD6B970F94DC
:105AB0009102811111C0C7C320E030E0A901C701E4
:105AC000B6010F949102882309F4BDC36B961CAEF6
:105AD0001DAE1EAE1FAE6B97D701C601B0586396C0
:105AE0008CAF9DAFAEAFBFAF63976B962CAD3DADA6
:105AF0004EAD5FAD6B97505867962CAF3DAF4EAF34
:105B00005FAF67979C01AD01BC01CD010F94F60218
:105B10004B015C0167962CAD3DAD4EAD5FAD679717
:105B2000CA01B9010F94F6029B01AC01C501B40191
:105B30000F94CA060F943509EB966CAF7DAF8EAF0C
:105B40009FAFEB978091210590912205A0912305AD
:105B5000B09124056F968CAF9DAFAEAFBFAF6F977E
:105B6000A7019601BC01CD010F94CA06AB966CAF9C
:105B70007DAF8EAF9FAFAB97209125053091260565
:105B80004091270550912805A3962CAF3DAF4EAF0D
:105B90005FAFA3976B962CAD3DAD4EAD5FAD6B97F0
:105BA000A3966CAD7DAD8EAD9FADA3970F94CA0645
:105BB000AF966CAF7DAF8EAF9FAFAF9780911A0954
:105BC00090911B09A0911C09B0911D09E3968CAF1F
:105BD0009DAFAEAFBFAFE397AB962CAD3DAD4EAD35
:105BE0005FADAB97BC01CD010F94C9066B017C0181
:105BF00020911E0930911F094091200950912109DF
:105C0000E7962CAF3DAF4EAF5FAFE797AF962CADA9
:105C10003DAD4EAD5FADAF97E7966CAD7DAD8EAD52
:105C20009FADE7970F94C9064B015C018091290550
:105C300090912A05A0912B05B0912C05C158DF4FFA
:105C400088839983AA83BB83CF57D0409C01AD0141
:105C5000609122097091230980912409909125096E
:105C60000F94C906A7966CAF7DAF8EAF9FAFA79775
:105C7000209126093091270940912809509129093E
:105C8000EF962CAF3DAF4EAF5FAFEF9780912D05F4
:105C900090912E05A0912F05B0913005CD57DF4F83
:105CA00088839983AA83BB83C358D040A7019601F8
:105CB00063966CAD7DAD8EAD9FAD63970F94F6028C
:105CC0002B013C01A501940167966CAD7DAD8EADB5
:105CD0009FAD67970F94F6029B01AC01C301B2011F
:105CE0000F94CA062B013C01A501940163966CAD8B
:105CF0007DAD8EAD9FAD63970F94F6024B015C01B5
:105D0000A701960167966CAD7DAD8EAD9FAD67978F
:105D10000F94F6029B01AC01C501B4010F94C906B2
:105D2000A30192010F943D076B017C0120E030E05C
:105D3000A9010F94910287FF0AC02BED3FE049ECC7
:105D400050E4C701B6010F94CA066B017C01112310
:105D500051F02BED3FE049EC50E4C701B6010F9440
:105D6000C9066B017C0120E030E0A901C701B60142
:105D70000F949102811128C0E3962CAD3DAD4EAD3C
:105D80005FADE3976F966CAD7DAD8EAD9FAD6F97B8
:105D90000F949102811118C0E7962CAD3DAD4EAD28
:105DA0005FADE797A3966CAD7DAD8EAD9FADA3972C
:105DB0000F949102811108C08BEDC82E8FE0D82E70
:105DC00089ECE82E80E4F82EEB962CAD3DAD4EAD7F
:105DD0005FADEB97C701B6010F94F6029B01AC01D2
:105DE0000F94F6024B015C01A7962CAD3DAD4EAD74
:105DF0005FADA797CA01B9010F94F6029B01AC01F0
:105E0000C501B4010F94CA060F9435094B015C011A
:105E10002FE632E143E85AE30F94910287FD0FC267
:105E2000C501B4010F943F080F941308A1967FAFEA
:105E30006EAFA197DB01AB2B31F4E1E0F0E0A1966E
:105E4000FFAFEEAFA197A1962EAD3FADA197B901DF
:105E500080E090E00F9495024B015C019B01AC0146
:105E6000C701B6010F94A6076F966CAF7DAF8EAFDA
:105E70009FAF6F97A5019401A7966CAD7DAD8EADD8
:105E80009FADA7970F94A607EB966CAF7DAF8EAF33
:105E90009FAFEB97CD57DF4F288139814A815B81D6
:105EA000C358D040EF966CAD7DAD8EAD9FADEF97F2
:105EB0000F94C906A50194010F94A607EF966CAF45
:105EC0007DAF8EAF9FAFEF976F962CAD3DAD4EADD2
:105ED0005FAD6F97CA01B9010F94F60220E030E080
:105EE00040E05FE30F94F6029B01AC0160E070E0DC
:105EF00080E89FE30F94C906A7966CAF7DAF8EAF85
:105F00009FAFA797C158DF4F88819981AA81BB8134
:105F1000CF57D04089879A87AB87BC87CD57DF4F53
:105F2000288139814A815B81C358D0402D873E87C3
:105F30004F87588B6091240270912502072E000C28
:105F4000880B990B0F949702209187023091880259
:105F50004091890250918A020F94F6022AE037EDAF
:105F600043E25CE30F94F602E3966CAF7DAF8EAF35
:105F70009FAFE3970E940A539B01AC0128533F4F08
:105F80004F4F5F4FE7962CAF3DAF4EAF5FAFE797F8
:105F900060964FAC609761965FAC619762966FAC0C
:105FA000629763967FAC639722242394312C09E196
:105FB000D02EA1964EAD5FADA1972416350609F4FB
:105FC0002AC10E9480D30E940A53DC01CB01E796CC
:105FD0002CAD3DAD4EAD5FADE797821B930BA40B8F
:105FE000B50BB7FD11C00E940A539B01AC012853A9
:105FF0003F4F4F4F5F4FE7962CAF3DAF4EAF5FAF78
:10600000E79780E00E945EEADA94DD2009F44BC055
:10601000A7962CAD3DAD4EAD5FADA79767966CAD25
:106020007DAD8EAD9FAD67970F94F6024B015C017D
:106030006F962CAD3DAD4EAD5FAD6F97B201C30114
:106040000F94F602A50194010F94CA067B018C01FE
:10605000A7962CAD3DAD4EAD5FADA797B201C30184
:106060000F94F6024B015C016F962CAD3DAD4EAD29
:106070005FAD6F9767966CAD7DAD8EAD9FAD679749
:106080000F94F6029B01AC01C501B4010F94C9063F
:106090002B013C01C701D80167968CAF9DAFAEAF15
:1060A000BFAF67975BC0B10180E090E00F949502AD
:1060B0006F962CAD3DAD4EAD5FAD6F970F94F60270
:1060C0004B015C010F94A3076B017C01C501B40176
:1060D0000F942B094B015C01A701960163966CADEF
:1060E0007DAD8EAD9FAD63970F94F6022B013C0101
:1060F000A50194016B966CAD7DAD8EAD9FAD6B9798
:106100000F94F6029B01AC01C301B2010F94CA06C1
:106110002B013C01A501940163966CAD7DAD8EAD64
:106120009FAD63970F94F6024B015C01A7019601A6
:106130006B966CAD7DAD8EAD9FAD6B970F94F602F7
:106140009B01AC01C501B4010F94C90667966CAF01
:106150007DAF8EAF9FAF6797B9E1DB2E9201A301B0
:10616000AB966CAD7DAD8EAD9FADAB970F94CA066F
:1061700069837A838B839C8367962CAD3DAD4EAD4E
:106180005FAD6797AF966CAD7DAD8EAD9FADAF97B0
:106190000F94CA066D837E838F839887EB962CAD10
:1061A0003DAD4EAD5FADEB9769857A858B859C855E
:1061B0000F94CA0669877A878B879C87EF962CADE8
:1061C0003DAD4EAD5FADEF976D857E858F8598892E
:1061D0000F94CA066D877E878F87988BCE010196B4
:1061E0000E94EDECC0904605E396ECACFDAC0EAD24
:1061F0001FADE3979E01235F3F4FAE01475F5F4FA7
:10620000BE016B5F7F4FCE0101960E94C2A43FEF9B
:10621000231A330ACECEC0904605E396ECACFDAC13
:106220000EAD1FADE39726E239E042E259E06EE1A0
:1062300079E08AE199E00E94C2A40E94CF910E9475
:1062400062530C941344E6ECF7E184918F010F5FE5
:106250001F4F882321F00E940669F801F6CFE1E57F
:10626000F2E084918F010F5F1F4F882311F40C948B
:1062700013440E940669F801F4CF80E50E94E04CC7
:10628000882329F00E943E4C6B017C0103C0C12C85
:10629000D12C760183E50E94E04C882361F00E94B6
:1062A0007E4C20E030E04AE754E40F94F6020F946D
:1062B00013086B017C010E94CCF98091330281119B
:1062C00005C060E087E692E00E9468C70E946253C2
:1062D0008091E2139091E313A091E413B091E51340
:1062E000C80ED91EEA1EFB1E0E940A53DC01CB0118
:1062F0008C199D09AE09BF09B7FD02C00C94134467
:1063000080E00E945EEAF0CF81E0809378021092F4
:106310004A050C9413440E94876181110C94134424
:1063200080E50E94E04C882321F00E944E4C262FED
:1063300001C020E06091290570912A0580912B050C
:1063400090912C05C12CD12CE12C51E4F52EC98261
:10635000DA82EB82FC82C12CD12CE5E8EE2EE3E45C
:10636000FE2ECD82DE82EF82F886C12CD12CF0EA9F
:10637000EF2EF1E4FF2EC986DA86EB86FC86C12C6F
:10638000D12CA0ECEA2EAFE7FA2ECD86DE86EF8682
:10639000F88A213071F1223021F518A219A21AA22F
:1063A0001BA220E030E040EA51E40F94CA066B01E2
:1063B0007C0120E030E04AE753E40F94F00818161F
:1063C00034F4C12CD12C4AE7E42E43E4F42ECBAEB6
:1063D000DCAEEDAEFEAEBE01605E7F4FCE01CB9671
:1063E00011C020E030E040EA51E40F94910287FFB1
:1063F0000BC018A219A21AA21BA2BE01605E7F4F99
:10640000CE0109960E941A8F18A219A21AA21BA2E5
:106410009E01205E3F4F49E255E0BE016B5F7F4F1A
:10642000CE0101960E943A8E0C94134410923F04C0
:106430000C94134481E080933F040C94134485E44E
:106440000E94E04C082F811102C00E94CCF923E485
:10645000A22E23E0B22E31E2E32E35E0F32ED12C32
:1064600010E0D5018D915D010E94E04C882359F028
:106470000E947E4CF7016083718382839383133083
:1064800011F0DD24D3941F5FF4E0EF0EF11C143003
:1064900041F7DD2019F00E94344C03C001110E9425
:1064A0001E620E94AF9E0C94134480914004909110
:1064B00041048737910509F418C70CF0CCC08C341F
:1064C000910509F44FC40CF06BC08831910509F4B3
:1064D0009FC2B4F58231910509F4AFC5C4F497FFAA
:1064E00002C00C941344823091050CF4B1C1419761
:1064F00011F00C94134460E087EA92E00E9468C7B0
:10650000179816981598149813980C94134485317D
:10651000910509F462C23CF4449711F00C941344C1
:10652000EFEBF2E019C28631910509F45AC24797A0
:1065300011F00C941344E0912C04F0912D045BC2F3
:106540008E31910509F4DBC2C4F48A31910509F456
:106550008CC20CF47CC28B31910509F494C24C9727
:1065600011F00C94134440E060E080912C04909171
:106570002D040E94885C0C9413448032910509F428
:10658000D8C30CF4E7C38A32910509F4E7C38B340E
:10659000910511F00C9413440E944D610C94134426
:1065A0008936910509F4C9C424F58335910509F4A8
:1065B0003FC57CF48135910509F432C50CF034C532
:1065C0008D34910511F00C9413440E940EBF0C946D
:1065D00013448535910509F434C50CF42EC58C356A
:1065E000910509F449C58836910509F4BFC30C9497
:1065F00013448F36910509F430C484F48B36910529
:1066000009F40AC50CF4E3C48D36910509F4C4C439
:106610008E36910509F40EC40C941344833791050A
:1066200009F4C8C55CF48237910511F00C94134449
:106630000E94CCF90E94AF9E0C94134485379105BB
:1066400009F44AC68637910511F00C9413440E9450
:10665000769E0C9413448C3221E0920709F48FC784
:106660000CF069C0893C910509F42AC764F58C389F
:10667000910509F45EC47CF48937910509F4A0C63C
:106680000CF497C68D37910511F00C9413440E94B9
:10669000C49D0C9413448B39910509F452C434F40D
:1066A0008139910509F492C60C9413448E3B9105EF
:1066B00009F476C4883C910511F00C9413440E94AF
:1066C0005A9D0C941344833D910509F405C7DCF4ED
:1066D0008C3C910509F4F8C64CF48B3C910511F003
:1066E0000C9413440E94EF9C0C9413448D3C910530
:1066F00009F4EEC68E3C910511F00C9413440E94EF
:106700006E9F0C9413448C3D910509F4E9C64CF43A
:106710008A3D910511F00C9413440E94199B0C942E
:1067200013448D3D910509F4DFC6823E910509F4BD
:10673000DFC60C941344843F41E0940711F40C9499
:1067400072410CF049C08E35A1E09A0711F40C9407
:106750001C43A4F48E32E1E09E0711F40C94063C35
:106760000CF437C78F3221E0920711F40C945A3C95
:106770008033914009F4CCC70C941344833641E034
:10678000940711F40C94A5433CF48F35914011F417
:106790000C9451430C9413448039B1E09B0711F4DD
:1067A0000C9494408C3A914011F00C94134466E69A
:1067B000C62E67E0D62E71E2E72E75E0F72EE8EEE2
:1067C0002E2EE4E03E2E00E010E0E22DE0956096F3
:1067D000EFAF60970C9497408835F2E09F0711F473
:1067E0000C949441B4F4863F31E0930711F40C9477
:1067F000784114F40C947541873F51E0950711F4EA
:106800000C947B418C31924011F40C9489410C948E
:1068100013448C38B3E09B0711F40C94024364F4E6
:106820008B38934011F00C94134443E4E42E43E07E
:10683000F42E10E00C94DB42803A23E0920709F436
:106840007CC2873E934011F40C94BE430C941344D5
:10685000A0902C04B0902D0480E50E94E04C882389
:1068600059F00E943E4C6B017C0111E0672B682BB4
:10687000692B31F410E004C010E0C12CD12C76015A
:1068800083E50E94E04C8823F1F00E947E4C20E0DA
:1068900030E04AE754E40F94F6020F9413086B01BA
:1068A0007C01111112C0672B682B692B71F4A114A4
:1068B000B10459F0D5018C91882339F061E0C5010C
:1068C0000E9486C707C0112391F360E084E992E03B
:1068D0000E9468C781E08093F10D0E94CCF90E946C
:1068E0006253C114D104E104F104F1F08091E21388
:1068F0009091E313A091E413B091E513C80ED91E53
:10690000EA1EFB1E0E940A53DC01CB018C199D0973
:10691000AE09BF09B7FF1CC08091F10D8823C1F0FB
:1069200080E00E945EEAEECF8091F10D882321F095
:1069300080E00E945EEAF8CF80911F0B60E0882320
:1069400019F085E892E002C080E792E00E9468C7F3
:106950001092F10D0C94134484918F010F5F1F4F1F
:10696000882321F00E940669F801F6CF1092CB0D22
:1069700040E050E0BA0187E79BE00E9490798BE10C
:10698000E7E7FBE0DE01159601900D928A95E1F7AD
:106990008091750B9091760B9C838B8384E993E0B7
:1069A0009A83898340E050E0BE016F5F7F4F89EC9E
:1069B00093E00E94AFC0CE0101960E94E5E9E0EBB2
:1069C000F2E084918F010F5F1F4F882311F40C9424
:1069D00013440E940669F801F4CF0E94B75F0C943B
:1069E000134410921F0B1092200B0C94134480320E
:1069F00009F41082319680818111F9CF40E061E085
:106A000080912C0490912D040E94885C0C94134476
:106A100019821A821B821C8218A219A21AA21BA216
:106A200080913B09882341F040E0BE016F5F7F4FBA
:106A3000CE0180960E94BF6C8091200B882319F0B4
:106A400081E080931F0B0E944D610C9413441092BF
:106A50001F0B0E94636280ED92E090935707809332
:106A600056070E9451490C9413448091200B8823AF
:106A700011F40C94134483E50E94E04C81110C94B2
:106A800027440C9413448091200B882351F1E5EDA9
:106A9000F2E084918F010F5F1F4F882321F00E9445
:106AA0000669F801F6CF6091C20D7091C30D809117
:106AB000C40D9091C50D4AE00E945F698FE20E946B
:106AC00006696091BE0D7091BF0D8091C00D9091CF
:106AD000C10D4AE00E945F698AE00E9406690C9439
:106AE0001344E7EEF2E084918F010F5F1F4F88237C
:106AF00011F40C9413440E940669F801F4CF8091BC
:106B0000200B882311F40C94134481E19DE00E9432
:106B10004D7981E19DE00E94C97A10921E0B10927E
:106B20001D0BE0902C04F0902D048091200B882305
:106B300011F40C9413440E9403BF1D8218861C821A
:106B40001B8284E993E09A83898383E79BE0909397
:106B5000930B8093920BF70180818F3209F068C00C
:106B60006FE270E0C7010F94F9098C010F5F1F4FAE
:106B70009E012F5F3F4F49010115110509F45EC0C9
:106B80006FE270E0C8010F94F9096C01009709F4F5
:106B900056C00817190708F052C05C01A01AB10AC4
:106BA000A501B801CE0180960F94190AE0E2F0E049
:106BB000EC0FFD1FEA0DFB1D10828E01005E1F4FC2
:106BC000D8018D918D01882319F00E940669F8CFB4
:106BD0008AE00E9406696091920B7091930B611597
:106BE000710511F06C5F7F4F21E0AE01405E5F4F99
:106BF000CE0105960E94B480811112C0BE01605E74
:106C00007F4F8EE193E00E94EAC28EE20E94066905
:106C10008AE00E940669C4010E94E5E90C941344CD
:106C20009092930B8092920B86010F5F1F4FA4CF1F
:106C300084E99BE09093930B8093920B8701609182
:106C4000920B7091930B6115710511F06C5F7F4F82
:106C500018A21BA222E0A801CE0180960E94B48057
:106C6000811102C0F12C1EC0CE0180960E9471BE1F
:106C70008823C1F36CA57DA58EA59FA541E00E9448
:106C8000D6B1882379F3E8A9B0E2EB9FF001112493
:106C9000E55BFA4F309731F385EE80831BA20E94AB
:106CA00096B1F82ECE0180960E94EC4CFF2011F197
:106CB00098EFE92E92E0F92EF7018491882331F0C4
:106CC000FFEFEF1AFF0A0E940669F6CFD8018D91F7
:106CD0008D01882319F00E940669F8CF8AE00E948E
:106CE00006691092C20D1092C30D1092C40D10923D
:106CF000C50D19C086E0E82E83E0F82EF7018491D7
:106D0000882331F0FFEFEF1AFF0A0E940669F6CFE1
:106D1000D8018D918D01882319F00E940669F8CF62
:106D20008EE20E940669CE0101960E94E5E90C946C
:106D300013440E94678B0C94134480912C0490910F
:106D40002D0421E020931E0B40E060E00E94885C4F
:106D50000C9413440E94AC8B0C9413440E94068B39
:106D60000C9413440E9463620C94134488E690E0F0
:106D70000E94499281110C9413448091F00983FF81
:106D800002C00C94134483E50E94E04C882311F464
:106D90000C9413440E947E4CF0902E042F2D30E072
:106DA000220F331F8901055F154F0F940E08F8015C
:106DB000718360838F2D0E949FCF0E947E4C20E0C4
:106DC00030E040E752E40F94910218163CF00E9424
:106DD0000EBF60E081E493E00E9468C70E947E4C91
:106DE00000912E0410E0F801EE0FFF1FEE0FFF1FC1
:106DF000E452FB4F20813181428153810F94F0088E
:106E0000181614F00C9413448BEE92E09F938F931A
:106E1000C80101969F938F9382E393E09F938F9392
:106E20001F920E9432610FB6F894DEBF0FBECDBF35
:106E30000C9413448EE40E94E04C882311F40C94CB
:106E400013440E944E4C6093C5137093C6138093F5
:106E5000C7139093C8130C94134483E50E94E04C2D
:106E6000882319F00E945E4C01C080E08093F009F5
:106E7000E4EFF2E284918F010F5F1F4F882321F02E
:106E80000E940669F801F6CFE4E6F3E084918F01F1
:106E90000F5F1F4F882321F00E940669F801F6CF8B
:106EA0008091F0098823A1F1F6E5CF2EF3E0DF2EE3
:106EB000E12CF12C20E08091F00990E00E2C02C032
:106EC000959587950A94E2F780FF17C0BB24B39489
:106ED000B20E222319F08CE20E940669F601259178
:106EE0003491F901849189010F5F1F4F882321F0AC
:106EF0000E9406699801F5CF2B2DFFEFEF1AFF0ACC
:106F000032E0C30ED11C45E0E416F104A1F60CC03A
:106F1000E0E6F3E084918F010F5F1F4F882321F09B
:106F20000E940669F801F6CF8AE00E9406690C9477
:106F300013440E942AA00C9413440E9449A20C946A
:106F4000904783E50E94E04C882311F40C9413448D
:106F50000E945E4C8093CD138D3318F08CE38093A8
:106F6000CD130E940A536B017C012091CD1330E0B8
:106F7000A8EEB3E00F94BA06DC01CB018C0D9D1D89
:106F8000AE1DBF1D8093C9139093CA13A093CB135A
:106F9000B093CC130C9413440E9443A00C9413445C
:106FA0008091F00983FF02C00C94134483E50E9492
:106FB000E04C68968FAF689781110C94384482E555
:106FC0000E94E04C81110C9438440C94134483E5E6
:106FD0000E94E04C882339F00E944E4C8B016F3F99
:106FE000710519F010F00FEF10E080E50E94E04C01
:106FF000882339F00E945E4C823010F00C941344C8
:1070000001C080E0E82FF0E0EE0FFF1FEB5FF54FCF
:10701000118300830C9413440E9434A20C941344F3
:107020000E9413A00C94134410923E040C94134439
:1070300081E080933E040C9413440E94C29F0C9400
:10704000134483E50E94B14C882311F40C9413443B
:107050000E947E4C20E030E04AE754E40F94F602B0
:107060000F9413086093E6137093E7138093E8136B
:107070009093E9130C9413448CE590E00E9449929C
:1070800081110C941344A3E4B3E06196BFAFAEAF9B
:10709000619751E3C52E55E0D52EF12C6196EEADEA
:1070A000FFAD619781916196FFAFEEAF61970E944E
:1070B000B14C882309F473C0F3E0FF1268C00E944A
:1070C0007E4C2B013C0120E030E040EA51E40F947B
:1070D0009102E0902E0487FF4FC00E2D10E00D5F4F
:1070E0001F4F000F111F000F111FF801EF5CFA4F27
:1070F000A301920160817181828193810F94A6071F
:107100004B015C019B01AC016091740A7091750A9E
:107110008091760A9091770A0F94F6026093740A30
:107120007093750A8093760A9093770A9801285E87
:10713000354F1901A5019401D1016D917D918D917A
:107140009C910F94F602F101608371838283938393
:107150000356114FD8016D917D918D919C910F94A3
:107160009502A50194010F94F6020F941308F801FB
:10717000608371838283938324E0E29EF001112473
:10718000E35CFA4F408251826282738208C00E949F
:107190007E4CD6016D937D938D939C931397F394BE
:1071A000B4E0CB0ED11CE4E0FE1278CF0E9490E751
:1071B0000C941344EEE6F4E084918F010F5F1F4FAF
:1071C000882321F00E940669F801F6CFE0E6F4E09A
:1071D00084918F010F5F1F4F882321F00E94066961
:1071E000F801F6CFE9E4F4E084918F010F5F1F4FBF
:1071F000882321F00E940669F801F6CFE9E3F4E064
:1072000084918F010F5F1F4F882321F00E94066930
:10721000F801F6CFE8E2F4E084918F010F5F1F4F91
:10722000882321F00E940669F801F6CFE7E1F4E037
:1072300084918F010F5F1F4F882321F00E94066900
:10724000F801F6CFE8E0F4E084918F010F5F1F4F63
:10725000882321F00E940669F801F6CFE3EFF3E0FE
:1072600084918F010F5F1F4F882321F00E940669D0
:10727000F801F6CFEDEDF3E084918F010F5F1F4F22
:10728000882321F00E940669F801F6CFE8ECF3E0CC
:1072900084918F010F5F1F4F882321F00E940669A0
:1072A000F801F6CFEBEAF3E084918F010F5F1F4FF7
:1072B000882321F00E940669F801F6CFE3E9F3E0A4
:1072C00084918F010F5F1F4F882311F40C94134496
:1072D0000E940669F801F4CF60E080912C0490913F
:1072E0002D040E9486C70C941344EEE7F5E08491C8
:1072F0008F010F5F1F4F882321F00E940669F8015C
:10730000F6CFE6E7F5E084918F010F5F1F4F8823EA
:1073100021F00E940669F801F6CF1E9B03C004ED20
:1073200012E002C009ED12E0D8018D918D01882391
:1073300019F00E940669F8CF8AE00E940669EEE61D
:10734000F5E084918F010F5F1F4F882321F00E9489
:107350000669F801F6CF1D9B03C004ED12E002C0E0
:1073600009ED12E0F80181918F01882319F00E9444
:107370000669F8CF8AE00E940669E6E6F5E08491A6
:107380008F010F5F1F4F882321F00E940669F801CB
:10739000F6CF1C9B03C004ED12E002C009ED12E021
:1073A000D8018D918D01882309F4BECD0E94066914
:1073B000F7CF81E080936507809364070C941344B2
:1073C00010926507109264070C94134483E50E94A1
:1073D000E04C882319F00E944E4C02C060E070E03F
:1073E0008B01112702301105D4F0E6ECF7E184910E
:1073F0008F010F5F1F4F882321F00E940669F8015B
:10740000F6CFE8E9F5E084918F010F5F1F4F8823E5
:1074100011F40C9413440E940669F801F4CF88E437
:107420000E94E04C8823A9F00E944E4C68377105F9
:107430003CF06332B1E07B072CF062E271E002C005
:1074400068E770E0F801EE0FFF1FE75DFA4E718309
:10745000608386E40E94E04C8823A9F00E944E4C91
:10746000F801EE0FFF1FEF5DFA4E718360836F3FEF
:10747000710519F014F06FEF70E077FF02C060E063
:1074800070E07183608382E40E94E04C882311F4F1
:107490000C9413440E944E4C6530710534F06838EA
:1074A00071052CF067E870E002C065E070E0000F45
:1074B000111FF801EB5DFA4E718360830C94134445
:1074C0000E941E9D0C9413440E94869C0C941344AD
:1074D0000E941C9C0C9413440E94869B0C941344A1
:1074E0000E940D9B0C9413440E94F29A0C94134436
:1074F00080E50E94B14C882311F40C9413440E943F
:107500004E4CF62E062F172F83E50E94E04C882361
:1075100021F00E944E4C6B0103C0CC24CA94DC2C99
:10752000C6010196039710F00C94134417FF02C094
:107530000C9413440E94CCF9EFEFCE16DE0631F026
:10754000CA94CD2871F401E010E00DC08F2D0E9487
:10755000B05131E020E0892B09F030E0032F122FE9
:1075600002C000E010E08F2D0E94B05180179107FB
:1075700011F40C94134480E00E945EEAF4CF83E59A
:107580000E94E04C882319F00E944E4C02C064E037
:1075900071E079A368A380E50E94E04C882339F06C
:1075A0000E944E4C693823E1720730F402C068EE45
:1075B00073E07A83698304C088E893E19A838983BE
:1075C000BE01605E7F4FCE0101960E94FE600C946A
:1075D000134485E40E94E04C811110C080E50E94B4
:1075E000B14C882391F00E947E4C60931D157093DE
:1075F0001E1580931F159093201507C00E945E4CA6
:10760000823060F3E6ECF7E172C089E40E94B14C8D
:10761000882381F00E947E4C2CEA35EC47E25EE341
:107620000F94F6026093191570931A1580931B1529
:1076300090931C1584E40E94B14C882381F00E9431
:107640007E4C2CEA35EC47E25EE30F94A60760938C
:107650001515709316158093171590931815E4EF70
:10766000F2E284918F010F5F1F4F882321F00E9467
:107670000669F801F6CF40911D1550911E156091D5
:107680001F157091201582EC95E00E948DC22CEAA6
:1076900035EC47E25EE36091191570911A158091FF
:1076A0001B1590911C150F94A607AB01BC018EEB26
:1076B00095E00E94E4682CEA35EC47E25EE36091D5
:1076C00015157091161580911715909118150F9436
:1076D000F602AB01BC018AEB95E00E94E4688AE007
:1076E0000E9406690C9413440E940669F801849173
:1076F0008F010F5F1F4F8111F7CF06EF12E0D80106
:107700008D918D01882309F40FCC0E940669F7CF73
:1077100080E50E94B14C882351F00E947E4C60931A
:10772000111570931215809313159093141589E415
:107730000E94B14C882381F00E947E4C2CEA35ECEB
:1077400047E25EE30F94F60260930D1570930E15F9
:1077500080930F159093101584E40E94B14C8823F8
:1077600081F00E947E4C2CEA35EC47E25EE30F94F8
:10777000A6076093091570930A1580930B159093D3
:107780000C15E4EFF2E284918F010F5F1F4F882305
:1077900021F00E940669F801F6CF40911115509131
:1077A000121560911315709114158EEC95E00E94DE
:1077B0008DC22CEA35EC47E25EE360910D157091C5
:1077C0000E1580910F15909110150F94A607AB011F
:1077D000BC018AEC95E00E94E4682CEA35EC47E2B3
:1077E0005EE36091091570910A1580910B159091D7
:1077F0000C150F94F602AB01BC0186EC95E00E94DB
:10780000E4688AE00E9406690C94134483E50E94B0
:10781000B14C182F882371F00E947E4C0F940E08F3
:1078200070931F0260931E0221E0672B09F020E095
:107830002093EF0980E50E94B14C882359F02091F4
:107840001E0230911F02232B11F00E946F4C809377
:10785000EF09E9C71111E7C7E4EFF2E284918F0164
:107860000F5F1F4F882321F00E940669F801F6CFB1
:107870008091EF09811103C063EE72E002C066EDF2
:1078800072E087EE95E00E94EAC260911E0270915C
:107890001F0286ED95E00E94D1C2E2EDF5E08491F1
:1078A0008F010F5F1F4F882309F4BDC70E9406692F
:1078B000F801F5CF85E40E94E04C882321F00E9476
:1078C0004E4C1B0102C0212C312C83E40E94E04C61
:1078D000882349F00E944E4CC856DF4F7983688355
:1078E000C859D04008C0E5E0F0E0C856DF4FF98342
:1078F000E883C859D04085E50E94B14CC257DF4F9C
:107900008883CE58D040882339F00E946F4CC257EC
:10791000DF4F8883CE58D04037FC07C0C12CD12C14
:10792000B6E1EB2EB3E4FB2E06C0C12CD12CACE8A3
:10793000EA2EA2E4FA2E83E50E94E04C882321F08F
:107940000E947E4C6B017C01F2E02F16310410F492
:1079500020922E040E940A532B013C01C101019682
:10796000039718F407E013E00BC00AE113E0D80115
:107970008D918D01882309F4D7CA0E940669F7CF3B
:10798000F80181918F01882319F00E940669F8CFD0
:107990008AE00E9406690E94F7CFFFEF2F163F068C
:1079A00049F487E68093920EF7E68F2E912CA12C56
:1079B000B12C0AC08FE7F101EB56F14F8083EFE75E
:1079C0008E2E912CA12CB12CC701B6010F940E085C
:1079D000072E000C880B990B0F949702AC966FAF93
:1079E000AC97E0967FAFE097E4968FAFE497C158ED
:1079F000DF4F9883CF57D04081E080939A022FEFDA
:107A00002216320629F48EEC90E0A0E0B0E004C02B
:107A10008FEF90E0A0E0B0E09C01AD01235131096F
:107A200041095109C056DF4F288339834A835B835C
:107A3000C05AD0409C01AD0124513109410951097E
:107A4000CC55DF4F288339834A835B83C45AD040A7
:107A50009C01AD015595479537952795C855DF4F42
:107A6000288339834A835B83C85AD0409C01AD0187
:107A70002150310941095109C455DF4F2883398309
:107A80004A835B83CC5AD0406B968CAE9DAEAEAE33
:107A9000BFAE6B97C057DF4F488259826A827B82A4
:107AA000C059D040C656DF4F488259826A827B82D5
:107AB000CA59D040CD57DF4F1882C358D04030E468
:107AC000E8963FAFE8974CE1EC964FAFEC9756E461
:107AD000C957DF4F5883C758D040C857DF4F188267
:107AE000C858D040C757DF4F1882C958D040C65732
:107AF000DF4F1882CA58D040C557DF4F1882CB5885
:107B0000D040AB961CAE1DAE1EAE1FAEAB97A79677
:107B10001CAE1DAE1EAE1FAEA797C12CD12C760198
:107B2000CC56DF4F188219821A821B82C459D0406A
:107B300081E0C157DF4F8883CF58D040A1961FAE58
:107B40001EAEA19760961FAE609764961FAE6497B5
:107B500000E010E0D101AB56B14FC256DF4FB98300
:107B6000A883CE59D040C101880F991F880F991F53
:107B7000FC01E452FB4FC457DF4FF983E883CC5834
:107B8000D04080919A02882309F4C7C20E940A5308
:107B90006F966CAF7DAF8EAF9FAF6F978091820E67
:107BA000882309F46CC10E94DDD0FFEF2F163F0639
:107BB00079F42091E40460962FAF60973091E5044A
:107BC00064963FAF64970091E6041091E7041FC0EC
:107BD000C457DF4FA881B981CC58D040BC91609682
:107BE000BFAF6097C457DF4FE881F981CC58D040D0
:107BF000F1816496FFAF6497C457DF4FA881B981C4
:107C0000CC58D04012960C91129713961C91609606
:107C10002FAD609764963FAD6497A801C857DF4FBA
:107C20006881C858D040C757DF4F7881C958D040C5
:107C3000C657DF4F8881CA58D040C557DF4F98815B
:107C4000CB58D0400F94910287FF1AC06096BFAD09
:107C50006097C857DF4FB883C858D0406496EFADDF
:107C60006497C757DF4FE883C958D040C657DF4FE6
:107C70000883CA58D040C557DF4F1883CB58D0402F
:107C800060962FAD609764963FAD6497A801CD577D
:107C9000DF4F6881C358D040E8967FADE897EC96F7
:107CA0008FADEC97C957DF4F9881C758D0400F94DC
:107CB000F0081816B4F46096FFAD6097CD57DF4F0B
:107CC000F883C358D04064962FAD6497E8962FAFE1
:107CD000E897EC960FAFEC97C957DF4F1883C7585A
:107CE000D040C157DF4F3881CF58D040AC962FAD30
:107CF000AC97332309F493C0E0963FADE097E49648
:107D00004FADE497C158DF4F5881CF57D0406096B0
:107D10006FAD609764967FAD6497C8010F94F008CB
:107D200018160CF0ACC06F968CAD9DADAEADBFAD6E
:107D30006F9784199509A609B709C055DF4F888345
:107D40009983AA83BB83C05BD04088589341A10923
:107D5000B109B7FD94C0D501C4016B962CAD3DAD02
:107D60004EAD5FAD6B97821B930BA40BB50BB59516
:107D7000A795979587953FEF2316330619F48093BF
:107D8000920E07C0C256DF4FE881F981CE59D0402C
:107D90008083C055DF4F288139814A815B81C05B78
:107DA000D040CC56DF4F288339834A835B83C45944
:107DB000D040AC963FADAC97C857DF4F3883C8581A
:107DC000D040E0964FADE097C757DF4F4883C95882
:107DD000D040E4965FADE497C657DF4F5883CA584A
:107DE000D040C158DF4F8881CF57D040C557DF4FB3
:107DF0008883CB58D0406F962CAD3DAD4EAD5FAD76
:107E00006F97C057DF4F288339834A835B83C059FC
:107E1000D040C157DF4F1882CF58D04030C0E096D5
:107E20003FADE097E4964FADE497C158DF4F5881DE
:107E3000CF57D04060966FAD609764967FAD6497E2
:107E4000C8010F94910287FF1AC06F968CAD9DAD4B
:107E5000AEADBFAD6F97C057DF4F288139814A81E2
:107E60005B81C059D040821B930BA40BB50BAC01B6
:107E7000BD01485853416109710977FF80C620E070
:107E800030E040EA51E4AC966FADAC97E0967FAD40
:107E9000E097E4968FADE497C158DF4F9881CF57B4
:107EA000D0400F94CA069B01AC0160966FAD6097FD
:107EB00064967FAD6497C8010F94F00818166CF4AF
:107EC000E7EBF6E084918F010F5F1F4F882309F4E1
:107ED000AAC40E940669F801F5CF80E398EFAFEFDE
:107EE000BFEFC656DF4F288139814A815B81CA596D
:107EF000D040821B930BA40BB50B6F962CAD3DAD00
:107F00004EAD5FAD6F97820F931FA41FB51FB7FDD6
:107F100013C00E94188A8AE00E9406696F968CAD91
:107F20009DADAEADBFAD6F97C656DF4F88839983C9
:107F3000AA83BB83CA59D0406F968CAD9DADAEADC0
:107F4000BFAD6F97880F991FAA1FBB1FC057DF4F88
:107F5000288139814A815B81C059D040821B930BB3
:107F6000A40BB50B84199509A609B70981389F445C
:107F7000A241B10568F0E9E9F6E084918F010F5F55
:107F80001F4F882309F44FC40E940669F801F5CFFA
:107F9000A1964EAD5FADA197C856DF4F88819981FC
:107FA000C859D040841795070CF0B4C0ECE3F6E054
:107FB00084918F010F5F1F4F882321F00E94066973
:107FC000F801F6CF9FEF2916390619F009EC13E0F6
:107FD00002C007EE12E0B8018AE296E00E94EAC20F
:107FE000B701A60186E296E00E948DC28AE00E9457
:107FF0000669B80184E196E00E94EAC2A7964CADFA
:108000005DAD6EAD7FADA79780E196E00E948DC219
:108010008AE00E940669B8018EEF95E00E94EAC2EC
:10802000AB964CAD5DAD6EAD7FADAB978AEF95E095
:108030000E948DC28AE00E940669C257DF4FA88164
:10804000CE58D040AA2309F4EEC32320209489F50A
:10805000C0921115D0921215E0921315F0921415DA
:108060002CEA35EC47E25EE3A7966CAD7DAD8EADB4
:108070009FADA7970F94F60260930D1570930E15A0
:1080800080930F15909310152CEA35EC47E25EE3D0
:10809000AB966CAD7DAD8EAD9FADAB970F94A60743
:1080A0006093091570930A1580930B1590930C1526
:1080B000BAC3C0921D15D0921E15E0921F15F09202
:1080C00020152CEA35EC47E25EE3A7966CAD7DAD5A
:1080D0008EAD9FADA7970F94F6026093191570931C
:1080E0001A1580931B1590931C152CEA35EC47E26A
:1080F0005EE3AB966CAD7DAD8EAD9FADAB970F944F
:10810000A607609315157093161580931715909315
:10811000181589C30E9496C734CD80919A028111A7
:1081200082C30E94F7CF7FC30E94CCF97CC3D101E8
:108130008D911D01882309F4A3C0F701408051806F
:1081400062807380F801EA5DFD4F208131814281B8
:108150005381F801E15DFB4F6081718182819381E0
:108160000F94CA0620E030E040E05FE30F94F6028F
:108170009B01AC01C301B2010F94F008181644F43E
:10818000F801EE5DF64C85909590A590B49003C0F3
:10819000812C912C5401F801E651FC4E2081318153
:1081A00042815381C301B2010F94C9069B01AC0106
:1081B000C501B4010F94C9064B015C0120E030E019
:1081C00040EA51EC0F94F00887FD2BC020E030E02E
:1081D00040EA51E4C501B4010F94910218160CF164
:1081E000D6012D913D914D915C91C501B4010F9443
:1081F000C9069B01AC01C301B2010F94CA06F70185
:108200006083718382839383D6018D929D92AD9218
:10821000BC92139760968FAD6097820D0E94F29189
:108220002FC0E6ECF7E184918F010F5F1F4F882389
:1082300021F00E940669F801F6CFE9E4F7E08491A5
:108240008F010F5F1F4F882321F00E940669F801FC
:10825000F6CF61E08BE397E00E9468C70E94115956
:1082600088E290E09A83898388EC90E099A388A3C0
:10827000BE016F5F7F4FCE0180960E94FE60D3C229
:10828000B4E0CB0ED11C0C5F1F4FE4E0EE0EF11CEE
:108290000C30110509F04BCF0E94344C0E94AF9E68
:1082A00060E08BE297E00E9468C783E992E099A3BF
:1082B00088A304E610E01A830983BE01605E7F4F45
:1082C000CE0101960E94FE608AEB92E099A388A3FA
:1082D0001A830983BE01605E7F4FCE0101960E9422
:1082E000FE60A1C20E9485DA9EC20E9466D59BC232
:1082F0000E9440F698C283E50E94B14C882319F091
:108300000E946F4C01C081E091E089270E943AF100
:108310008AC283E50E94B14C882309F484C20E947A
:108320006F4C809376077FC20E948761882319F083
:1083300081E00E942B8F84E50E94B14C811103C023
:10834000DD24DA940CC00E945E4CD0904605D8160D
:10835000B9F321E040E050E0BA010E94679A85E459
:108360000E94B14C882319F00E947E4C04C060E04A
:1083700070E080E090EC2F966CAF7DAF8EAF9FAF3A
:108380002F978AE50E94E04C882319F00E947E4CCA
:1083900004C060E070E080E291E42B966CAF7DAFAA
:1083A0008EAF9FAF2B9788E50E94E04C882319F091
:1083B0000E947E4C04C060E070E080E291E4279669
:1083C0006CAF7DAF8EAF9FAF279789E50E94E04CE1
:1083D000882319F00E947E4C04C060E070E085E8BC
:1083E00093E423966CAF7DAF8EAF9FAF239785E567
:1083F0000E94B14C882319F00E947E4C04C060E0BA
:1084000070E088EC92EC6BAF7CAF8DAF9EAF8CE4EC
:108410000E94B14C882319F00E947E4C03C060E09A
:1084200070E0CB0168A379A38AA39BA382E40E9496
:10843000E04C882321F00E944E4CF62E02C055E0FD
:10844000F52EB090100B80913B098111A4C0CC2473
:10845000C394EF2C8E01055C1F4F9E01215C3F4FA2
:10846000AE014D5B5F4FBE01695B7F4FCE01855B07
:108470009F4F0E94386B882309F48DC081E0809360
:10848000F10D11E08091F10D882309F470C060E0D6
:108490008F2D0E94E98C80918A0A90918B0A91110C
:1084A00003C0882309F45FC01093DE0D40E050E064
:1084B000BA018FE494E70E94D6538091F10D88238E
:1084C00021F081E00E945EEAF8CF1092620E1092D5
:1084D000630E1092640E1092650E10928A0A0E942A
:1084E0009FCF1092660E1092670E1092680E109237
:1084F000690E10928B0A81E00E949FCF0E947B8CB4
:108500001093DE0D40E050E0BA018EEB93E70E943D
:10851000D6530E940A53DC01CB0188539045AF4FDC
:10852000BF4F8093620E9093630EA093640EB0933E
:10853000650E10928A0A0E940A53DC01CB0188530F
:108540009045AF4FBF4F8093660E9093670EA093F8
:10855000680EB093690E10928B0A1093F10D61E0D2
:108560008F2D0E94E98C81E00E945EEA8BCF80E033
:1085700090E0A8E4B2E489839A83AB83BC838091C2
:108580003B09882341F04F2DBE016F5F7F4FCE0125
:1085900080960E94BF6C21E040E050E0BA018D2D32
:1085A0000E94679AF1E0BF123EC10E944D613BC13B
:1085B0001F5F143069F0D7018D917D010E94B14C8D
:1085C0008823B1F30E944E4C812F0E946CF9F0CFAA
:1085D00082E40E94B14C882329F00E944E4C84E032
:1085E0000E946CF983E50E94B14C882309F41BC1F9
:1085F00010E00E944E4C812F0E946CF91F5F1530D5
:10860000C1F711C183E50E94E04C882321F00E944C
:108610004E4C8B0102C000E010E080E50E94E04C6F
:10862000882321F00E944E4CCB0102C080E090E0F4
:10863000B8010E945DF9F7C083E50E94B14C811139
:1086400006C033E4E32E33E0F32E10E00EC010E05A
:108650000E945E4C682F812F0E9446F91F5F1530E3
:10866000B9F7EFCF1F5F143071F0F70181917F01EF
:108670000E94B14C8823B1F30E945E4C682F812F79
:108680000E9446F9EFCF82E40E94B14C882331F07A
:108690000E945E4C682F84E00E9446F90E94E4F735
:1086A000C2C083E50E94E04C882309F44BC00E94BD
:1086B0005E4C813049F0823009F044C093E4E92EE9
:1086C00093E0F92E10E023C023E4E22E23E0F22E03
:1086D00010E0D7018D917D010E94E04C882339F094
:1086E0000E945E4C4FEF682F812F0E949CF81F5F05
:1086F000143079F782E40E94E04C882319F10E943B
:108700005E4C4FEF682F1BC01F5F143079F0F701EC
:1087100081917F010E94E04C8823B1F30E945E4C5E
:10872000482F6FEF812F0E949CF8EECF82E40E94C9
:10873000E04C882339F00E945E4C482F6FEF84E0B4
:108740000E949CF80E94E4F76EC0E6ECF7E1849189
:108750008F010F5F1F4F882321F00E940669F801E7
:10876000F6CFE7E6F7E084918F010F5F1F4F882374
:1087700009F459C00E940669F801F5CF81E08093A1
:10878000780210924A0583E50E94B14C811103C022
:108790000E94ACED48C00E946F4C811144C0F8CFDC
:1087A0000091400480914605081751F083E50E942E
:1087B000B14C182F882329F00E946F4C182F01C04C
:1087C00011E086E40E94E04C882319F00E947E4C60
:1087D00003C060E070E0CB0120E030E040E752E40D
:1087E0000F94A607AB01BC01212F802F0E94679A2E
:1087F0001AC0E4EFF2E284918F010F5F1F4F8823CC
:1088000021F00E940669F801F6CF6091E0137091A3
:10881000E11386E797E00E94EAC282E20E940669BD
:108820008AE00E9406690E9442ED7AC340912C04BE
:1088300050912D04452B39F4AF014150510950930B
:108840002D0440932C0440E050E00C945E2A0E94DA
:108850004E4CAB01BC014093C20D5093C30D6093CD
:10886000C40D7093C50D81E19DE00E949079DBCF2E
:108870000E947E4C0F940E086739710514F066E96A
:1088800070E070930A0A6093090A0E9454CF0E9414
:108890007E4C20E030E040EA50E40F94F0081816D7
:1088A00014F40E944D616091090A70910A0A072E22
:1088B000000C880B990B0F9497022091E4043091DF
:1088C000E5044091E6045091E7040F94910260E0C2
:1088D00087FF03C086E893E002C089E793E00E9427
:1088E00068C781E080939A028091460580932E04A8
:1088F00067961CAE1DAE1EAE1FAE67976F961CAE80
:108900001DAE1EAE1FAE6F9760961FAE6097A0960D
:108910001FAEA0975CE3A4965FAFA4978CE1A896E6
:108920008FAFA89796E4AC969FAFAC97C12CD12C93
:1089300070E8E72EEFEBFE2E812C912C5401609114
:10894000090A70910A0A072E000C880B990B0F94E4
:108950009702162F072F782E692E262F372F482F94
:10896000592FB601C7010F949102882331F120914C
:10897000E4043091E5044091E6045091E704612F4E
:10898000702F872D962D0F949102881F8827881F9E
:1089900060968FAF60976896CFAC6897CC2089F0CF
:1089A000882379F080919A02882309F43CCF60E013
:1089B0008BE693E00E9468C736CF1C2D0D2D7E2CD0
:1089C0006F2C0E940A536B017C01DC01CB016F9676
:1089D0002CAD3DAD4EAD5FAD6F97821B930BA40BDD
:1089E000B50BB7FD3DC0D701C60188519C4FAF4FB5
:1089F000BF4F6F968CAF9DAFAEAFBFAF6F970E946A
:108A0000188AE5E7F3E084912F019FEF491A590A8C
:108A1000882321F00E940669F201F5CF81149104A8
:108A2000A104B104B9F0D501C40188519C4FAF4FE6
:108A3000BF4FBC01CD016C197D098E099F0928EE3D
:108A400033E040E050E00F946C06CA01B9010E9487
:108A5000C56903C08FE30E9406698AE00E94066927
:108A600080E00E945EEA0E9462532090E40430900D
:108A7000E5044090E6045090E7049101A201612FC3
:108A8000702F872D962D0F94C9069F7720E030E038
:108A900040EA50E481149104A104B10429F40F9434
:108AA000910287FF07C004C00F94F008181614F451
:108AB000460157016096AFAD6097AA2309F443C001
:108AC00067962CAD3DAD4EAD5FAD67972115310575
:108AD0004105510541F0D701C601821B930BA40B40
:108AE000B50BB7FD30C09101A201A0966FADA09764
:108AF000A4967FADA497A8968FADA897AC969FAD8E
:108B0000AC970F94C90620E030E040EC5FE30F948F
:108B1000910287FD47CFD701C601805A9541AF4FDB
:108B2000BF4F67968CAF9DAFAEAFBFAF6797A096B4
:108B30002FAEA097A4963FAEA497A8964FAEA89745
:108B4000AC965FAEAC9780919A02882309F42ACF45
:108B500081149104A104B10429F4C12ED02EE72C74
:108B6000F62CEDCE98EEC91A93E0D90AE108F10887
:108B7000C818D908EA08FB08F7FE14CFEECFA19673
:108B80004EAD5FADA197141615060CF05EC1CC5624
:108B9000DF4F488059806A807B80C459D040480E9E
:108BA000591E6A1E7B1ECC56DF4F288139814A81AF
:108BB0005B81C459D040281B390B4A0B5B0BCA019F
:108BC000B9016B962CAD3DAD4EAD5FAD6B970F947B
:108BD0005D06A30192010F948E06820E931EA41EC1
:108BE000B51E34E183169104A104B1040CF47FC1D5
:108BF000C056DF4F88819981AA81BB81C05AD0407D
:108C000088169906AA06BB060CF081C1C855DF4F2D
:108C1000288139814A815B81C85AD040281539059D
:108C20004A055B059CF4C455DF4F88819981AA8170
:108C3000BB81CC5AD04088199909AA09BB096B9607
:108C40008CAF9DAFAEAFBFAF6B9706C06B968CAECF
:108C50009DAEAEAEBFAE6B97B501A40183E297E0C7
:108C60000E94AAC26B964CAD5DAD6EAD7FAD6B97A9
:108C70008EE197E00E94AAC2CD57DF4F4881C358CA
:108C8000D040E8965FADE897EC966FADEC97C9578A
:108C9000DF4F7881C758D04087E197E00E948DC2AE
:108CA000C857DF4F4881C858D040C757DF4F588159
:108CB000C958D040C657DF4F6881CA58D040C55701
:108CC000DF4F7881CB58D04080E197E00E948DC281
:108CD000A196AEADBFADA19713970CF4B6C06B963D
:108CE0006CAD7DAD8EAD9FAD6B970F94970220E07C
:108CF00030E040E850E40F94F6026B017C01CD5760
:108D0000DF4F2881C358D040E8963FADE897EC96F6
:108D10004FADEC97C957DF4F5881C758D040C8575F
:108D2000DF4F6881C858D040C757DF4F7881C95896
:108D3000D040C657DF4F8881CA58D040C557DF4F53
:108D40009881CB58D0400F94C9062BED3FE049E401
:108D500050E40F94F60220E030E040E05FE30F942F
:108D6000F6029B01AC01C701B6010F94A6076B0187
:108D70007C01C301B2010F9497022FE632E143E870
:108D80005AE30F94F6022B013C01B701A6018AE0D9
:108D900097E00E948DC2B301A20184E097E00E9497
:108DA0008DC22AE939E949E15FE3C701B6010F94B1
:108DB000F6026B017C019B01AC010F94CA06A30172
:108DC00092010F94A607A7966CAF7DAF8EAF9FAFB1
:108DD000A797A3019201C701B6010F94F60220E004
:108DE00030E040E05EE30F94F602AB966CAF7DAFEF
:108DF0008EAF9FAFAB97E4EFF6E084913F01BFEFFA
:108E00006B1A7B0A882321F00E940669F301F5CFD3
:108E1000B701A6018EEE96E00E948DC2A7964CADDA
:108E20005DAD6EAD7FADA79788EE96E00E948DC2D6
:108E3000AB964CAD5DAD6EAD7FADAB9782EE96E07F
:108E40000E948DC28AE00E9406696B968CAD9DAD32
:108E5000AEADBFAD6B97880D991DAA1DBB1DB59515
:108E6000A79597958795EFEF2E163E0619F48093F8
:108E7000920E07C0C256DF4FE881F981CE59D0402B
:108E80008083A1962EAD3FADA1972F5F3F4FA19656
:108E90003FAF2EAFA197AC963FADAC97CD57DF4F0C
:108EA0003883C358D040E0964FADE097E8964FAF77
:108EB000E897E4965FADE497EC965FAFEC97C15806
:108EC000DF4F8881CF57D040C957DF4F8883C758BD
:108ED000D0406F964CAC5DAC6EAC7FAC6F9791E0C0
:108EE000C157DF4F9883CF58D0400C943F3F84E167
:108EF000882E912CA12CB12C24E130E040E050E0F0
:108F00006B962CAF3DAF4EAF5FAF6B97A5CECC55F8
:108F1000DF4F88809980AA80BB80C45AD04083CE1E
:108F2000CD54DF4F0FB6F894DEBF0FBECDBFDF913B
:108F3000CF911F910F91FF90EF90DF90CF90BF9056
:108F4000AF909F908F907F906F905F904F903F90E9
:108F50002F90089590915615E92FF0E0EE58F84FB4
:108F600080839F5F943018F49093561502C010923E
:108F70005615809119098F5F809319090895CF9232
:108F8000DF92EF92FF920F931F93CF93DF936C01C9
:108F90007A018B01C0E0D0E0CE15DF0589F0D80161
:108FA0006D918D01D601ED91FC910190F081E02D44
:108FB000C6011995892B11F47E0102C02196ECCFD0
:108FC000C701DF91CF911F910F91FF90EF90DF903C
:108FD000CF900895089580E090E0089580E008958E
:108FE0000B96FC01849108950A96FC0184910895E2
:108FF000FC0184910895FCDF882321F0823011F078
:1090000083E0089586E00895FC01E60FF11D849148
:1090100090E0982F88273196E4918E0F911D089546
:1090200068E0F2CF66E0F0CF0895FC01A681B78139
:109030008281481B8581483018F0A80FB11D477008
:10904000382F369536953695562F577080E890E034
:1090500002C0959587955A95E2F7439F402D1124BC
:10906000669566956695E62FF0E0E40FF11DEA0F30
:10907000FB1F3081222311F0832B02C080958323B4
:1090800080830895FB014181DC0112962C91129797
:10909000421760F013962C911397241738F06081D3
:1090A00015962C91621710F42481BFCF0895FC010E
:1090B00080819281980F92832181921760F494812C
:1090C0009F5F94839381890F821710F08FEF820F37
:1090D000838381E0089580E00895FC0112828081FD
:1090E000815083831482089581E00895089590E06B
:1090F000FC013197E231F10508F04EC08827EE58A7
:10910000FF4F8F4F0D94B509809180008F7703C07A
:10911000809180008F7D80938000089580918000F1
:10912000877FF9CF84B58F7702C084B58F7D84BDEA
:1091300008958091B0008F7703C08091B0008F7D3B
:109140008093B0000895809190008F7707C0809140
:1091500090008F7D03C080919000877F8093900066
:1091600008958091A0008F7707C08091A0008F7D27
:1091700003C08091A000877F8093A0000895809114
:1091800020018F7707C0809120018F7D03C08091DF
:109190002001877F8093200108953FB7F894809144
:1091A000480490914904A0914A04B0914B0426B51B
:1091B000A89B05C02F3F19F00196A11DB11D3FBF0F
:1091C000BA2FA92F982F8827820F911DA11DB11D9D
:1091D000BC01CD0142E0660F771F881F991F4A9599
:1091E000D1F70895EF92FF920F931F93CF93DF93E0
:1091F0001F92CDB7DEB7082F162FE6ECF7E184916A
:109200007F012FEFE21AF20A882331F099830E943E
:109210000669F7019981F3CFE02FF92F84917F013F
:109220009FEFE91AF90A882321F00E940669F701E5
:10923000F5CF6091C5137091C6138091C7139091BB
:10924000C8130E94C5698AE00E94066911110E9434
:10925000ACED1092B3041092B2040F90DF91CF9155
:109260001F910F91FF90EF900895CF93FC018081A3
:109270008B33A1F080911909843080F4C62FBF018F
:109280008091561520E6829FC00111248856984F80
:109290000F94040A8C2F5EDE81E001C080E0CF9144
:1092A0000895DF92EF92FF920F931F93CF93DF9376
:1092B000CDB7DEB76E970FB6F894DEBF0FBECDBF49
:1092C00060915607709157076115710501F14DE1E5
:1092D00050E0CE0101967C010F9401021E8EF70131
:1092E0008F010E191F09D190DD2019F09AE0D912D3
:1092F000F7CFF701E00FF11F108260E0C701B5DF83
:10930000882329F0C7010E94A7E9811109C081E0E3
:109310002091560730915707232BA1F480E012C00B
:10932000DD2049F00F5F1F4F80915607909157073E
:10933000080F191F02C000E010E0109357070093B8
:109340005607E5CF6E960FB6F894DEBF0FBECDBFC1
:10935000DF91CF911F910F91FF90EF90DF900895D3
:109360002F923F924F925F927F928F929F92AF92F5
:10937000BF92CF92DF92EF92FF920F931F93CF9302
:10938000DF931F92CDB7DEB78CDF81115AC2809177
:109390001909843058F42FB7F8948091BD09909141
:1093A000BE092FBF891B8F7709F044C180911F0B25
:1093B000882309F446C280911909811102C01092D4
:1093C000B604EE24E3944091C20D5091C30D609118
:1093D000C40D7091C50D8091BE0D9091BF0DA091EF
:1093E000C00DB091C10D481759076A077B0708F4F3
:1093F000E12C00E010E09924939480E6882E93ED10
:10940000C92E98E0D92E2FECA22E28E0B22E3DE8EE
:10941000732E80911909843008F013C2E11011C233
:109420008091B60481110DC28091190D90911A0D91
:10943000A0911B0DB0911C0D8093C20D9093C30D94
:10944000A093C40DB093C50D41E050E0BE016F5F25
:109450007F4F81E19DE00E948F7D019719F4898102
:1094600090E002C08FEF9FEFF82EEE24E39420905F
:10947000C20D3090C30D4090C40D5090C50D409169
:10948000BE0D5091BF0D6091C00D7091C10D24169D
:10949000350646065706C8F4E12C8F3FFFEF9F07BD
:1094A00009F47AC02AE0821709F495C08DE0F81615
:1094B00009F491C093E2F91619F0EAE3FE12A0C094
:1094C0008091B50481119CC081C0EEEEF8E08491DA
:1094D0002F012FEF421A520A882321F00E940669B9
:1094E000F201F5CF0E94CCF981E19DE00E94C97A9A
:1094F00080912C0D882359F1815080932C0D789EFA
:10950000C001112441E061E08F5C924F0E94885CB1
:10951000E0912C0D84E0E89FF0011124E35DF24F0F
:1095200040815181628173814093C20D5093C30D7C
:109530006093C40D7093C50D81E19DE00E94907908
:109540008091200B8823C1F090921F0B15C01092C0
:109550001F0BD0925707C0925607A3DE0E940EBF82
:109560000E947BC06D3371058105910528F0B09292
:109570005707A092560795DE1092CA0D8091200BD6
:10958000882319F00E94065F21C00E94B75F809176
:10959000200B8111F7CF1AC0E6ECF7E184912F017F
:1095A0009FEF491A590A882321F00E940669F201A7
:1095B000F5CFEFEDF8E084912F012FEF421A520A18
:1095C000882321F00E940669F201F5CF83E2F812A8
:1095D00002C09092B6041092B5040115110509F469
:1095E00018CF80915615889E000D111D1124F80189
:1095F000E856F84F108280E0ADDC00E010E009CFC3
:109600000F35110508F005CF9BE3F91202C09092C7
:10961000B5048091B5048111FCCE80915615F801F6
:10962000889EE00DF11D1124E856F84FF0820F5F7F
:109630001F4FEFCE0E94506A2091B2043091B304C4
:109640008A3019F08D3009F0CBC01092B404211586
:10965000310509F49CCEF901EE5AFB4F10821092AD
:10966000B3041092B20422E534E08901F90180814B
:109670002F5F3F4F8032C9F378018E3411F000E044
:1096800010E06AE270E0C7010F94F9096C0101155E
:10969000110509F474C06AEC78E0C7010F94100258
:1096A000BB24B394892B11F4B12C09C06EE470E093
:1096B000C70104960F94F909009709F08C014AE05C
:1096C00050E060E070E0C80101960E9485FF609361
:1096D0004E0470934F048093500490935104009172
:1096E000C5131091C6132091C7133091C8130F5F93
:1096F0001F4F2F4F3F4F601771078207930731F0BD
:10970000B11004C061E087E998E026C0C114D1041B
:1097100001F180E010E0F701E80FF11D90819A322D
:1097200019F08F5F1927F7CF4AE050E060E070E052
:10973000C60101960E9485FF012F10E020E030E075
:10974000601771078207930749F061E088E798E0A6
:1097500003C061E08EE498E045DD28CE80914E04A0
:1097600090914F04A0915004B09151048093C5137F
:109770009093C613A093C713B093C81306C0892B48
:1097800021F060E083EA97E0E7CF809178028111D1
:1097900022C067E470E0C7010F94F9090097D9F07F
:1097A0004AE050E060E070E001960E9485FF64307E
:1097B000710588F4E7EDF7E084918F010F5F1F4F8B
:1097C000882321F00E940669F801F6CF60E08DEC55
:1097D00097E00E9468C761E082E594E046DDD7CD5E
:1097E0002F3531050CF0D3CD8C35B1F42FB7F8946B
:1097F0008091BD099091BE092FBF891B8F7709F415
:10980000C6CD0E94506A9091B4049111C0CD2091B0
:10981000B2043091B30409C08B3319F491E09093F2
:10982000B4049091B4049111B2CDA9014F5F5F4F80
:109830005093B3044093B204F901EE5AFB4F808376
:10984000A6CD0F90DF91CF911F910F91FF90EF90D8
:10985000DF90CF90BF90AF909F908F907F905F9060
:109860004F903F902F9008952DE235E049E255E06A
:1098700065E275E081E295E00C94C6E680914C04C7
:1098800090914D04009731F04AE050E060E070E0C4
:109890000D94AD0060E070E0CB01089580914C0420
:1098A00090914D04009731F04AE050E060E070E0A4
:1098B0000C9485FF60E070E0CB010895EFDF97FD29
:1098C0000AC0ECDF6F3F71058105910509F02CF4AA
:1098D000E5DF862F089580E008958FEF0895809149
:1098E0004C0490914D04892B31F0E8DF91E0811117
:1098F00003C090E001C091E0892F08950F931F935A
:10990000CF9380914C0490914D040097F1F0FC01AD
:109910008F01C1912C2F2F7D89F0C53411F0C536F0
:10992000B9F7F801108260E070E00E941EFEF801B5
:10993000C083562F472F382F292F0BC060E070E0CF
:10994000CF911F910F910C941EFE50E040E030E04B
:1099500020E0652F742F832F922FCF911F910F91AD
:10996000089581548A3150F5482F50E0FA0193E070
:10997000F595E7959A95E1F7E85DFB4F208130E09A
:109980008770B90102C0759567958A95E2F760FF07
:1099900015C0FA01E25FFB4F2081222339F080914C
:1099A000E0139091E113820F911D02C080E090E0DE
:1099B00090934D0480934C0481E0089580E00895D5
:1099C000D0DF882341F081E020914C0430914D0498
:1099D000232B09F480E00895FC01238121110C94CC
:1099E000C97A0895CF93DF939091EF0991111CC02C
:1099F00094E0899FE0011124C452DB4F60911E0264
:109A000070911F02072E000C880B990B0F94970280
:109A10009B01AC01688179818A819B810F949102BD
:109A2000881F8827881F01C080E0DF91CF910895AB
:109A30008091F00A9091F10A891B8F700895CF925E
:109A4000DF92FF920F931F93CF93DF931F921F928A
:109A5000CDB7DEB76901DB0112960D911C9113970A
:109A6000423309F470C0B8F4453109F477C0473186
:109A700009F487C0443109F09DC0D80115962C9196
:109A800015971696ED91FC911797CF01820F911DB6
:109A9000820F911D5CC0463409F483C0473409F439
:109AA00084C04B3309F086C0F901818193819130E4
:109AB00029F0933031F4482F885004C048E0480F13
:109AC00001C0482F21E0D80113963C91381708F4C3
:109AD00020E031E0F8015281451708F430E051E010
:109AE000481708F050E0822F852B382319F42523DE
:109AF00009F460C0D6011296FC90913051F030F01C
:109B0000923049F0933051F42FEF09C020E031E05A
:109B100007C021E004C020E03FEF02C020E030E0B9
:109B2000F7FE07C0B601C8012A833983ABDA398151
:109B30002A81F6018081830F80838181820F818356
:109B4000FF0C71F737C0B901C8019CDA33C011921C
:109B5000E817F907E1F7C801C0DA2CC0C801A7DA95
:109B6000882349F1F80125810680F781E02DCF0196
:109B7000820F911D820F911D1192E817F907E1F7ED
:109B800019C0D9011C92F801828111968C9311970A
:109B90008581815012968C931297838113968C93B2
:109BA00009C0D80115968C9103C0D80111968C91EB
:109BB000F601808381E00F900F90DF91CF911F918C
:109BC0000F91FF90DF90CF90089588E290E0019789
:109BD000F1F708952EE93FE0009729F0F901319758
:109BE000F1F70197F9CF08950F93FC010150040F8D
:109BF00084A996A9941718F0081728F402C008172A
:109C000050F0041740F42150260F83A995A9961708
:109C100020F4281720F480E007C0281720F481E002
:109C2000261710F0F8CF81E00F910895DB01ED9138
:109C3000FC9119942F923F925F926F927F928F9234
:109C40009F92AF92BF92CF92DF92EF92FF920F93CB
:109C50001F93CF93DF931F92CDB7DEB71C01C62EA3
:109C6000142FD22EDC011496ED90FC901597C701AD
:109C7000BFD9082FF10184819581BDD9982E01307B
:109C800019F48FE0A82E02C0AA24AA94D101149638
:109C90008D919C911597A8D9082FF1018481958108
:109CA0009FD9B82ED10114968D919C911597B8D952
:109CB000B0E6BD1530F4009721F0E80EF91E01E67C
:109CC00010C0F10184819581ADD9F0E4FD1530F427
:109CD000009721F0E80EF91E01E403C021E1E20E35
:109CE000F11CBD1480F4D10150961C9250975396EC
:109CF0001C92539754961C92549751961C925197CC
:109D000052961C92C3C0B01670F3892D90E0F701F3
:109D100024912F3F21F4FFEFEF1AFF0A59C00D11D4
:109D20004EC0D10114968D919C91159761D99701E0
:109D30002F5F3F4FF701882311F08230E1F48491C7
:109D4000D10153968C935397F901249154962C93F7
:109D50005497F7013396E4915096EC935097F7019E
:109D60003496E4915196EC935197F7013596E4912E
:109D70005296EC9320C08491982F9F709250D101FD
:109D800052969C93529782958F7051968C935197CF
:109D9000F9012491822F8F7054968C9354972295B9
:109DA0002F7053962C935397F7013296E491E295D6
:109DB000EF705096EC93E114F10479F467C0F70169
:109DC0003296E491EA219C012E0F311DE20EF31E22
:109DD0000B1509F488CF0F5F9ACFF101848195812B
:109DE0000AD9B82ED10153969C9053975496DC9083
:109DF000549751968C915197C80E52969C919D0DF7
:109E0000512E591A0D2D292D452D6C2DC101ECDE39
:109E10008823C9F1C7018B0D911D5C0187E0890D75
:109E2000F82EF694F694F694D50C41019CE1890E37
:109E3000911C6F2C712C5D1431F15C2D8501802FEC
:109E40008A198F15E0F4F8018491D10112966D9171
:109E50007C9113975C965C935C975D965C925D97A2
:109E60005F961C925F975E968C9394014BE3C101C1
:109E70005983DCDE0F5F1F4F5981585FE0CFA60C7E
:109E8000B71C5394D8CFF101808901C080E00F90B6
:109E9000DF91CF911F910F91FF90EF90DF90CF90C6
:109EA000BF90AF909F908F907F906F905F903F900A
:109EB0002F9008958F929F92BF92CF92DF92EF9250
:109EC000FF920F931F93CF93DF931F92CDB7DEB70F
:109ED0004C01062FF42E122F522FE62EE20EBB2439
:109EE000BA946C018CE1C80ED11C8E2D851B5830A4
:109EF00078F0F40162817381848FF58E178EB68EAF
:109F000096014BE3C401598391DE59815850EDCF3E
:109F1000812F887F080F212F277019F187E02827CC
:109F2000F40162817381048FF58E178E2F5F277085
:109F30008FEF90E001C0880F2A95EAF7868F940191
:109F4000245E3F4F4BE3C4010F90DF91CF911F91EF
:109F50000F91FF90EF90DF90CF90BF909F908F90E8
:109F600065CE0F90DF91CF911F910F91FF90EF90F1
:109F7000DF90CF90BF909F908F900895EF92FF92C7
:109F80000F931F93CF93DF937C01D62F122FC42FF3
:109F9000040F212F4C2F6D2FC7018CDFCF5F0C13C7
:109FA000F8CFDF91CF911F910F91FF90EF9008951F
:109FB000DF92EF92FF920F931F93CF93DF93EC0109
:109FC000162FF42EE22E10DE882329F02E2D4F2D91
:109FD000612FCE01D3DFDF91CF911F910F91FF90C1
:109FE000EF90DF900895EF92FF920F931F93CF931E
:109FF000DF931F92CDB7DEB78C01DC011296ED9096
:10A00000FC901397D196ED91FC91D29782E019952F
:10A0100020E030E04AE0B701C80108DEF82ED801A0
:10A02000D196ED91FC91D29783E01995D801D19604
:10A03000ED91FC91D29780E01995FF2081F1F80114
:10A04000628173819E012F5F3F4F46E4C801EEDDC0
:10A050008981D8018C9312966D917C9113979E0102
:10A060002F5F3F4F47E4C801E1DD8981F80181831B
:10A070006281738120E030E048E4C801D7DDD80177
:10A080001B968C931B9798012D5C3F4F12966D91F8
:10A090007C91139747E1C801C9DD81E001C080E0F0
:10A0A0000F90DF91CF911F910F91FF90EF90089546
:10A0B0001F920F920FB60F9211240BB60F922F938F
:10A0C0003F934F935F936F937F938F939F93AF9340
:10A0D000BF93EF93FF93E0910E02F0910F02199559
:10A0E000FF91EF91BF91AF919F918F917F916F9170
:10A0F0005F914F913F912F910F900BBE0F900FBE2C
:10A100000F901F9018951F920F920FB60F92112467
:10A110000BB60F922F933F934F935F936F937F9361
:10A120008F939F93AF93BF93EF93FF93E0910C02B4
:10A13000F0910D021995FF91EF91BF91AF919F9111
:10A140008F917F916F915F914F913F912F910F90E0
:10A150000BBE0F900FBE0F901F9018951F920F927D
:10A160000FB60F9211240BB60F922F933F934F937C
:10A170005F936F937F938F939F93AF93BF93EF936F
:10A18000FF93E0910202F09103021995FF91EF9184
:10A19000BF91AF919F918F917F916F915F914F91FF
:10A1A0003F912F910F900BBE0F900FBE0F901F90FD
:10A1B00018951F920F920FB60F9211240BB60F92A3
:10A1C0002F933F934F935F936F937F938F939F93BF
:10A1D000AF93BF93EF93FF93E0910002F0910102E0
:10A1E0001995FF91EF91BF91AF919F918F917F91C1
:10A1F0006F915F914F913F912F910F900BBE0F90F8
:10A200000FBE0F901F9018951F920F920FB60F92CE
:10A2100011240BB60F922F933F934F935F936F933D
:10A220007F938F939F93AF93BF93EF93FF93E091AF
:10A230000A02F0910B021995FF91EF91BF91AF9136
:10A240009F918F917F916F915F914F913F912F914E
:10A250000F900BBE0F900FBE0F901F9018951F927E
:10A260000F920FB60F9211240BB60F922F933F93BC
:10A270004F935F936F937F938F939F93AF93BF930E
:10A28000EF93FF93E0910802F09109021995FF9175
:10A29000EF91BF91AF919F918F917F916F915F915E
:10A2A0004F913F912F910F900BBE0F900FBE0F90CB
:10A2B0001F9018951F920F920FB60F9211240BB694
:10A2C0000F922F933F934F935F936F937F938F934F
:10A2D0009F93AF93BF93EF93FF93E0910602F091AA
:10A2E00007021995FF91EF91BF91AF919F918F91C7
:10A2F0007F916F915F914F913F912F910F900BBE86
:10A300000F900FBE0F901F9018951F920F920FB6CF
:10A310000F9211240BB60F922F933F934F935F939D
:10A320006F937F938F939F93AF93BF93EF93FF931D
:10A33000E0910402F09105021995FF91EF91BF9110
:10A34000AF919F918F917F916F915F914F913F91CD
:10A350002F910F900BBE0F900FBE0F901F9018956E
:10A36000CF93DF93282F30E0F901EF5EF94E84910F
:10A37000F901E254FC4DD491F901E858FC4DC49127
:10A38000CC2391F081110E947748EC2FF0E0EE0F82
:10A39000FF1FE757F84FA591B491EC91ED2381E0B1
:10A3A00090E021F480E002C080E090E0DF91CF9166
:10A3B00008951F93CF93DF93282F30E0F901EF5ECC
:10A3C000F94E8491F901E254FC4DD491F901E85819
:10A3D000FC4DC491CC23C9F0162F81110E947748FF
:10A3E000EC2FF0E0EE0FFF1FEC5BFC4DA591B4915C
:10A3F0008FB7F894111105C09C91ED2FE095E923DA
:10A4000002C0EC91ED2BEC938FBFDF91CF911F91A8
:10A4100008951F93CF93DF93182FEB010E940BBD7C
:10A42000209711F460E004C0CF3FD10531F461E022
:10A43000812FDF91CF911F91BCCFE12FF0E0EF5E34
:10A44000F94EE4914E2F50E0FA013197E231F105D7
:10A4500008F09DC08827EC57FF4F8F4F0D94B5092A
:10A4600084B5806884BDC7BD97C084B5806284BD53
:10A47000C8BD92C080918000806880938000D09396
:10A480008900C093880088C080918000806280939A
:10A490008000D0938B00C0938A007EC080918000A2
:10A4A000886080938000D0938D00C0938C0074C02E
:10A4B0008091B00080688093B000C093B3006CC0FE
:10A4C0008091B00080628093B000C093B40064C0FB
:10A4D00080919000806880939000D0939900C09301
:10A4E00098005AC080919000806280939000D09331
:10A4F0009B00C0939A0050C0809190008860809328
:10A500009000D0939D00C0939C0046C08091A00015
:10A5100080688093A0008091A0008F7B8093A00032
:10A52000D093A900C093A80037C08091A00080629A
:10A530008093A000D093AB00C093AA002DC080915F
:10A54000A00088608093A000D093AD00C093AC00C1
:10A5500023C080912001806880932001D09329013D
:10A56000C093280119C0809120018062809320014E
:10A57000D0932B01C0932A010FC0809120018860E5
:10A5800080932001D0932D01C0932C0105C0C038C9
:10A59000D1050CF04CCF46CFDF91CF911F9108959C
:10A5A0008F929F92AF92BF92CF92DF92EF92FF92E3
:10A5B0006B017C010E94CD484B015C01C114D104A8
:10A5C000E104F104F1F00E94CD48DC01CB018819CF
:10A5D0009909AA09BB09883E9340A105B10570F30A
:10A5E00021E0C21AD108E108F10888EE880E83E064
:10A5F000981EA11CB11CC114D104E104F10419F787
:10A60000DDCFFF90EF90DF90CF90BF90AF909F9005
:10A610008F9008952FB7F894609144047091450489
:10A6200080914604909147042FBF08950F931F9384
:10A63000CF93DF93EC01EEDF0E811F8128853985F2
:10A64000011511052105310559F52C852223A9F1A4
:10A650003A8521502C8721E0230F2A874D8524132A
:10A6600001C01A86FE0124E0329FE00DF11D112485
:10A6700006851785208931890A831B832C833D83B6
:10A68000DC01CB01800F911FA11DB11D8E839F8323
:10A69000A887B9878C819D81892B79F0769A0DC026
:10A6A000DC01CB01801B910BA20BB30BB7FD05C0E6
:10A6B00076981E821F8218861986DF91CF911F918E
:10A6C0000F910895A7DF6093E2137093E3138093D3
:10A6D000E4139093E51308951F920F920FB60F9213
:10A6E00011242F933F938F939F93AF93BF938091A8
:10A6F000440490914504A0914604B09147043091E0
:10A70000430423E0230F2D3720F40196A11DB11D32
:10A7100005C026E8230F0296A11DB11D2093430416
:10A720008093440490934504A0934604B093470457
:10A730008091480490914904A0914A04B0914B043F
:10A740000196A11DB11D8093480490934904A093E4
:10A750004A04B0934B04BF91AF919F918F913F9169
:10A760002F910F900FBE0F901F9018958091DB04D2
:10A770008630D8F496E0899FF0011124E954FB4F0C
:10A780002091100230911102318320834091FC040A
:10A790005091FD046091FE047091FF044283538345
:10A7A000648375838F5F8093DB040895209110028A
:10A7B0003091110228173907D9F090931102809334
:10A7C00010024093FC045093FD046093FE047093C8
:10A7D000FF04895F934521F41092DE0D1092DB0493
:10A7E00082E08093120281E08093E2091092EA0DE8
:10A7F00008954F925F926F927F928F929F92AF9245
:10A80000BF92CF92DF92EF92FF920F931F93CF935D
:10A81000DF93CDB7DEB72A970FB6F894DEBF0FBE31
:10A82000CDBF1092E90D8091F00D882349F00E9470
:10A83000CFEF40E050E0BA0187ED99EFB7DFDAC41F
:10A8400020912402309125024091FC045091FD0496
:10A850006091FE047091FF04C901840F951F243696
:10A86000310524F4853691053CF416C024363105B3
:10A8700031F08436910584F484E690E00DC04B30CD
:10A8800051056105710514F00A9706C0463F5F4FF8
:10A890006F4F7F4F6CF40A969093250280932402A9
:10A8A0001092FC041092FD041092FE041092FF041A
:10A8B00080912402909125028A3091053CF0883ED7
:10A8C00043E094072CF087EE93E002C08AE090E02A
:10A8D00090932502809324020E9470CAF82E0E9451
:10A8E000EBC68091C60A853198F4FF2049F080912B
:10A8F000050A9091060A892B19F004EF14E102C0B1
:10A9000007ED13E123E14FE061E089E00E9464BDBF
:10A910008091C60A8D3108F098C1ABE08A2EAAE07A
:10A920009A2EBAE8CB2EBAE0DB2E1CEDA12E14E055
:10A93000B12E1DE002E1602E712C87E0E82E9CE133
:10A94000592E4424439408EF010F8091C60A8830A1
:10A95000D8F5F6018081F11002C0811135C0F401F3
:10A9600060817181072E000C880B990B0F94970260
:10A9700020E030E040E05FE30F94CA060F940E0839
:10A98000643671052CF46A30710524F426E003C0A6
:10A9900022E101C02CE0A301421B51099A0157FF9B
:10A9A00002C02F5F3F4F35952795502F521B509374
:10A9B000C90AE092CA0ACB010E9499C50E9483F09D
:10A9C00084ED93E10E9476F08091C60A8D3198F56E
:10A9D0008091C80A853178F120E030E040E05FE303
:10A9E000F50160817181828193810F94CA060F9471
:10A9F0000E089B01643671050CF0F7C22A30310550
:10AA00000CF0F1C226E0F301E21BF1099F01F7FF10
:10AA100002C02F5F3F4F35952795021B0093C90A4F
:10AA20005092CA0ACB010E9499C50E9483F084ED1E
:10AA300093E10E9476F08091C60A853110F58091ED
:10AA4000C80A8131F0F0F40160817181072E000C99
:10AA5000880B990B0F949702F50120813181428177
:10AA600053810F94F00818160CF0C1C21092B20A6C
:10AA700002E022E041E1612F82E99AE099DA409216
:10AA8000B20A175EF2E08F0E911C2FEFC21AD20AA3
:10AA900044E0A40EB11C1F3309F055CF8091C60AC3
:10AAA000883008F03FC080917D0AF11002C081110A
:10AAB00039C06091090A70910A0A072E000C880BB0
:10AAC000990B0F94970220E030E040E05FE30F9491
:10AAD000CA060F940E08643671052CF46A307105AD
:10AAE00024F446E003C042E101C04CE022E130E042
:10AAF000241B310937FF02C02F5F3F4F3595279543
:10AB00003195219531092F5A2093C90A27E02093C6
:10AB1000CA0ACB010E9499C50E9483F084ED93E19B
:10AB20000E9476F08091C60A8D31D0F58091C80AD6
:10AB30008531B0F120E030E040E05FE36091E40473
:10AB40007091E5048091E6049091E7040F94CA06A1
:10AB50000F940E089B01643671050CF053C22A3025
:10AB600031050CF04DC246E022E130E0241B3109F2
:10AB700037FF02C02F5F3F4F3595279531952195BF
:10AB800031092F5A2093C90A2CE12093CA0ACB011C
:10AB90000E9499C50E9483F084ED93E10E9476F0B3
:10ABA0008091C60A853138F58091C80A813118F143
:10ABB0006091090A70910A0A072E000C880B990B04
:10ABC0000F9497022091E4043091E5044091E6044B
:10ABD0005091E7040F94F00818160CF015C210926B
:10ABE000B20A02E022E042E168E582E99AE0E0D9B7
:10ABF00081E08093B20A8091C60A8C3130F5809151
:10AC0000C80A843110F18091050A9091060A0196D4
:10AC100044E6489F9001499F300D112437FF02C040
:10AC200021503F4F832F932F990F990B009769F075
:10AC300028E62093C90A2BE12093CA0A0E9499C5ED
:10AC40000E9483F085E20E9466BE8091C60A84332A
:10AC500028F48091C80A8A3208F0DFC18091C60AC0
:10AC6000853328F48091C80A813308F0FCC18091B3
:10AC70001F0B882309F44AC08091C60A843308F068
:10AC800045C08091C80A823308F440C02091140D59
:10AC9000222319F18091BE0D9091BF0DA091C00D9E
:10ACA000B091C10D0097A105B10509F4E1C1BC0146
:10ACB000CD016D597F4F8F4F9F4F24E630E040E02C
:10ACC00050E00F946C066091C20D7091C30D80919D
:10ACD000C40D9091C50D0F946C0658E4259FB001EA
:10ACE0001124072E000C880B990B0F9497022AE071
:10ACF00037ED43E25CE30F94F6020F941308262F1E
:10AD000002E042E367E382E99AE052D98091C60A01
:10AD1000813308F060C08091C80A893208F45BC0B2
:10AD20000E947BC02B013C018CE3882E912CA12C2E
:10AD3000B12CC301B201A50194010F946C06CA01A4
:10AD4000B901A50194010F946C06CA01E62ED72E15
:10AD500059018E010F5F1F4FF1E84F16F1E55F06B5
:10AD6000F1E06F06710408F485C1B90128E130E013
:10AD700040E050E00F946C0629013A01DF92EF9217
:10AD8000C50168E170E00F948E099F938F935F92E5
:10AD90004F9284E199E09F938F931F930F930F94A9
:10ADA0002A020FB6F894DEBF0FBECDBF9AE0491657
:10ADB00051046104710408F08CC197E0892F880F59
:10ADC000980F9195955A9093C90A80E38093CA0A87
:10ADD000C8010E9483F0E0918C0AF0918D0A848171
:10ADE0008111CEC0609121057091220580912305CB
:10ADF000909124050F940E08CB010E9432C5BC012E
:10AE000087EF94E00F94040A609125057091260560
:10AE100080912705909128050F940E08CB010E9480
:10AE200032C5BC0182EF94E00F94040A2CEA35ECA1
:10AE300047E257E36091290570912A0580912B051F
:10AE400090912C050F94CA0620E030E048EC52E4C3
:10AE50000F94F6020F940E084B015C0197FD19C088
:10AE600090E1891697E29906A104B104E4F0C501C6
:10AE7000B40120E137E240E050E00F948E06CA01B1
:10AE8000B9012AE030E040E050E00F948E06605DAA
:10AE90000BC0B094A09490948094811C911CA11C30
:10AEA000B11C6DE201C060E26093010EE8EE8E1607
:10AEB000E3E09E06A104B10494F0C501B40128EEBC
:10AEC00033E040E050E00F948E06CA01B9012AE059
:10AED00030E040E050E00F948E06605D01C060E21B
:10AEE0006093020EC501B40124E630E040E050E07A
:10AEF0000F948E069AE0492E512C612C712CCA01B8
:10AF0000B901A30192010F948E06605D6093030E58
:10AF1000C501B401A30192010F948E064B015C019F
:10AF2000672B682B692B79F08EE28093040ECA019F
:10AF3000B901A30192010F948E06605D6093050E26
:10AF400080E3880D15C0CA01B901A30192010F94D5
:10AF50008E06662339F08EE28093040E605D609366
:10AF6000050E05C080E28093050E8093040E80E2FA
:10AF70008093060E61E07EE08BEE94E00F94040A6D
:10AF80008091C60A8632A0F48091C80A8E3180F082
:10AF900008E020E84EE160E082E99AE009D880917B
:10AFA000C60A863228F48091C80A8F3108F093C00F
:10AFB0008091C60A823328F48091C80A8C3208F046
:10AFC000FAC08091C60A8F3308F014C18091C80A74
:10AFD000883308F40FC11092C90A8EE38093CA0A1D
:10AFE0000E9423BF07C12CE00ECD22E10CCD02E070
:10AFF00022E041E1612F82E99AE00E94D84F41CDE1
:10B000004CE0B2CD42E1B0CD02E022E042E168E5A1
:10B0100082E99AE00E94D84FEECD07E028E04AE2AC
:10B020006AE282E99AE00E94D84F05E022E04CE211
:10B0300062E382E99AE00E94D84F6AE08AE20E94C5
:10B04000BABD6091940A7091950A82E38093AE0A2A
:10B050008BE28093AF0A2EEA3AE042E382E99AE07B
:10B060000E94164EFBCD6AE486E30E94BABDFFCD76
:10B0700020E033CEE4E6AE16B104C0F4DF92EF92E6
:10B08000C50168E170E00F948E099F938F938AE069
:10B0900099E09F938F931F930F930F942A020FB6FB
:10B0A000F894DEBF0FBECDBF95E088CEDF92EF9261
:10B0B0003F932F9382E099E09F938F931F930F9379
:10B0C0000F942A020FB6F894DEBF0FBECDBF96E0F4
:10B0D00075CE98E073CE1092B20A83E08093C90ACD
:10B0E00085E28093CA0AFF2029F082ED93E10E9455
:10B0F00076F00DC08091E804811102C08FE305C095
:10B10000809147058111F1CF80E20E9466BE8BE0FD
:10B110008093C90A15E21093CA0A87EF94E00E944F
:10B1200083F08BE28093C90A1093CA0AFF2029F0AA
:10B1300080ED93E10E9476F00DC08091E9048111C9
:10B1400002C08FE305C0809148058111F1CF80E2F4
:10B150000E9466BE83E38093C90A15E21093CA0A6F
:10B1600082EF94E00E9483F083E58093C90A1093F4
:10B17000CA0AFF2029F08EEC93E10E9476F00DC000
:10B180008091EA04811102C08FE305C080914905D6
:10B190008111F1CF80E20E9466BE8BE58093C90ADF
:10B1A00085E28093CA0A8BEE94E00E9483F081E0EE
:10B1B0008093B20AFDCE84E00E9431F083E0809358
:10B1C000C90A12E31093CA0A86E00E9462F00E9444
:10B1D000EBC68CE08093C90A1093CA0A80912402BE
:10B1E000909125020E9499C50E9483F085E20E94F9
:10B1F00066BEE7CE2A960FB6F894DEBF0FBECDBF6F
:10B20000DF91CF911F910F91FF90EF90DF90CF9042
:10B21000BF90AF909F908F907F906F905F904F9076
:10B22000089540E050E0BA0189EF93E5BFCAE0918C
:10B23000DB04EE2381F0E150E093DB0486E0E89F3D
:10B24000F0011124E954FB4F4281538164817581DF
:10B2500080819181ABCAE5CFAF92BF92CF92DF924E
:10B26000EF92FF920F931F93CF93DF935C017B01CB
:10B2700020E030E0F501E20FF31FE491EE2319F036
:10B280002F5F3F4FF7CFF701CF018E199F094191F3
:10B290004111FACF04E110E0081B1109332702170E
:10B2A00013071CF0DD24D39402C082E0D82E8091D5
:10B2B000930A90E06D2D70E06F5F7F4F0F94A209AD
:10B2C000C62EC6E0C60F8091C60AC81750F08091FE
:10B2D000C80A90E02C2F30E02B50310982179307D9
:10B2E0009CF5D0E0E114F104C1F18AE30E9466BE4E
:10B2F00082E0D8120FC0CC0D8091C60AC81768F141
:10B300002091C80A30E08C2F90E00B97281739075E
:10B310001CF423C0DD2309F1802F880F080F000FD4
:10B320000093C90AC093CA0A80E20E9466BEC701A0
:10B33000DF91CF911F910F91FF90EF90DF90CF9011
:10B34000BF90AF900C9483F01092C90AC093CA0AC0
:10B35000C5010E9476F0D1E0C5CFDF91CF911F915A
:10B360000F91FF90EF90DF90CF90BF90AF90089536
:10B370000F934CE0849F402D112421E0240F209353
:10B380000F058CE0840F80931005E091C60AF0E071
:10B3900090E002968E179F070CF1822F90E020918B
:10B3A000C80A30E082179307CCF4662371F081E07D
:10B3B0008093B20A4D5F0BE020E860E082E99AE0FA
:10B3C0000E94D84F1092B20A03C081E08093B20A63
:10B3D000809110051092C90A8093CA0A0F910895AE
:10B3E000CF92DF92EF92FF920F93CF93DF93982F3C
:10B3F000862F6A017901692FBBDF9091C60A80917F
:10B400001005891708F453C09091C80A80910F0560
:10B41000981708F44CC0002359F060E070E0F70181
:10B42000E60FF71FE491EE2351F06F5F7F4FF7CFE8
:10B43000D701BD016E197F098D918111FACFC62FF9
:10B44000D4E1D61BF6018491882339F00E944BF099
:10B45000D81BFFEFCF1ADF0AF5CF8AE30E9466BE42
:10B46000DD2329F080E20E9466BED150F9CF8091A1
:10B4700010056AEFC69F602D112460586093C90AB9
:10B480008093CA0AC701002349F0DF91CF910F9141
:10B49000FF90EF90DF90CF900C9476F0DF91CF91FA
:10B4A0000F91FF90EF90DF90CF900C9483F0DF919D
:10B4B000CF910F91FF90EF90DF90CF9008950F9371
:10B4C000CF93DF93CDB7DEB7ED85FE8560817181C7
:10B4D000828193810F940E08CB010E9499C500E0F0
:10B4E0009C0149855A8568858F817ADFDF91CF91EC
:10B4F0000F9108959CE0899F802D112421E0280F51
:10B5000020930F05845F809310056091C60A70E058
:10B51000482F50E04E5F5F4F461757070CF445C069
:10B5200030E04091C80A50E024173507F4F59EE357
:10B530009093C90A8093CA0A85E40E9462F08091C0
:10B5400046058F5C0E9462F080E20E9462F0E0910A
:10B55000460584E0E89FF0011124E452FB4F60812E
:10B560007181828193810F940E08CB010E9499C54D
:10B570000E9483F08FE20E9462F00E9470CAE09104
:10B580004605811107C0AE2FB0E0A657B54F8C918C
:10B5900081110BC0F0E0EE0FFF1FE55FF54F8081DA
:10B5A00091810E9499C50C9483F008954F925F9207
:10B5B0006F927F928F929F92AF92BF92FF920F9362
:10B5C0001F93CF93DF93182F8AEE9CE0909355073B
:10B5D000809354071092060D82E090E0A0E0B0E066
:10B5E0008093EF0C9093F00CA093F10CB093F20CBD
:10B5F0001092530710924F07109250071092510764
:10B60000109252078FEF9FEFDC0180934B079093CE
:10B610004C07A0934D07B0934E07112379F11530D5
:10B6200008F0F9C040E060E070E0CB010E94D6B1C4
:10B63000882309F4F0C020E1129FC0011124855C29
:10B640009A4FFC01E254FE4F20812F7709F0E3C0AE
:10B650003C96408151816281738144365105610578
:10B66000710508F4D8C0349780809180A280B3809F
:10B6700081149104A104B10421F4CDC0812C912C3A
:10B68000540140E0C501B4010E94D6B1F82E8823D0
:10B6900009F4C1C0809156059091570581159240DB
:10B6A00009F0B9C0A0915B05AA2309F4B4C0609168
:10B6B000590570915A056115710509F4ACC02091C6
:10B6C0005805222309F4A7C0A093010D2093F30C81
:10B6D00080E030E0E1E0F0E0C82FAF01082E02C0CA
:10B6E000440F551F0A94E2F72417350741F0982FAD
:10B6F0008F5F983089F789E08093FC0C8CC0809331
:10B70000FC0C20916105309162052115310519F07D
:10B7100040E050E008C020916F05309170054091E5
:10B720007105509172052093F40C3093F50C409301
:10B73000F60C5093F70C24013501460E571E611C80
:10B74000711C4092020D5092030D6092040D709294
:10B75000050DE0915C05F0915D05F093080DE09317
:10B76000070DB0E00F94AA06460E571E681E791EFC
:10B770004092090D50920A0D60920B0D70920C0DC3
:10B7800085E0EE0FFF1F8A95E1F7E150FE4FEF2FA6
:10B79000FF27E6954E0E5F1E611C711C4092FD0C4A
:10B7A0005092FE0C6092FF0C7092000D20915E058D
:10B7B00030915F052115310521F0890120E030E04D
:10B7C00008C000916B0510916C0520916D053091BA
:10B7D0006E05B501A4014419550966097709400FA2
:10B7E000511F621F731F04C0769567955795479543
:10B7F000CA95D2F74093F80C5093F90C6093FA0C69
:10B800007093FB0C453F2FE052076105710528F44A
:10B810008CE08093060DF12C1AC0453F5F4F610507
:10B82000710510F480E111C0809177059091780541
:10B83000A0917905B0917A058093090D90930A0D36
:10B84000A0930B0DB0930C0D80E28093060D8F2D0D
:10B85000DF91CF911F910F91FF90BF90AF909F907C
:10B860008F907F906F905F904F900895EF92FF922E
:10B870000F931F93CF93DF93CDB7DEB76F970FB6BC
:10B88000F894DEBF0FBECDBF7B0102E91BE024E9C7
:10B890003BE0F8013183208322E02093CB0D90938D
:10B8A000CD0D8093CC0D40E050E0BA0188E99BE0DB
:10B8B0000E949079F801808191812BE1FC013496FE
:10B8C000DE01159601900D922A95E1F7FC01828127
:10B8D00093819C838B8384E993E09A838983A70176
:10B8E000BE016F5F7F4F89EC93E00E94AFC0CE0135
:10B8F00001960E94E5E96F960FB6F894DEBF0FBE81
:10B90000CDBFDF91CF911F910F91FF90EF900895E0
:10B910006F927F928F929F92AF92BF92DF92EF923F
:10B92000FF920F931F93CF93DF93CDB7DEB7AD9701
:10B930000FB6F894DEBF0FBECDBF2091200B22239F
:10B9400009F4F0C1D62E7C018091140D882309F4EE
:10B950009FC0442309F4BBC180912C0D882329F199
:10B96000E6ECF7E184918F010F5F1F4F882321F0F0
:10B970000E940669F801F6CFE3E8F7E184918F01B0
:10B980000F5F1F4F882321F00E940669F801F6CF50
:10B9900061E070E080E090E00E94C5698AE00E946A
:10B9A00006698AE797E10E94F9E98FE28093310DF9
:10B9B000B12C21E002E31DE09FE1A92E8091E90C6A
:10B9C000B816B8F4AB9CC0011124B8018954944F47
:10B9D0002DA70E94797AC8012DA58C010196F80146
:10B9E0003081332321F02D3811F02F5FF6CFB3943F
:10B9F000E5CF27FD08C0B80181E19DE00E94797A7A
:10BA0000E4EFF2E203C0F8011082FACF84918F01D3
:10BA10000F5F1F4F882321F00E940669F801F6CFBF
:10BA2000B70181E697E10E94EAC260912C0DFDE822
:10BA30006F9FB00111246F5C724F86E597E10E9401
:10BA4000EAC24091C20D5091C30D6091C40D709136
:10BA5000C50D80E597E10E94C9688AE00E940669E9
:10BA600080912C0D94E0899FF0011124E35DF24F49
:10BA70004091C20D5091C30D6091C40D7091C50DE0
:10BA800040835183628373838F5F80932C0D0DC03D
:10BA900010922C0D82E0B82E1CC1B70183E497E10F
:10BAA0000E94EAC28AE00E9406690E9403BF1D82CA
:10BAB00018861C821B8284E993E09A83898383E73A
:10BAC0009BE09093930B8093920BF70180818F32D0
:10BAD00009F067C087010F5F1F4FCE0101963C013F
:10BAE0000115110509F463C06FE270E0C8010F94FD
:10BAF000F9095C01009709F45BC00817190708F001
:10BB000057C04C01801A910AA401B801CE01809659
:10BB10000F94190AE0E2F0E0EC0FFD1FE80DF91DAB
:10BB20001082FE01B0964F018F01F80181918F01C3
:10BB3000882319F00E940669F8CF8AE00E940669FE
:10BB40006091920B7091930B6115710511F06C5F10
:10BB50007F4F21E0AE01405E5F4FCE0105960E940F
:10BB6000B480811116C0EFE2F7E184918F010F5F7D
:10BB70001F4F882321F00E940669F801F6CFF401D7
:10BB800081914F01882319F00E940669F8CF8EE257
:10BB900087C07092930B6092920B85010F5F1F4FCD
:10BBA0009FCF84E99BE09093930B8093920B870146
:10BBB0009091920B8091930B692F782FDD2009F4DF
:10BBC00059C06115710511F06C5F7F4F21E0A8012C
:10BBD00081E19DE00E94B480882309F447C08091F0
:10BBE000220D9091230DA091240DB091250D8093ED
:10BBF000BE0D9093BF0DA093C00DB093C10DB801C1
:10BC000081E297E10E94EAC24091BE0D5091BF0DC2
:10BC10006091C00D7091C10D89E197E10E94C968E2
:10BC20008AE00E9406691092C20D1092C30D109214
:10BC3000C40D1092C50DEAE0F7E184917F019FEFFA
:10BC4000E91AF90A882321F00E940669F701F5CF65
:10BC5000B80180E090E00ADE80912F0B882319F074
:10BC60008FE29BE001C0C80160E02AC0B80186EF06
:10BC700096E110C06115710511F06C5F7F4F26E5EC
:10BC8000A80181E19DE00E94B48081110CC0B8013F
:10BC900082EE96E10E94EAC28EE20E9406698AE084
:10BCA0000E9406690FC081E080931D0BB70180EDF3
:10BCB00096E10E94EAC28AE00E94066960E0C8013B
:10BCC0000E9486C7CE0101960E94E5E92BC0BB24E5
:10BCD000B394E4EFF2E284918F010F5F1F4F88234A
:10BCE00021F00E940669F801F6CFEBE4F7E18491B8
:10BCF0008F010F5F1F4F882321F00E940669F80112
:10BD0000F6CFE1E0BE1619F007E413E002C00DE43F
:10BD100013E0F80181918F01882309F4BECE0E94BF
:10BD20000669F7CFAD960FB6F894DEBF0FBECDBF54
:10BD3000DF91CF911F910F91FF90EF90DF90BF9017
:10BD4000AF909F908F907F906F900895CF92DF92E9
:10BD5000EF92FF920F931F93CF93DF93CDB7DEB790
:10BD6000EDB6FEB6DC010D900020E9F79D01281B21
:10BD7000390B2C5F3F4F4DB75EB7421B530B0FB6CD
:10BD8000F8945EBF0FBE4DBF0DB71EB70F5F1F4FBC
:10BD90009F938F9389EC96E19F938F931F930F93BB
:10BDA0000F942A02680154E0C50ED11C0F900F9029
:10BDB0000F900F900F900F90F6018081882339F03B
:10BDC00090E00F94BD09F60181936F01F5CF60E01B
:10BDD000C8010E943549882319F0C8010E94A7E9CB
:10BDE00085EC96E190935707809356070E9451493E
:10BDF0000FB6F894FEBE0FBEEDBEDF91CF911F913E
:10BE00000F91FF90EF90DF90CF900895AF92BF9287
:10BE1000CF92DF92EF92FF920F931F93CF93DF9316
:10BE2000CDB7DEB7AA970FB6F894DEBF0FBECDBF71
:10BE30008091720B8F938091710B8F938CEB96E1B5
:10BE40009F938F937E0181E2E80EF11CFF92EF92A7
:10BE50000F942A020F900F900F900F900F900F9059
:10BE600010E0F70101900020E9F73197EE19FF0982
:10BE70001E1774F46701C10ED11C17FDDA94F60188
:10BE8000808190E00F94BD09F60180831F5FE9CFA8
:10BE900040E050E0BA0187E79BE00E94907900E023
:10BEA000CE0101966C0180917A0B823028F4011149
:10BEB00014C08FEF9FEF16C080917F0B9091800B85
:10BEC000A091810BB091820B8F719927AA27BB2774
:10BED000892B8A2B8B2B59F71AC08091710B90916B
:10BEE000720B01969093720B8093710BAA960FB60A
:10BEF000F894DEBF0FBECDBFDF91CF911F910F91A0
:10BF0000FF90EF90DF90CF90BF90AF90089540E00A
:10BF100050E0B60187E79BE00E9486B318163CF616
:10BF2000F60101900020E9F731971E2F1C191150DE
:10BF300068F05601A10EB11C17FDBA94F50180817D
:10BF400090E00F94BD09F5018083F1CF8A858E378B
:10BF500009F4A9CF45E050E0B701C6010F940B0AE0
:10BF6000892B09F0A0CFC701F1DE01E09CCFCF9271
:10BF7000DF92EF92FF921F93CF93DF931092200BEB
:10BF800080917A0B882321F087E79BE00E94C97A91
:10BF90001092EE0C1092EB0C85E38093EA0C0E9459
:10BFA0000A53EB01A8958091EA0C0E940BBD8AEE22
:10BFB0009CE00E94D17A2398229A219A209A289A6A
:10BFC00085E08093EC0C82E58CBD1DBC1AE08FEF00
:10BFD0000E94D67A1150D9F720E030E0A90160E044
:10BFE0008AEE9CE00E94DB7A182F8093ED0C813062
:10BFF00049F00E940A536C1B7D0B613D774060F352
:10C0000081E054C02AEA31E040E050E068E08AEE86
:10C010009CE00E94DB7A82FF03C01093EE0C0EC0FE
:10C0200014E00E94FF688093ED0C1150D1F78A3A1A
:10C0300011F082E03BC082E08093EE0C8091EE0C28
:10C04000823021F0C12CD12C760105C0C12CD12C1D
:10C05000E12C80E4F82E20E030E0A90167E38AEECD
:10C060009CE00E94DB7AA701960169E28AEE9CE0DF
:10C070000E94DB7A8093ED0C882349F00E940A53DA
:10C080006C1B7D0B613D774030F38AE00FC08091DF
:10C09000EE0C823011F520E030E0A9016AE38AEE6F
:10C0A0009CE00E94DB7A882351F088E08093EB0CBF
:10C0B0008AEE9CE00E94D17AE4EFF2E219C00E947D
:10C0C000FF68807C803C19F483E08093EE0C0E9432
:10C0D000FF680E94FF680E94FF688AEE9CE00E9451
:10C0E000D17A1092EC0C81E061DA811131C015C077
:10C0F0008491EF012196882321F00E940669FE01B8
:10C10000F7CFEEEAF6E18491EF012196882309F456
:10C1100056C00E940669FE01F6CF80E047DA811121
:10C1200017C0E6ECF7E18491EF012196882321F016
:10C130000E940669FE01F7CFEAE9F6E18491EF017A
:10C140002196882309F43BC00E940669FE01F6CFC0
:10C150006FEE7CE087E79BE00E94267A811116C093
:10C16000E6ECF7E18491EF012196882321F00E940B
:10C170000669FE01F7CFE9E8F6E18491EF01219627
:10C180008823E9F00E940669FE01F7CF81E08093E1
:10C19000200BE4EFF2E28491EF012196882321F055
:10C1A0000E940669FE01F7CFEDE7F6E18491EF0109
:10C1B0002196882321F00E940669FE01F7CF8BE1CA
:10C1C000E7E7FBE0A8E9BBE001900D928A95E1F773
:10C1D0008091750B9091760B9093970B8093960BB3
:10C1E00083E79BE09093930B8093920BDF91CF9129
:10C1F0001F91FF90EF90DF90CF9008950F931F93C2
:10C20000CF93DF938C01EB019091FE0A2091FF0AFE
:10C21000921307C082EF9AE00E9416530E9480D3C7
:10C22000F3CFF801A081B181488159818091FD0A45
:10C2300034E0839FF0011124EA50F54FB387A287C1
:10C24000558744879F5F9093FE0A8F5F821719F08E
:10C250008093FD0A02C01092FD0ADF91CF911F91D9
:10C260000F910895CF93DF93CDB7DEB780914A0544
:10C27000811110C09E01275F3F4F4F81588562E4B6
:10C2800070E083E392E00F9459020E944AC783E072
:10C2900080931202DF91CF9108958091100B81302D
:10C2A000A1F1823059F40E947BC06093110B70930E
:10C2B000120B8093130B9093140B18C01092150B54
:10C2C0001092160B1092170B1092180B1092190B5C
:10C2D00010921A0B10921B0B10921C0B1092110B48
:10C2E0001092120B1092130B1092140B81E080939A
:10C2F000100B0E940A536093150B7093160B8093DA
:10C30000170B9093180B81E0089580E00895EF9249
:10C31000FF921F93CF93DF93D091470581E0D827F9
:10C32000109148051827C0914905C827D11102C0AE
:10C33000112319F0E4EFF2E203C0C111FBCF77C083
:10C3400084917F019FEFE91AF90A882319F05ED7DB
:10C35000F701F6CFE7E7F6E184917F019FEFE91A55
:10C36000F90A882319F052D7F701F6CFDD2361F0DF
:10C37000E5E7F6E184917F019FEFE91AF90A882346
:10C3800019F044D7F701F6CF112361F0E3E7F6E1A6
:10C3900084917F019FEFE91AF90A882319F036D7B3
:10C3A000F701F6CFC11103C0E9E6F6E10CC0E1E701
:10C3B000F6E184917F019FEFE91AF90A8823A1F33E
:10C3C00025D7F701F6CF84917F019FEFE91AF90A8B
:10C3D000882319F01BD7F701F6CFC11103C049EC30
:10C3E00053E002C043E553E0111103C029EC33E0F0
:10C3F00002C025E533E0D11103C089EC93E002C00F
:10C4000087E593E05F934F933F932F939F938F9391
:10C4100087E596E19F938F931F9224DF8DB79EB798
:10C4200009960FB6F8949EBF0FBE8DBFC1E08C2F4A
:10C43000DF91CF911F91FF90EF900895CF92DF92FF
:10C44000EF92FF92E0914605E0934505C0902D05DF
:10C45000D0902E05E0902F05F0903005ED5F84E040
:10C46000E89FF0011124EF5CFA4F20813181428175
:10C470005381C701B6010F94F6020F94FB08609335
:10C48000EC0A7093ED0A8093EE0A9093EF0AC701CD
:10C49000B6010F940E082FB7F89460931D057093A2
:10C4A0001E0580931F05909320052FBF1092DC0A74
:10C4B0001092DD0A1092DE0A1092DF0AFF90EF90D0
:10C4C000DF90CF9008958091100B813079F482E055
:10C4D0008093100B0E940A536093190B70931A0BF0
:10C4E00080931B0B90931C0B81E0089580E00895CE
:10C4F000E82FF0E0EF5EF94EE4918E2F90E0FC0122
:10C500003797EC30F10508F58827EA56FF4F8F4F33
:10C510000D94B5098091B100887F84608093B1004B
:10C52000089580919100887F8460809391000895A0
:10C530008091A100887F84608093A10008958091FC
:10C540002101887F8460809321010895FC01DB0133
:10C550008C9120813181382798E0A901440F551F23
:10C5600037FD06C09A019150C1F7318320830895A9
:10C570009A01B1E22B27B0E13B27F5CFBC0180E067
:10C5800090E04AE09CD68DE041D68AE03FC6EF922B
:10C59000FF920F931F93CF93DF931F92CDB7DEB718
:10C5A0008B01622F49830E94B8599091C60A8091ED
:10C5B00010054981891708F43FC09091C80A8091FD
:10C5C0000F05981708F438C0442399F120E030E0B3
:10C5D000F801E20FF31FE491EE2319F02F5F3F4FB4
:10C5E000F7CF86E190E0821B930B97FD019695951E
:10C5F000879536E1F32E49EEE42EE80E8E2D8F0D51
:10C6000087FD0EC080E20E9466BEFA94F7CFF80163
:10C610008491882339F00E944BF0F81A0F5F1F4F66
:10C620001F14ACF31F1444F480E20E9466BEFA9417
:10C63000F9CF86E1F82EF4CF0F90DF91CF911F91C3
:10C640000F91FF90EF900895CF92DF92EF92FF92BB
:10C650000F931F93CF93DF937C018B016A01E90154
:10C660000E94B65383E080931202F0920B05E09291
:10C670000A0510930905009308051092040510920D
:10C6800005051092060510920705A601DD0C660B44
:10C69000770B40930005509301056093020570935A
:10C6A0000305F80180819181092E000CAA0BBB0BB8
:10C6B0008093FC049093FD04A093FE04B093FF04C8
:10C6C00083E292E79093110280931002D0930E05BB
:10C6D000C0930D0510920C05DF91CF911F910F9122
:10C6E000FF90EF90DF90CF900895CF93DF931F924C
:10C6F000CDB7DEB7789484B5826084BD84B581609F
:10C7000084BD85B5826085BD85B5816085BD80911C
:10C710006E00816080936E00109281008091810094
:10C72000826080938100809181008160809381008C
:10C73000809180008160809380008091B10084604E
:10C740008093B1008091B00081608093B0008091AF
:10C75000910082608093910080919100816080932C
:10C760009100809190008160809390008091A10061
:10C7700082608093A1008091A10081608093A100DC
:10C780008091A00081608093A0008091210182604F
:10C79000809321018091210181608093210180910A
:10C7A000200181608093200180917A0084608093D1
:10C7B0007A0080917A00826080937A0080917A007A
:10C7C000816080937A0080917A00806880937A00FB
:10C7D0001092C1006F98779A82E08093C000109207
:10C7E000C50087E08093C4008091C1008061809380
:10C7F000C1008091C10088608093C1008091C10018
:10C8000080688093C1008091C1008F7D8093C100BA
:10C8100010925807E8E4F9E184918F010F5F1F4FF0
:10C82000882319F0F3D4F801F7CFE4EFF2E2849112
:10C830008F010F5F1F4F882319F0E8D4F801F7CF5D
:10C8400014B710FF0CC0EFE3F9E184917F019FEF73
:10C85000E91AF90A882319F0D9D4F701F6CF11FFA4
:10C860000CC0EEE2F9E184917F019FEFE91AF90A29
:10C87000882319F0CBD4F701F6CF12FF0CC0ECE1FE
:10C88000F9E184917F019FEFE91AF90A882319F0F1
:10C89000BDD4F701F6CF13FF0CC0EBE0F9E18491B2
:10C8A0007F019FEFE91AF90A882319F0AFD4F70145
:10C8B000F6CF15FF0BC0EAEFF8E184918F010F5F0F
:10C8C0001F4F882319F0A2D4F801F7CF14BEE3EF6D
:10C8D000F8E184918F010F5F1F4F882319F096D4E0
:10C8E000F801F7CF80E292D4ECEEF8E184918F0169
:10C8F0000F5F1F4F882319F089D4F801F7CF8AE022
:10C9000085D4E4EFF2E284918F010F5F1F4F8823FB
:10C9100019F07CD4F801F7CFECEDF8E184918F01A8
:10C920000F5F1F4F882319F071D4F801F7CFE8EC9F
:10C93000F8E184918F010F5F1F4F882319F066D4AF
:10C94000F801F7CFEFE8F8E184918F010F5F1F4FF7
:10C95000882319F05BD4F801F7CFE4EFF2E2849179
:10C960008F010F5F1F4F882319F050D4F801F7CFC4
:10C97000E8E7F8E184918F010F5F1F4F882319F0DA
:10C9800045D4F801F7CFE4EFF2E284918F010F5F15
:10C990001F4F882319F03AD4F801F7CF80915B1527
:10C9A00090915C15BE016F5F7F4F009719F0681B77
:10C9B000790B02C06156754189E698E10E94D1C2A7
:10C9C00060EF74E082E598E10E94D1C28AE01ED453
:10C9D00081E080937207809373078093740780933C
:10C9E00075070E9466D58CE0E6E6F7E0A1E2B5E0C7
:10C9F00001900D928A95E1F70E94344C80911902C2
:10CA000090911A0290931C0280931B028091010165
:10CA10008064809301018091010180618093010114
:10CA2000809101018860809301016D9A80910101DC
:10CA300088608093010186E05BDD80910101806266
:10CA40008093010188E054DD6C9A82E051DD87ED2E
:10CA500080937A0010927E0010927D0080917E007B
:10CA6000816080937E0080917E00826080937E0052
:10CA700080917E00846080937E0080E888BD8091F4
:10CA80006E00846080936E006AEF70E080E090E05A
:10CA90000E94D05285E090E09093600780935F07FA
:10CAA00060E080911502909116020E945CCE20E019
:10CAB00030E040EA50E40F94910287FF0AC0809171
:10CAC00015029091160240979093160280931502DA
:10CAD000E7CF81E391E090931A028093190260E01E
:10CAE00080915B0790915C070E945CCE20E030E86B
:10CAF00048E953E40F94F008181654F480915B074A
:10CB000090915C07409690935C0780935B07E7CF1A
:10CB100085E090E0909362078093610761E08091E7
:10CB20001702909118020E945CCE20E030E040EAAB
:10CB300050E40F94910287FF0AC0809117029091F0
:10CB4000180240979093180280931702E7CF81E371
:10CB500091E090931C0280931B0261E080915D073D
:10CB600090915E070E945CCE20E030E848E953E4F3
:10CB70000F94F008181654F480915D0790915E07A9
:10CB8000409690935E0780935D07E7CF80911302F4
:10CB9000909114020E943ED020E030E040EA50E440
:10CBA0000F94910287FF0AC08091130290911402A2
:10CBB00040979093140280931302E8CF8091590715
:10CBC00090915A070E943ED020E030E046E153E4C5
:10CBD0000F94F008181654F48091590790915A0751
:10CBE000409690935A0780935907E8CF98E288E1DE
:10CBF0000FB6F894A895809360000FBE90936000E4
:10CC00001FB7F89480916307811124C0EDEAF3E225
:10CC10008491E3EFF3E29491E82FF0E0EE0FFF1F31
:10CC2000E25AFC4DA591B491EC91E92321F461E025
:10CC300085E30E94D95185E30E940BBD8CB58061CC
:10CC40008CBD8CB580648CBD84E30E940BBD83E3F6
:10CC50000E940BBD809163078F5F809363071FBFA6
:10CC6000579A13E7E12E13E0F12E10E0F7016191DE
:10CC70007F0170E0812F0E946CF91F5F1530B1F7C2
:10CC8000999A989A809107018068809307019A9AEF
:10CC90008091070180648093070180910701806281
:10CCA000809307018091070188608093070180913C
:10CCB0000701806180930701809107018260809362
:10CCC000070180910701846080930701B8E7EB2E8C
:10CCD000B3E0FB2E10E0F70161917F01812F0E94EC
:10CCE00046F91F5F1530B9F780910A018260809381
:10CCF0000A0180910A01816080930A0180910A01F2
:10CD0000846080930A0180910A01806480930A0103
:10CD100080910A01806880930A010F9A179A0E9AEF
:10CD2000169A0D9A159A0C9A149A0B9A139A269899
:10CD30002E9A25982D9A24982C9A389A4098179ACA
:10CD400010924705399A4198169A109248053A9AD6
:10CD50004298159A109249053B9A4398149A3C9A26
:10CD60004498139A809180008C7F809380008091FA
:10CD70008100877E886080938100809180008F731E
:10CD80008093800080918100887F82608093810001
:10CD900080E090E490938900809388001092850051
:10CDA0001092840080916F00826080936F0081E018
:10CDB0008093650778940E9408DF6C9A0E94A8CA45
:10CDC00064EC79E080E090E00E94CFC580911D0284
:10CDD000811118C064EC79E080E090E00E94CFC53A
:10CDE00081E0809365078093640770E6572EEDE03D
:10CDF0004E2EF6E6CF2EF9E1DF2EA0E0AA2EA0E01F
:10CE0000BA2E8EC010921D022091920A30E0790154
:10CE1000F8E3EF1AF108F7FE04C0790187E3E81A96
:10CE2000F108F594E7942E51310936952795F22EA5
:10CE30000E9432BF0DEC17E123E147E06CE08E2D3C
:10CE40000E9464BD84E00E9431F00091920A10E0DB
:10CE500002571109169507956091930A625149E5A9
:10CE600053E08F2D0E94E4BD6091930A66504FE518
:10CE700053E0802F0E94E4BD0E942ABD8111DACFC9
:10CE8000A9CF8091970780FD2FC18091970784FDDE
:10CE90002BC190E2F92E8091970781FD42C18091CC
:10CEA000970785FD3EC100E28091970782FD55C13D
:10CEB0008091970786FD51C110E28AE0A7D11F92A9
:10CEC0006F921F921F931F920F931F92FF92DF92F8
:10CED000CF921F92C7D9109297070FB6F894DEBF72
:10CEE0000FBECDBF80917607882391F010921F0B63
:10CEF00081E19DE00E944D7981E19DE00E94C97A27
:10CF000010921E0B10921D0B0E949C9A0E94F7CF4C
:10CF100080E00E945EEAA114B10431F00E9400009A
:10CF20002AE0722E30E2632E80911909843010F4C9
:10CF30000E94B0498091CA0D8823E9F00E940A53EB
:10CF40000091C60D1091C70D2091C80D3091C90DEB
:10CF5000DC01CB01801B910BA20BB30BB7FD0BC007
:10CF60001092CA0D8091200B8111BBC000D8809116
:10CF7000200B8111B6C080911909882309F495C04E
:10CF800080911D0B882309F47DC000911809509EE3
:10CF9000800111240856184F69EA79E1C8010F94FD
:10CFA0001002892BF1F081E19DE00E944D7981E131
:10CFB0009DE00E94C97A10921E0B10921D0BE6E9AB
:10CFC000F9E184918F010F5F1F4F882339F01ED143
:10CFD000F801F7CF80911E0B811154C00E9442EDE1
:10CFE00053C0F80101900020E9F731977F01E01A62
:10CFF000F10A1092110D6EE470E0C8010F94F90966
:10D000004C01009729F4F7013197E00FF11F0EC092
:10D0100060E270E00F94F9098C010F5F1F4F6AE224
:10D0200070E0C4010F94F909FC01319741827282CA
:10D030001382F80101900020E9F73197AF01401BFE
:10D04000510BB80181E19DE00E94B07B8091110DF0
:10D05000882309F4BFCFE6ECF7E184918F010F5FDD
:10D060001F4F882319F0D2D0F801F7CFEFE4F9E190
:10D0700084918F010F5F1F4F882309F4ABCFC6D077
:10D08000F801F6CF0E94472980911909882369F099
:10D09000815080931909809118098F5F843018F4AA
:10D0A0008093180902C0109218098091970788236D
:10D0B00009F42ECFE4EFF2E284918F010F5F1F4F4E
:10D0C000882319F0A3D0F801F7CFE7E8F9E18491BC
:10D0D0008F010F5F1F4F882309F4D3CE97D0F8013B
:10D0E000F6CF0E94065F47CF60918B0770918C0747
:10D0F00080918D0790918E070F949702209177076A
:10D10000309178074091790750917A070F94F60291
:10D11000AB01BC0183E899E10E948DC288E5F82E3D
:10D12000BACE60918F07709190078091910790918E
:10D1300092070F94970220917B0730917C074091D2
:10D140007D0750917E070F94F602AB01BC018FE77B
:10D1500099E10E948DC209E5A7CE60919307709175
:10D16000940780919507909196070F9497022091CC
:10D170007F073091800740918107509182070F947B
:10D18000F602AB01BC018BE799E10E948DC21AE562
:10D1900094CECF92DF92EF92FF92CF93DF936A010A
:10D1A0007B01FC018491EF012196882319F02ED098
:10D1B000FE01F8CF4AE0C701B601DF91CF91FF90A1
:10D1C000EF90DF90CF907BC0CF92DF92EF92FF92F3
:10D1D000CF93DF936A017B01FC018491EF012196DB
:10D1E000882319F013D0FE01F8CF42E0C701B60141
:10D1F000DF91CF91FF90EF90DF90CF90E0C08FEF65
:10D200008EBD0DB407FEFDCF8EB5089591E09093CD
:10D2100058073FB7F8942091DF099091E0093FBF8C
:10D22000291304C09091C00095FD3EC09091DF0984
:10D230009F5F9F712091E009921325C00FB607FCF4
:10D24000F9CF2091C00025FFF5CF2091E009E22F12
:10D25000F0E0E154F64F30812F5F2F712093E00909
:10D260003093C6002091C00020642093C00030910C
:10D27000DF092091E0093213DDCF2091C1002F7D1D
:10D280002093C100D7CFE091DF09F0E0E154F64FE1
:10D2900080832FB7F8949093DF098091C10080625A
:10D2A0008093C1002FBF08959FB7F8948093C60064
:10D2B0008091C00080648093C0009FBF08958F92CA
:10D2C0009F92AF92BF92EF92FF921F93CF93DF9303
:10D2D000CDB7DEB7A0970FB6F894DEBF0FBECDBFB7
:10D2E000611571058105910579F110E0842E912C6D
:10D2F000A12CB12CEE24E394F12CEC0EFD1EE10EDA
:10D30000F11C17FDFA94A50194010F946C06F70126
:10D310006083B901CA011F5F61157105810591051F
:10D3200049F7115010F1E1E0F0E0EC0FFD1FE10FC3
:10D33000F11D17FDFA9580818A3010F097E301C046
:10D3400090E3890F63DFEDCF80E3A0960FB6F894EA
:10D35000DEBF0FBECDBFDF91CF911F91FF90EF9049
:10D36000BF90AF909F908F9051CFA0960FB6F8943A
:10D37000DEBF0FBECDBFDF91CF911F91FF90EF9029
:10D38000BF90AF909F908F900895CF92DF92EF92D1
:10D39000FF926B017C0197FF0AC08DE237DFF094AA
:10D3A000E094D094C094C11CD11CE11CF11C4AE053
:10D3B000C701B601FF90EF90DF90CF9080CF8F92A2
:10D3C0009F92AF92BF92CF92DF92EF92FF92CF9354
:10D3D0006B017C01B42E20E030E0A9010F94910292
:10D3E00087FF06C08DE212DFF7FAF094F7F8F094A9
:10D3F000C0E060E070E080E09FE3CB1541F02DECF1
:10D400003CEC4CEC5DE30F94F602CF5FF6CF9B0152
:10D41000AC01C701B6010F94CA066B017C010F94E1
:10D4200013084B015C014AE04ADFCC2379F1C501C6
:10D43000B4010F9495029B01AC01C701B6010F9492
:10D44000C9066B017C018EE2E1DE20E030E040E2C3
:10D4500051E4C701B6010F94F6024B015C010F9431
:10D460000E086B01770FEE08FF08C701B6018DDFCC
:10D47000C701B6010F9497029B01AC01C501B4012D
:10D480000F94C9066B017C01C150F9F6CF91FF9052
:10D49000EF90DF90CF90BF90AF909F908F900895C6
:10D4A0008FB7F8949091BE092091BD09291759F0C2
:10D4B000E92FF0E0E35CF64F208130E09F5F9F773B
:10D4C0009093BE0902C02FEF3FEF8FBFC9010895AF
:10D4D0001F920F920FB60F9211240BB60F922F933B
:10D4E0003F934F935F936F937F938F939F93AF93EC
:10D4F000BF93EF93FF939091C6002FB7F894E091FC
:10D50000BD0981E08E0F8F773091BE09831731F00E
:10D51000F0E0E35CF64F90838093BD092FBF20912C
:10D520003C09422F50E04C30510508F046C0FA014A
:10D530008827EE55FF4F8F4F0D94B5099D3441F06C
:10D540009E34B9F481E005C09A3330F09D3471F512
:10D5500082E080933C0946C0903308F043C090328B
:10D5600009F440C09D3211F53DC0913329F0943348
:10D5700029F09032D9F436C083E0EBCF88E0E9CFD0
:10D58000903321F0913391F486E0E3CF84E0E1CF52
:10D59000983361F485E0DDCF923341F487E0D9CF51
:10D5A000913321F489E0D5CF903311F08BE0D1CFC6
:10D5B0008AE0CFCF9A30B1F413C09A3099F4273073
:10D5C00049F02A3059F0253059F410929A021092FD
:10D5D000F10D06C086ED99E10E94F9E90E949C9A3E
:10D5E00010923C09FF91EF91BF91AF919F918F9164
:10D5F0007F916F915F914F913F912F910F900BBE53
:10D600000F900FBE0F901F9018951F920F920FB69C
:10D610000F9211240BB60F928F939F93EF93FF936A
:10D620008091E009E82FF0E0E154F64F90818F5FA0
:10D630008F718093E0099093C6008091C000806450
:10D640008093C0009091DF098091E009981305C094
:10D650008091C1008F7D8093C100FF91EF919F91D8
:10D660008F910F900BBE0F900FBE0F901F901895CB
:10D670004F925F926F927F928F929F92AF92BF92E2
:10D68000CF92EF92FF920F931F93CF93DF93CDB77B
:10D69000DEB728970FB6F894DEBF0FBECDBF5C0192
:10D6A0004B013A0129018091F00983FD45C020E03A
:10D6B00030E0A901F80160817181828193810F942A
:10D6C000910281110CC020E030E0A901F5016081D8
:10D6D0007181828193810F949102882369F1F09086
:10D6E000EF09F11027C0E0914605F0E0EE0FFF1FB3
:10D6F000E55FF54F2081318180911E0290911F02DC
:10D7000028173907BCF4E6ECF7E184918F010F5F2D
:10D710001F4F882319F07ADDF801F7CFEDEAF9E120
:10D7200084918F010F5F1F4F882309F411C16EDDB3
:10D73000F801F6CF0E947B8C81E080933B099091A9
:10D740001F0B992321F010921F0B80933A090E941E
:10D750006362CC2051F081E08093DE0D40E050E028
:10D76000BA0182E096E70E94D6530E94CCF980E18C
:10D77000E1E2F5E0AAE2B9E001900D928A95E1F7C5
:10D7800020E030E0A901F5016081718182819381FF
:10D790000F949102882309F10E94218FF5012081C5
:10D7A00031814281538160912609709127098091CE
:10D7B0002809909129090F94CA066093260970934D
:10D7C0002709809328099093290960E070E080E799
:10D7D00092E40E94D9910E94CCF9F401808091805A
:10D7E000A280B38020E030E0A901C501B4010F940C
:10D7F000F0081816FCF480E090E0A0EAB0E4898319
:10D800009A83AB83BC83A501940160912905709133
:10D810002A0580912B0590912C050F94CA066D83E3
:10D820007E838F839887BE016F5F7F4FCE01059601
:10D830000E941A8F80E090E0A8ECB2E489839A837A
:10D84000AB83BC839E012F5F3F4F49E255E0B2019D
:10D85000C3010E943A8E20E030E0A901F801608106
:10D860007181828193810F949102882381F1CC2070
:10D8700069F081E08093DE0D40E050E0BA0181E77D
:10D8800095E70E94D65380E00E945EEA0E94218FB5
:10D89000F801208131814281538160912609709184
:10D8A000270980912809909129090F94CA0660934D
:10D8B000260970932709809328099093290960E02D
:10D8C00070E080E291E40E94D9910E94CCF9CC20D2
:10D8D00051F081E08093DE0D40E050E0BA018EEB24
:10D8E00093E70E94D65361E08E2D0E94E98C80E080
:10D8F0000E945EEA0E94EDE964E670E080E090E05C
:10D900000E94CFC50E940A53DC01CB018853904589
:10D91000AF4FBF4F8093620E9093630EA093640E3F
:10D92000B093650E10928A0A0E940A53DC01CB0163
:10D9300088539045AF4FBF4F8093660E9093670E0C
:10D94000A093680EB093690E10928B0AFF24F39493
:10D950008F2D28960FB6F894DEBF0FBECDBFDF9196
:10D96000CF911F910F91FF90EF90CF90BF90AF900C
:10D970009F908F907F906F905F904F900895AF929F
:10D98000BF92CF92DF92EF92FF921F93CF93DF93DC
:10D9900000D01F92CDB7DEB77C015B01D42E109171
:10D9A0008A0A1092620E1092630E1092640E109208
:10D9B000650E10928A0A80E00E949FCF90918B0A98
:10D9C000192B1092660E1092670E1092680E10922C
:10D9D000690E10928B0A81E00E949FCF11110E9464
:10D9E0007B8C61E08D2D0E94E98C0E94218F20E0CC
:10D9F00030E0A901F70160817181828193810F94E8
:10DA00009102882309F446C0112351F081E08093EC
:10DA1000DE0D40E050E0BA018EEB93E70E94D65352
:10DA200081E08093F10D8091F10D882351F0112355
:10DA300041F060E08D2D0E94E98C81E00E945EEA59
:10DA4000F2CF81E08093DE0D40E050E0BA018DE23C
:10DA500093E70E94D653F70120813181428153819F
:10DA600060912609709127098091280990912909D0
:10DA70000F94CA066093260970932709809328099A
:10DA80009093290960E070E080EC90E40E94D991C5
:10DA90000E94CCF9F501C080D180E280F38011E0D2
:10DAA00020E030E0A901C701B6010F94F008181674
:10DAB0002CF51093DE0D40E050E0BA018CE992E7BE
:10DAC0000E94D653A70196016091260970912709FB
:10DAD00080912809909129090F94CA06609326091C
:10DAE00070932709809328099093290960E070E0DA
:10DAF00080E490E40E94D9910E94CCF91092F10D3B
:10DB00001093DE0D1092E10940E050E0BA0183E984
:10DB100096E70E94D6538091E109811104C081E00B
:10DB20000E945EEAF8CFC12CD12C98E4E92E92E451
:10DB3000F92E813009F4B4CF11E01093DE0D40E0EE
:10DB400050E0BA018CE292E70E94D65380913609E8
:10DB500090913709A0913809B091390980932D052A
:10DB600090932E05A0932F05B0933005809326093E
:10DB700090932709A0932809B09329090E941E6257
:10DB800080E090E0A8ECB2E489839A83AB83BC8305
:10DB90009E012F5F3F4F49E255E06EE279E08AE255
:10DBA00099E00E943A8E80E090E0A0EAB0E4898398
:10DBB0009A83AB83BC83BE016F5F7F4F82E399E0A2
:10DBC0000E941A8F0E94115980913A09882339F0D6
:10DBD0008091200B811110931F0B10923A09109223
:10DBE0003B090F900F900F900F90DF91CF911F91F5
:10DBF000FF90EF90DF90CF90BF90AF900895CF92BD
:10DC0000DF92EF92FF920F931F93CF93DF9300D099
:10DC10001F92CDB7DEB78091FC049091FD04A091D6
:10DC2000FE04B091FF04B7FF08C01092FC041092EC
:10DC3000FD041092FE041092FF0480910005909163
:10DC40000105A0910205B09103054091FC0450919B
:10DC5000FD046091FE047091FF0484179507A607E8
:10DC6000B70744F48093FC049093FD04A093FE0452
:10DC7000B093FF0480911202882379F14091FC0453
:10DC80005091FD046091FE047091FF0480910405A1
:10DC900090910505A0910605B09107056A017B01E9
:10DCA000C80ED91EEA1EFB1EC701B6010F949502CD
:10DCB00020E030E048EC52E40F94F60269837A8366
:10DCC0008B839C83CE0101960E9448C4BC01809145
:10DCD0000A0590910B050E942C598091F00D10912E
:10DCE0000C05811106C01123E1F1809112028823F5
:10DCF000C1F14091FC045091FD046091FE047091CB
:10DD0000FF048091040590910505A0910605B0914E
:10DD100007056A017B01C80ED91EEA1EFB1EC7015A
:10DD2000B6010F94950220E030E048EC52E40F94E5
:10DD3000F6020F941308E0910805F0910905309759
:10DD400021F06083718382839383112329F0E09112
:10DD50000D05F0910E0519958091F00D81110E942D
:10DD600017598091F00D882329F0E0910D05F0916D
:10DD70000E0519950F900F900F900F90DF91CF9196
:10DD80001F910F91FF90EF90DF90CF900895CF9269
:10DD9000DF92EF92FF920F931F93CF93DF9300D008
:10DDA0001F92CDB7DEB78091FC049091FD04A09145
:10DDB000FE04B091FF04B7FF08C01092FC0410925B
:10DDC000FD041092FE041092FF04809100059091D2
:10DDD0000105A0910205B09103054091FC0450910A
:10DDE000FD046091FE047091FF0484179507A60757
:10DDF000B70744F48093FC049093FD04A093FE04C1
:10DE0000B093FF0480911202882379F14091FC04C1
:10DE10005091FD046091FE047091FF04809104050F
:10DE200090910505A0910605B09107056A017B0157
:10DE3000C80ED91EEA1EFB1EC701B6010F94970239
:10DE400020E030E048EC52E40F94F60269837A83D4
:10DE50008B839C83CE0101960E9448C4BC018091B3
:10DE60000A0590910B050E942C598091F00D10919C
:10DE70000C05811106C01123D1F180911202882373
:10DE8000B1F14091FC045091FD046091FE04709149
:10DE9000FF048091040590910505A0910605B091BD
:10DEA00007056A017B01C80ED91EEA1EFB1EC701C9
:10DEB000B6010F94970220E030E048EC52E40F9452
:10DEC000F602E0910805F0910905309721F0608392
:10DED000718382839383112329F0E0910D05F091E2
:10DEE0000E0519958091F00D81110E9417590F9020
:10DEF0000F900F900F90DF91CF911F910F91FF9096
:10DF0000EF90DF90CF900895CF92DF92EF92FF9243
:10DF10000F931F93CF93DF9300D01F92CDB7DEB73F
:10DF20008091FC049091FD04A091FE04B091FF0447
:10DF3000B7FF08C01092FC041092FD041092FE047A
:10DF40001092FF048091000590910105A0910205B7
:10DF5000B09103054091FC045091FD046091FE04D2
:10DF60007091FF0484179507A607B70744F48093C0
:10DF7000FC049093FD04A093FE04B093FF048091F1
:10DF80001202882379F14091FC045091FD046091C4
:10DF9000FE047091FF048091040590910505A09105
:10DFA0000605B09107056A017B01C80ED91EEA1E5D
:10DFB000FB1EC701B6010F9497022AE037ED43E23A
:10DFC0005CE30F94F60269837A838B839C83CE0192
:10DFD00001960E9412C3BC0180910A0590910B0525
:10DFE0000E942C598091F00D10910C05811106C0F2
:10DFF0001123D1F1809112028823B1F14091FC04E8
:10E000005091FD046091FE047091FF04809104051D
:10E0100090910505A0910605B09107056A017B0165
:10E02000C80ED91EEA1EFB1EC701B6010F94970247
:10E030002AE037ED43E25CE30F94F602E091080535
:10E04000F0910905309721F0608371838283938377
:10E05000112329F0E0910D05F0910E05199580919D
:10E06000F00D81110E9417598091F00D882329F03D
:10E07000E0910D05F0910E0519950F900F900F90FE
:10E080000F90DF91CF911F910F91FF90EF90DF9054
:10E09000CF900895CF92DF92EF92FF920F931F934C
:10E0A000CF93DF9300D01F92CDB7DEB78091FC04F1
:10E0B0009091FD04A091FE04B091FF04B7FF08C049
:10E0C0001092FC041092FD041092FE041092FF04C2
:10E0D0008091000590910105A0910205B091030582
:10E0E0004091FC045091FD046091FE047091FF0486
:10E0F00084179507A607B70744F48093FC04909310
:10E10000FD04A093FE04B093FF04809112028823C3
:10E1100079F14091FC045091FD046091FE047091EE
:10E12000FF048091040590910505A0910605B0912A
:10E1300007056A017B01C80ED91EEA1EFB1EC70136
:10E14000B6010F9497022AE037ED43E25CE30F94A7
:10E15000F60269837A838B839C83CE0101960E94A9
:10E16000C7C3BC0180910A0590910B050E942C59F0
:10E170008091F00D10910C05811106C01123D1F191
:10E18000809112028823B1F14091FC045091FD046A
:10E190006091FE047091FF04809104059091050543
:10E1A000A0910605B09107056A017B01C80ED91E32
:10E1B000EA1EFB1EC701B6010F9497022AE037ED55
:10E1C00043E25CE30F94F602E0910805F091090543
:10E1D000309721F06083718382839383112329F028
:10E1E000E0910D05F0910E0519958091F00D8111CA
:10E1F0000E9417590F900F900F900F90DF91CF91C1
:10E200001F910F91FF90EF90DF90CF9008950F93A3
:10E210001F93CF938091FC049091FD04A091FE0484
:10E22000B091FF04B7FF08C01092FC041092FD04E7
:10E230001092FE041092FF04809100059091010558
:10E24000A0910205B09103054091FC045091FD049A
:10E250006091FE047091FF0484179507A607B70725
:10E2600044F48093FC049093FD04A093FE04B093C7
:10E27000FF0480911202882331F14091FC045091F7
:10E28000FD046091FE047091FF048091040590915B
:10E290000505A0910605B09107058A019B01080FAD
:10E2A000191F2A1F3B1FC901B8010F9497020F9431
:10E2B0000E08CB010E9499C5BC0180910A0590917E
:10E2C0000B050E942C598091F00DC0910C05811115
:10E2D00006C0CC23A1F180911202882381F14091E4
:10E2E000FC045091FD046091FE047091FF04809144
:10E2F000040590910505A0910605B09107058A01D6
:10E300009B01080F191F2A1F3B1FC901B8010F9459
:10E310009702E0910805F0910905309721F060839C
:10E32000718382839383CC2329F0E0910D05F091D2
:10E330000E0519958091F00D81110E941759809159
:10E34000F00DCF911F910F91089561CF60DF882369
:10E3500029F0E0910D05F0910E0519940895809132
:10E36000FC049091FD04A091FE04B091FF04B7FF5E
:10E3700008C01092FC041092FD041092FE0410924A
:10E38000FF048091000590910105A0910205B091D4
:10E3900003054091FC045091FD046091FE047091CE
:10E3A000FF0484179507A607B70744F48093FC047D
:10E3B0009093FD04A093FE04B093FF048091120299
:10E3C000882399F020910405309105058091FC0483
:10E3D0009091FD04820F931F0E9499C5BC0180910A
:10E3E0000A0590910B050E942C598091F00D209107
:10E3F0000C05811106C0222311F18091120288239D
:10E40000F1F040910405509105058091FC04909134
:10E41000FD04840F951FE0910805F09109053097E0
:10E4200011F091838083222329F0E0910D05F09172
:10E430000E0519958091F00D81110E941759809158
:10E44000F00D08958CCF8BDF882329F0E0910D0526
:10E45000F0910E0519940895CF93DF931092E90D72
:10E460008091FC049091FD04A091FE04B091FF0402
:10E4700081309048A105B10540F01092FC04109243
:10E48000FD041092FE041092FF04C091FC048091E0
:10E49000EC0918160CF5282F082E000C330B25500C
:10E4A00031094C2F0C2E000C550B42175307A4F0CA
:10E4B00085301CF0CBEFC80F01C0C0E08C2F0C2EB4
:10E4C000000C990BAA0BBB0B8093FC049093FD04EA
:10E4D000A093FE04B093FF04C093EB09D0E0C111F8
:10E4E00009C0809112028823E9F021E041E06FEA3F
:10E4F0007BE115C0C13049F480911202882391F06C
:10E5000020E041E060EA7BE10AC0C23059F480912A
:10E510001202882339F020E041E066E97BE18D2F8B
:10E520000E94C762DF5FCF5FD530C9F683E080937A
:10E53000EC09DF91CF9108951F93CF93DF93109251
:10E54000E90D8091FC049091FD04A091FE04B0912E
:10E55000FF0481309048A105B10540F01092FC0401
:10E560001092FD041092FE041092FF04C091FC046E
:10E570008091EA0918160CF5282F082E000C330B91
:10E58000255031094C2F0C2E000C550B4217530708
:10E59000A4F085301CF0CBEFC80F01C0C0E08C2F79
:10E5A0000C2E000C990BAA0BBB0B8093FC049093D0
:10E5B000FD04A093FE04B093FF04C093EB09D0E0E8
:10E5C00012E0C11109C0809112028823D9F121E023
:10E5D00041E069E87BE115C0C13049F48091120245
:10E5E000882381F120E041E060E87BE10AC0C2308D
:10E5F00061F480911202882329F120E041E06FE666
:10E600007BE18D2F0E94C7621DC0C33049F4809109
:10E6100012028823B9F020E041E06DE67BE1F1CF02
:10E62000C43081F480911202882351F021E040E04F
:10E6300062E67BE18D2F0E94C7628D2F0E947A5A7D
:10E6400010931202DF5FCF5FD53009F0BACFD093BD
:10E65000EA09DF91CF911F9108951F93CF93DF9324
:10E660001092E90D8091FC049091FD04A091FE04AC
:10E67000B091FF0481309048A105B10540F010929F
:10E68000FC041092FD041092FE041092FF04C0914D
:10E69000FC048091E90918160CF5282F082E000CAF
:10E6A000330B255031094C2F0C2E000C550B421703
:10E6B0005307A4F085301CF0CBEFC80F01C0C0E0B9
:10E6C0008C2F0C2E000C990BAA0BBB0B8093FC0417
:10E6D0009093FD04A093FE04B093FF04C093EB0954
:10E6E000D0E012E0C11109C0809112028823D9F153
:10E6F00021E041E065E57BE115C0C13049F480913E
:10E700001202882381F120E041E06CE47BE10AC041
:10E71000C23061F480911202882329F120E041E0A7
:10E720006EE37BE18D2F0E94C7621DC0C33049F4A8
:10E73000809112028823B9F020E041E06CE37BE194
:10E74000F1CFC43081F480911202882351F021E08E
:10E7500040E061E37BE18D2F0E94C7628D2F0E9414
:10E760007A5A10931202DF5FCF5FD53009F0BACF2B
:10E77000D093E909DF91CF911F9108951F93CF9313
:10E78000DF931092E90D8091FC049091FD04A0911B
:10E79000FE04B091FF0481309048A105B10540F01E
:10E7A0001092FC041092FD041092FE041092FF04DB
:10E7B000C091FC048091E80918160CF5282F082E4A
:10E7C000000C330B255031094C2F0C2E000C550B2F
:10E7D00042175307A4F085301CF0CBEFC80F01C0DF
:10E7E000C0E08C2F0C2E000C990BAA0BBB0B809356
:10E7F000FC049093FD04A093FE04B093FF04C09327
:10E80000EB09D0E012E0C11109C080911202882307
:10E81000D9F121E041E064E27BE115C0C13049F467
:10E8200080911202882381F120E041E064E17BE1E4
:10E830000AC0C23061F480911202882329F120E0DD
:10E8400041E063E07BE18D2F0E94C7621DC0C330B1
:10E8500049F4809112028823B9F020E041E064EF8E
:10E860007AE1F1CFC43081F480911202882351F013
:10E8700021E040E069EE7AE18D2F0E94C7628D2F82
:10E880000E947A5A10931202DF5FCF5FD53009F0F1
:10E89000BACFD093E809DF91CF911F9108951F93CC
:10E8A000CF93DF931092E90D8091FC049091FD04C9
:10E8B000A091FE04B091FF0481309048A105B105FC
:10E8C00040F01092FC041092FD041092FE0410928D
:10E8D000FF04C091FC048091E70918160CF5282F5D
:10E8E000082E000C330B255031094C2F0C2E000C38
:10E8F000550B42175307A4F085301CF0CBEFC80F1F
:10E9000001C0C0E08C2F0C2E000C990BAA0BBB0B86
:10E910008093FC049093FD04A093FE04B093FF0445
:10E92000C093EB09D0E012E0C11109C0809112023E
:10E930008823D9F121E041E06CED7AE115C0C130C6
:10E9400049F480911202882381F120E041E06CECCF
:10E950007AE10AC0C23061F480911202882329F161
:10E9600020E041E06FEB7AE18D2F0E94C7621DC06D
:10E97000C33049F4809112028823B9F020E041E0CD
:10E980006DEB7AE1F1CFC43081F4809112028823DB
:10E9900051F021E040E062EB7AE18D2F0E94C762E6
:10E9A0008D2F0E947A5A10931202DF5FCF5FD5300D
:10E9B00009F0BACFD093E709DF91CF911F91089565
:10E9C0001F93CF93DF931092E90D8091FC049091F7
:10E9D000FD04A091FE04B091FF0481309048A10590
:10E9E000B10540F01092FC041092FD041092FE0458
:10E9F0001092FF04C091FC048091E60918160CF5F2
:10EA0000282F082E000C330B255031094C2F0C2ECB
:10EA1000000C550B42175307A4F085301CF0CBEFC8
:10EA2000C80F01C0C0E08C2F0C2E000C990BAA0B54
:10EA3000BB0B8093FC049093FD04A093FE04B09361
:10EA4000FF04C093EB09D0E012E0C11109C080912E
:10EA500012028823D9F121E041E065EA7AE115C08C
:10EA6000C13049F480911202882381F120E041E015
:10EA700066E97AE10AC0C23061F48091120288230B
:10EA800029F120E041E067E87AE18D2F0E94C7621A
:10EA90001DC0C33049F4809112028823B9F020E0F0
:10EAA00041E065E87AE1F1CFC43081F4809112024F
:10EAB000882351F021E040E06AE77AE18D2F0E943F
:10EAC000C7628D2F0E947A5A10931202DF5FCF5FC8
:10EAD000D53009F0BACFD093E609DF91CF911F91DD
:10EAE00008951F93CF93DF931092E90D8091FC045A
:10EAF0009091FD04A091FE04B091FF0481309048F4
:10EB0000A105B10540F01092FC041092FD04109292
:10EB1000FE041092FF04C091FC048091E5091816D0
:10EB20000CF5282F082E000C330B255031094C2FE3
:10EB30000C2E000C550B42175307A4F085301CF027
:10EB4000CBEFC80F01C0C0E08C2F0C2E000C990B2E
:10EB5000AA0BBB0B8093FC049093FD04A093FE04CE
:10EB6000B093FF04C093EB09D0E012E0C11109C0DB
:10EB7000809112028823D9F121E041E06DE67AE12B
:10EB800015C0C13049F480911202882381F120E040
:10EB900041E064E67AE10AC0C23061F48091120279
:10EBA000882329F120E041E064E57AE18D2F0E947D
:10EBB000C7621DC0C33049F4809112028823B9F0A6
:10EBC00020E041E062E57AE1F1CFC43081F4809148
:10EBD0001202882351F021E040E067E47AE18D2FB2
:10EBE0000E94C7628D2F0E947A5A10931202DF5F33
:10EBF000CF5FD53009F0BACFD093E509DF91CF913F
:10EC00001F9108951F93CF93DF931092E90D809188
:10EC1000FC049091FD04A091FE04B091FF048130AA
:10EC20009048A105B10540F01092FC041092FD043B
:10EC30001092FE041092FF04C091FC048091E4093C
:10EC400018160CF5282F082E000C330B255031090F
:10EC50004C2F0C2E000C550B42175307A4F0853097
:10EC60001CF0CBEFC80F01C0C0E08C2F0C2E000CA5
:10EC7000990BAA0BBB0B8093FC049093FD04A0930B
:10EC8000FE04B093FF04C093EB09D0E012E0C11181
:10EC900009C0809112028823D9F121E041E06AE3A2
:10ECA0007AE115C0C13049F480911202882381F1C4
:10ECB00020E041E06BE27AE10AC0C23061F4809169
:10ECC0001202882329F120E041E06BE17AE18D2FE7
:10ECD0000E94C7621DC0C33049F48091120288238C
:10ECE000B9F020E041E064E17AE1F1CFC43081F491
:10ECF00080911202882351F021E040E069E07AE13E
:10ED00008D2F0E94C7628D2F0E947A5A1093120293
:10ED1000DF5FCF5FD53009F0BACFD093E409DF9140
:10ED2000CF911F910895FF920F931F93CF93DF937D
:10ED30001092E90D8091FC049091FD04A091FE04D5
:10ED4000B091FF0481309048A105B10540F01092C8
:10ED5000FC041092FD041092FE041092FF04C09176
:10ED6000FC048091E3091816DCF4282F082E000C0F
:10ED7000330B215031094C2F0C2E000C550B421730
:10ED8000530774F0CFEFC80F8C2F90E0A0E0B0E0F5
:10ED90008093FC049093FD04A093FE04B093FF04C1
:10EDA0001092E2098091EB09C81714F4C093EB09A3
:10EDB0008091EB09082E000C990B04962C2F0C2E39
:10EDC000000C330B8217930724F48CEF8C0F809385
:10EDD000EB091091EB09D0E081E001E092E0F92E1F
:10EDE000111125C08823B1F01C16A4F08091FC04F9
:10EDF0009091FD04A091FE04B091FF040196A11D25
:10EE0000B11D8093FC049093FD04A093FE04B09385
:10EE1000FF04CF5F80911202882309F442C020E0F2
:10EE200041E069EF79E18D2F0E94C7623AC011304D
:10EE3000D1F48091F00D811105C0809112028823D8
:10EE400081F109C0C130C9F7F092E1098091E2096E
:10EE5000882399F32FC081E0C13009F080E020E2DF
:10EE60004CEE59E11BC01230E1F48091F00D81119C
:10EE700005C0809112028823A1F009C0C230C9F7F1
:10EE80000093E1098091E209882399F313C081E09E
:10EE9000C23009F080E020E24FED59E16D2F0E9471
:10EEA000ACC6DF5F1F5F80E0D53009F099CF83E00B
:10EEB0008093E309DF91CF911F910F91FF90089507
:10EEC0006F927F928F929F92AF92BF92CF92DF927A
:10EED000EF92FF920F931F93CF93DF9300D01F9277
:10EEE000CDB7DEB76C013B014701580129833A8356
:10EEF0004B835C830E94B65383E080931202D092CE
:10EF00000B05C0920A0570920905609208052981D7
:10EF10003A814B815C81CA01B9010F940E0860935C
:10EF200004057093050580930605909307050F94DB
:10EF300097026B017C019B01AC01C501B4010F94E8
:10EF4000C9060F940E086093000570930105809325
:10EF5000020590930305A7019601F3016081718179
:10EF6000828193810F94C9060F9413086093FC0467
:10EF70007093FD048093FE049093FF0485EA91E76B
:10EF800090931102809310020F900F900F900F90AA
:10EF9000DF91CF911F910F91FF90EF90DF90CF9075
:10EFA000BF90AF909F908F907F906F900895CF9279
:10EFB000DF92EF92FF920F931F93CF93DF938C0119
:10EFC000EB016A0179010E94B65323E020931202FB
:10EFD00010930B0500930A05D0930905C09308050B
:10EFE000A601DD0C660B770B4093040550930505D5
:10EFF0006093060570930705C701FF0CAA0BBB0BB6
:10F00000841B950BA60BB70B80930005909301050D
:10F01000A0930205B093030588819981092E000C05
:10F02000AA0BBB0B841B950BA60BB70B8093FC04A0
:10F030009093FD04A093FE04B093FF0482E292E754
:10F040009093110280931002DF91CF911F910F9145
:10F05000FF90EF90DF90CF9008953F924F925F9294
:10F060006F927F928F929F92AF92BF92CF92DF92D8
:10F07000EF92FF920F931F93CF93DF93CDB7DEB73D
:10F080002C970FB6F894DEBF0FBECDBF5C01DC013C
:10F0900059968D909C905A97F40181859285A3850D
:10F0A000B4859C01AD012F5F3F4F4F4F5F4F2987C4
:10F0B0003A874B875C87D5011496CD90DD90ED9013
:10F0C000FC901797C114D104E104F10439F0BFEFAB
:10F0D000CB1ADB0AEB0AFB0A312C07C0F401C08013
:10F0E000D180E280F38033243394260137011D82DE
:10F0F0001E821F821886F40181859285A385B485BE
:10F100002D813E814F815885281739074A075B07B3
:10F1100008F064C089859A85AB85BC858C159D05F2
:10F12000AE05BF0550F482E0C82ED12CE12CF12CA5
:10F1300092E0492E512C612C712C9E012F5F3F4F84
:10F14000B701A601C4010E949FB2882309F446C0FA
:10F1500089819A81AB81BC81892B8A2B8B2B41F0D1
:10F16000260137019FEF491A590A690A790A05C031
:10F17000C414D504E604F70491F02D813E814F813B
:10F1800058852F5F3F4F4F4F5F4F2D833E834F83F7
:10F1900058873FEFC31AD30AE30AF30AACCF0FEF45
:10F1A0001FEF2FEF3FE0B301A201C4010E940EB296
:10F1B000F82E882399F0D50114964D915D916D91AB
:10F1C0007C911797411551056105710549F093012F
:10F1D0008201C4010E940EB2811102C0F12C29C02B
:10F1E000D50114964D925D926D927C9217973320C3
:10F1F00051F0D301C2010196A11DB11DF40180831C
:10F200009183A283B383F50185899689A789B08DFF
:10F21000892B8A2B8B2B69F4D50155964D925D92E3
:10F220006D927C92589711968C91119780681196E7
:10F230008C938F2D2C960FB6F894DEBF0FBECDBFEA
:10F24000DF91CF911F910F91FF90EF90DF90CF90C2
:10F25000BF90AF909F908F907F906F905F904F90F6
:10F260003F9008950F931F93CF93DF938B010E94DC
:10F270000A53EB010E94FF688F3F49F00E940A5336
:10F280006C1B7D0B60177107A8F380E001C081E063
:10F29000DF91CF911F910F910895CF93DF93EC01F0
:10F2A0008B818823B9F1898187FF30C06C857D858A
:10F2B0008E859F8541E00E94D6B1882359F1E88967
:10F2C00080E2E89FF0011124DF01A55BBA4F10979F
:10F2D00009F18C91853EF1F08B81823050F449899F
:10F2E0005A896B897C895C964D935D936D937C9371
:10F2F0005F978D899E89AF89B88DE55BFA4F938FB3
:10F30000828FB58BA48B89818F778983DF91CF9191
:10F310000C9496B181E0888380E0DF91CF910895CD
:10F320008F929F92AF92BF92CF92DF92EF92FF9215
:10F330000F931F93CF93DF93EC018B81811102C058
:10F3400080E077C009891A892B893C890417150741
:10F3500026073707A8F36A017B01823029F4C886A3
:10F36000D986EA86FB860DC0C114D104E104F104FC
:10F3700051F41C821D821E821F82188619861A86ED
:10F380001B8681E056C088849984AA84BB84E98D59
:10F39000FA8D258530E0275F3F4FB501A40141502C
:10F3A000510961097109022E04C076956795579538
:10F3B00047950A94D2F7D701C6010197A109B1096F
:10F3C00004C0B695A795979587952A95D2F7841787
:10F3D0009507A607B70720F089288A288B2849F4C3
:10F3E0004D895E896F89788D4C835D836E837F83C1
:10F3F00004C0841B950BA60BB70B4C015D018E015D
:10F400000C5F1F4F81149104A104B10409F4A7CF2C
:10F410004C815D816E817F819801898D9A8D0E94DA
:10F420009FB291E0891A9108A108B1088111EACF31
:10F4300087CFDF91CF911F910F91FF90EF90DF90D9
:10F44000CF90BF90AF909F908F9008950F931F9390
:10F45000CF93DF93FC012381222311F080E044C08D
:10F460008B01EC01FB018789803139F18032B1F7E2
:10F4700083E08B83F801428D538D648D758D4D8BA8
:10F480005E8B6F8B788F9E012F5E3F4FC8010E946D
:10F4900020B3882319F31A8F098F81E089831C8296
:10F4A0001D821E821F82188619861A861B861C865C
:10F4B0001D861E861F86188A17C082E08B831D8AD0
:10F4C0001E8A1F8A188EFB01808D918DA0E0B0E00E
:10F4D00025E0880F991FAA1FBB1F2A95D1F7898B9A
:10F4E0009A8BAB8BBC8BD7CFDF91CF911F910F91B4
:10F4F00008950F931F93CF93DF93EB01FC012381BA
:10F50000211102C080E040C02250223028F48FE256
:10F510008883198281E038C08C01FC01648575857F
:10F520008685978540E00E94D6B1882359F3F8017B
:10F530004089F0E24F9FA00111249A01255B3A4FC8
:10F54000232B01F320E030E090E06EE2F901E40FBC
:10F55000F51FE55BFA4F7081703271F0283031058C
:10F5600029F4DE01A90FB11D6C939F5F7081FE012C
:10F57000E90FF11D70839F5F2F5F3F4F2B303105E7
:10F5800029F7C90FD11D1882DF91CF911F910F91DB
:10F590000895CF93DF93EC0180DE1B82DF91CF9142
:10F5A000089561E0FC0180810C94D9518EBD0DB4A9
:10F5B00007FEFDCF0895CF92DF92EF92FF921F9347
:10F5C000CF93DF9300D01F92CDB7DEB76C01162F1B
:10F5D000FC019281892F806A86958CBD90FD03C0C5
:10F5E00081E0963009F480E08DBD60E0F601808115
:10F5F00029833A834B835C830E94D9516CE271E08A
:10F60000C60130DE812F8064D1DF88E1E82EF12C45
:10F610005C814B813A812981DA01C9010E2C04C039
:10F62000B695A795979587950A94D2F729833A833B
:10F630004B835C83BBDFF8E0EF1AF10829813A8144
:10F640004B815C8188EFE8168FEFF80629F71123CC
:10F6500021F0183021F08FEF03C085E901C087E861
:10F66000A5DF1C3011F40E94FF6810E00E94FF68C3
:10F67000F601838387FF04C01F3F11F01F5FF6CFA1
:10F680000F900F900F900F90DF91CF911F91FF90EF
:10F69000EF90DF90CF9008950F931F93CF93DF9358
:10F6A000EC0189018C81833039F089E0440F551FCA
:10F6B000661F771F8A95D1F79A01AB0168E1CE01E9
:10F6C0007ADF882311F086E030C08EEF8EBD80E0B7
:10F6D00090E00DB407FEFDCFF801E80FF91F20817F
:10F6E0002EBD0DB407FEFDCF21812EBD02968115E2
:10F6F00022E0920771F70DB407FEFDCF8FEF56DFC2
:10F700008FEF54DF0E94FF688B838F71853029F063
:10F7100083E18983CE0145DF09C068E572E0CE014F
:10F72000A1DD182F811106C087E18983CE0139DF61
:10F7300010E010C020E030E0A9016DE0CE013BDF19
:10F74000811104C00E94FF68882311F086E1EDCF8B
:10F75000CE0127DF812FDF91CF911F910F91089567
:10F760002F923F924F925F926F927F928F929F92D1
:10F77000AF92BF92CF92DF92EF92FF920F931F93BF
:10F78000CF93DF9300D01F92CDB7DEB78C014B0132
:10F790001A01DC0113968C9113978130C1F41196F4
:10F7A0008C9181FF14C082FF18C0F80141895289F1
:10F7B0006389748980859185A285B38584179507AF
:10F7C000A607B70751F0C801ABDD811106C081E083
:10F7D000F80180838FEF9FEF2DC1610184C0D801B4
:10F7E00059968D919C915A97FC01248121502A01B0
:10F7F0003B0139E076946794579447943A95D1F752
:10F80000722E74207A01F1E0FF22772009F477C08C
:10F8100080E092E08E199F0956018C159D0508F431
:10F820005C01D80159962D913C915A9714968D916F
:10F830009D910D90BC91A02D0297A109B109F901EC
:10F84000058404C0880F991FAA1FBB1F0A94D2F712
:10F850004685578560897189840F951FA61FB71F3C
:10F860009C01AD01270D311D411D511D29013A019A
:10F87000A11432E0B30609F088C080914B07909143
:10F880004C07A0914D07B0914E0784159505A6052C
:10F89000B70569F4109253078FEF9FEFDC01809357
:10F8A0004B0790934C07A0934D07B0934E079401DC
:10F8B000B301A2018091540790915507EDDE882392
:10F8C00009F485CFF80180859185A285B3858A0DDD
:10F8D0009B1DA11DB11D80879187A287B3878A0CCC
:10F8E0009B1CCA18DB08D80118964D915D916D914B
:10F8F0007C911B97C114D10409F071CF7CC0E11435
:10F90000F10409F085CF14964D915D916D917C9134
:10F910001797411551056105710559F455968D915B
:10F920009D910D90BC91A02D0097A105B10539F5D1
:10F9300021C09E012F5F3F4F0E949FB2882309F490
:10F9400046CF89819A81AB81BC81F801218D328DAE
:10F95000F9012789203139F4883FFFEF9F07A1057E
:10F96000B10540F40CC0883F2FEF9207A2072FE0AB
:10F97000B20728F0C80171DB81114ACF28CFF80106
:10F9800084839583A683B78343CFE114F10419F5EB
:10F99000D80118964D915D916D917C911B97519670
:10F9A0008D919D910D90BC91A02D481759076A0724
:10F9B0007B0788F00E9496B1882309F408CF81E084
:10F9C0008093530740924B0750924C0760924D072B
:10F9D00070924E0708C041E0C301B2010E94D6B147
:10F9E000882309F4F4CEA501B401C701855B9A4FC1
:10F9F0000F94D20967CF51968D919D910D90BC9136
:10FA0000A02D84179507A607B70740F4F801418B8E
:10FA1000528B638B748B818180688183D8011196AE
:10FA20008C9183FD02C0C10105C0C80136DC811183
:10FA3000FACFCDCE0F900F900F900F90DF91CF9116
:10FA40001F910F91FF90EF90DF90CF90BF90AF90FC
:10FA50009F908F907F906F905F904F903F902F90EE
:10FA60000895EF92FF920F931F93CF93DF93EC01D2
:10FA700079018C81833039F089E0440F551F661F6E
:10FA8000771F8A95D1F79A01AB0161E1CE0193DD31
:10FA9000882329F084E08983CE0183DD38C00E9469
:10FAA0000A538B010E94FF688B838F3F49F40E94A9
:10FAB0000A53601B710B6D327140A0F381E103C0EA
:10FAC0008E3F39F08FE08983CE016BDD8FEF6EDDE5
:10FAD0001EC08FEF8EBDF701D701A150BE4F0DB4F0
:10FAE00007FEFDCF9EB591938EBDEA17FB07B9F7D0
:10FAF0000DB407FEFDCF8EB58C930E94FF680E9467
:10FB0000FF68CE014EDD8FEF51DD81E001C080E066
:10FB1000DF91CF911F910F91FF90EF9008952F9259
:10FB20003F924F925F926F927F928F929F92AF928D
:10FB3000BF92CF92DF92EF92FF920F931F93CF93DA
:10FB4000DF9300D01F92CDB7DEB79C838B834B0130
:10FB50005A01DC0113968C91811103C08FEF9FEF46
:10FB6000EAC0EB81FC81818180FFF8CFAB81BC8151
:10FB700051960D911D912D913C91549718964D9150
:10FB80005D916D917C911B97C501A0E0B0E068018B
:10FB90007901C41AD50AE60AF70AC816D906EA0690
:10FBA000FB0618F45801A41AB50A75018B819C81D3
:10FBB00004969A838983612C92E0792EE114F104F2
:10FBC00009F48BC0AB81BC8118964D915D916D910C
:10FBD0007C911B976A01B1E0DB22EB81FC812381E0
:10FBE0001A012B0189E056944794379427948A95FB
:10FBF000D1F7818D928D223061F4FC01828D938D3D
:10FC0000A48DB58DBC01CD01620D731D841D951DA4
:10FC10004AC0DC0114961C9111501221C114D10468
:10FC200001F511111EC0452B462B472B59F4EB81D2
:10FC3000FC8185899689A789B08D84839583A68365
:10FC4000B7830FC0AB81BC8114964D915D916D91CE
:10FC50007C91179729813A810E949FB2882309F4E9
:10FC60007DCFEB81FC81218D328D84819581A681B0
:10FC7000B7810297A109B109F901058404C0880F71
:10FC8000991FAA1FBB1F0A94D2F746855785608922
:10FC90007189840F951FA61FB71FBC01CD01610F8D
:10FCA000711D811D911D93012C193D0987012E1590
:10FCB0003F0508F489010115F2E01F0771F5209155
:10FCC0004B0730914C0740914D0750914E076217FA
:10FCD00073078407950719F420C0C5012CC094014F
:10FCE000AB01BC018091540790915507BADE88237F
:10FCF00009F434CF800E911EEB81FC8180859185C3
:10FD0000A285B385800F911FA11DB11D80879187AA
:10FD1000A287B387E01AF10A51CF40E00E94D6B122
:10FD2000882309F41BCFB601655B7A4FA801C40193
:10FD30000F94D209DFCF0F900F900F900F90DF91AB
:10FD4000CF911F910F91FF90EF90DF90CF90BF90D8
:10FD5000AF909F908F907F906F905F904F903F906B
:10FD60002F9008954F925F926F927F929F92AF92E1
:10FD7000BF92CF92DF92EF92FF920F931F93CF9398
:10FD8000DF931F92CDB7DEB78C017B016A01A22EF3
:10FD9000DB0159968D919C915A97F801928F818F32
:10FDA00040E050E0BA01C701BBDA912CF701808531
:10FDB0009185A285B38541895289638974898417A5
:10FDC0009507A607B70708F063C025E0B695A79585
:10FDD000979587952A95D1F7F82FFF70BF2ED701F9
:10FDE00013968C91823008F469C041E050E0BE0166
:10FDF0006F5F7F4FC70193DE019719F4898190E00F
:10FE000002C08FEF9FEF019609F458C0F70180857B
:10FE10009185A285B3854F96A11DB11D80879187DD
:10FE2000A287B387F0E2BF9EC0011124BC01655BCD
:10FE30007A4F6115710509F441C0DB012C91222331
:10FE400019F0253ED1F47CC191100EC040914B07B2
:10FE500050914C0760914D0770914E07F80144870F
:10FE6000558766877787B08AFC01E55BFA4F80810A
:10FE7000882361F09924939499CF4BE050E0C60118
:10FE80000F94C509892B09F091CF1AC09924939436
:10FE90008A2D8274823491F4992009F49CC0D8018F
:10FEA0005096BC9050971C966D917D918D919C9130
:10FEB0001F9741E00E94D6B1811180C080E043C10C
:10FEC000A7FCFCCFF0E2BF9EA00111249A01255BA4
:10FED0003A4FD9011B968C91817121F08A2D827144
:10FEE00009F068C080914B0790914C07A0914D0795
:10FEF000B0914E07F80184879587A687B787B08AA7
:10FF0000FA01E55BFA4F4489558960E070E0BA0177
:10FF100055274427D80155964D935D936D937C9357
:10FF20005897828D938DA0E0B0E0482B592B6A2B17
:10FF30007B2BD80155964D935D936D937C93589789
:10FF4000D9011B968C91887159F4848D958DA68D5D
:10FF5000B78DF801818B928BA38BB48B81E010C09D
:10FF6000803141F598012F5E3F4FD80159968D9110
:10FF70009C915A970E9420B38823E1F084E0F80115
:10FF800083838A2D8F70D80111968C931197F80175
:10FF9000148215821682178218961D921D921D9248
:10FFA0001C921B97A4FEC0C0C8010E9471BE8111A3
:10FFB000BBC084CFD80113961C9280CFF801608912
:10FFC000F0E26F9FB0011124655B7A4F61157105F6
:10FFD00009F08AC073CFD70113968C9113978230A2
:10FFE00009F46CCF51968D919D910D90BC91A02DEF
:10FFF000803E9F4FAF41B10508F060CFC7012DD8BB
:020000021000EC
:10000000882309F45BCF0E9496B1882309F456CF68
:10001000D70159962D913C915A9714968D919D91A7
:100020000D90BC91A02D0297A109B109F901058499
:1000300004C0880F991FAA1FBB1F0A94D2F74684D9
:10004000578460887188480E591E6A1E7B1E81E0A5
:100050008093530740924B0750924C0760924D0794
:1000600070924E0780E092E0EBE4F5E0DF019C0146
:100070001D9221503040E1F7BB24B394D70159962B
:10008000ED91FC915A978481B81690F42BE435E0F9
:10009000B301A2014B0D511D611D711D80915407CB
:1000A00090915507F9DA882309F408CFB394E6CF85
:1000B00080E092E0A0E0B0E0058404C0880F991FC2
:1000C000AA1FBB1F0A94D2F7F7014189528963899D
:1000D0007489840F951FA61FB71F818B928BA38BEA
:1000E000B48B6BE475E0B12C80E2DB011D928A9544
:1000F000E9F78BE0F601DB0101900D928A95E1F7BB
:1001000081E298E2FB01918B808B20E038E0378719
:100110002687938B828B918F808F378B268B0E94C3
:1001200096B18111CFCECACEA5FE08C0F801418993
:10013000528963897489C801F3D805C081E003C07E
:10014000911098CE83CE0F90DF91CF911F910F9198
:10015000FF90EF90DF90CF90BF90AF909F907F90F7
:100160006F905F904F9008952F923F924F925F92C1
:100170006F927F928F929F92AF92BF92CF92DF92B7
:10018000EF92FF920F931F93CF93DF93CDB7DEB71C
:10019000C554D1090FB6F894DEBF0FBECDBF3C01E8
:1001A0005B018A01322E1C8E1F8E19821C82672BE6
:1001B00011F410E0A7C0FC0183818111FACFFA018C
:1001C00080818F3261F4CA018C010196F80120818F
:1001D0002F32D1F3F50183818250823010F4750102
:1001E0000AC0618D728DCE01019630D9882309F342
:1001F000CE0101967C016E019CE1C90ED11C260145
:100200004E01E7E38E0E911CFBE0F80D2596FFAF43
:100210002597CE01019624969FAF8EAF2497269600
:10022000CFAE26972D2C35C080E2819325969FADC9
:1002300025979E13F9CFD80190E027E04A2F3B2F56
:100240008D91811128C08FA9803209F4B2CF842FFB
:10025000932F8C01FC01208101962F32D1F32223B0
:1002600009F44AC021E0A401B701C6017BDD88235F
:1002700009F49FCFEA14FB0411F0C7018AD9C41412
:10028000D50499F126969FAD2697822D7601C92E29
:10029000D82EF401C9CF8F32B1F28E3219F0ECEBC7
:1002A000FBE10AC02A3009F484CF98E02AE0C6CFE7
:1002B0003196381709F47DCF34913111F9CF2917D0
:1002C00008F477CF813208F474CF8F3709F471CFF7
:1002D00031E0390FF401E90FF11D9FE9980F9A31D0
:1002E00008F480528083932FA9CF23969FAD239744
:1002F00024968FAD2497CACF232DA401B701C30143
:1003000031DD182FCE0101960E94EC4CCE014C96A7
:100310000E94EC4C812FCB5BDF4F0FB6F894DEBF11
:100320000FBECDBFDF91CF911F910F91FF90EF9046
:10033000DF90CF90BF90AF909F908F907F906F9005
:100340005F904F903F902F90089521E02093DE0D15
:100350006093F2097093F3098093F4099093F5097F
:1003600040E050E0BA018091F7099091F8090C94AF
:10037000D65360E070E080E291E4E7CF60E070E0A7
:1003800080E89FE3E2CF6DEC7CEC8CEC9DE3DDCF6D
:10039000CF92DF92EF92FF92CF93C82F833029F450
:1003A00067FD609146056093D50D0E940A536B016D
:1003B0007C0124EA30E74DE75FE36091F209709138
:1003C000F3098091F4099091F5090F94910287FD4A
:1003D00005C08AEF90E0A0E0B0E003C080E090E0CC
:1003E000DC01C80ED91EEA1EFB1EC092D60DD092AB
:1003F000D70DE092D80DF092D90DC0937602CF912F
:10040000FF90EF90DF90CF900895CF93DF9390917E
:10041000F00D992321F0DF91CF910C941759C82F3B
:100420006091FC047091FD048091FE049091FF04A2
:10043000611571058105910571F10F949702209165
:10044000F2093091F3094091F4095091F5090F94A4
:10045000F6029B01AC0160912D0570912E058091F3
:100460002F05909130050F94CA0660932D05709367
:100470002E0580932F05909330051092FC04109266
:10048000FD041092FE041092FF046C2F83E080DFC5
:1004900081E08093120280911202882389F0C1309A
:1004A00019F4C9EEDCE102C0C3EFDCE18DE295E0B6
:1004B0000E94EAC4BC01CE01DF91CF910C942C596B
:1004C000DF91CF91089581E0A0CF8FEF9ECF3F9233
:1004D0004F925F926F927F928F929F92AF92BF9254
:1004E000CF92DF92EF92FF920F931F93CF93DF9300
:1004F00000D000D0CDB7DEB72091F00D2223C9F097
:1005000026960FB6F894DEBF0FBECDBFDF91CF9118
:100510001F910F91FF90EF90DF90CF90BF90AF9021
:100520009F908F907F906F905F904F903F900C9432
:100530001759362E8C018091FC049091FD04A091F6
:10054000FE04B091FF04892B8A2B8B2B09F492C0F7
:100550000E946253932DA4E09A02C00111249E834D
:100560008D83FC01EF5DFA4F408051806280738083
:100570008091320281110BC020E030E04AE754E460
:10058000C301B2010F94CA066B017C0108C0ED8162
:10059000FE81EA5DFD4FC080D180E280F3808091D2
:1005A000FC049091FD04A091FE04B091FF048983A6
:1005B0009A83AB83BC83BC01CD010F949702209139
:1005C000F2093091F3094091F4095091F5090F9423
:1005D000F6029B01AC01C301B2010F94CA064B01A4
:1005E0005C01AD81BE81AF5DBA4FBE83AD83FD01BD
:1005F000608371838283938389819A81AB81BC817B
:10060000B7FF13C020E030E04AE754E4C301B20171
:100610000F94C9066B017C019B01AC01C501B401BB
:100620000F94910287FF18C010C089819A81AB8115
:10063000BC81892B8A2B8B2B79F0A7019601C501F0
:10064000B4010F94F00818163CF4AD81BE81CD9230
:10065000DD92ED92FC9213976FEF832D99DE10924D
:10066000FC041092FD041092FE041092FF0481E03D
:100670008093120280911202882309F4A1C02DEC0C
:100680003CEC4CEC5DE36091F2097091F3098091D0
:10069000F4099091F5090F94F008632D330C770B52
:1006A00087FD0AC0CB01880F991F880F991F8F5DA6
:1006B0009A4F0E94EAC469C0660F771F660F771FC2
:1006C000FB01EF5DFA4F20E030E04AE754E460813F
:1006D0007181828193810F94F6020F940E086B0151
:1006E0007C01611571058105910561F097FF0AC0D4
:1006F000F094E094D094C094C11CD11CE11CF11C76
:100700008DE201C080E28093010EC701B60128EEA0
:1007100033E040E050E00F948E068AE0882E912C62
:10072000A12CB12CCA01B901A50194010F948E0628
:10073000605D6093020E8EE28093030EC701B601E6
:1007400024E630E040E050E00F948E06CA01B90183
:10075000A50194010F948E06605D6093040EC7019D
:10076000B601A50194010F948E06F62ECA01B901B7
:10077000A50194010F948E06605D6093050E80E3E1
:100780008F0D8093060E81E09EE0BC01C801269685
:100790000FB6F894DEBF0FBECDBFDF91CF911F9192
:1007A0000F91FF90EF90DF90CF90BF90AF909F9010
:1007B0008F907F906F905F904F903F900C942C594A
:1007C00026960FB6F894DEBF0FBECDBFDF91CF9156
:1007D0001F910F91FF90EF90DF90CF90BF90AF905F
:1007E0009F908F907F906F905F904F903F90089573
:1007F00062E082EE9CE16BCE61E08BED9CE167CE26
:1008000060E084ED9CE163CE80E00C949FCF81E0BA
:100810000C949FCF0C9454CFFF920F931F93CF93C0
:10082000DF931092E90D8091FC049091FD04A0915A
:10083000FE04B091FF0481309048A105B10540F05D
:100840001092FC041092FD041092FE041092FF041A
:10085000C091FC048091F1091816DCF4282F082EB1
:10086000000C330B215031094C2F0C2E000C550B72
:100870004217530774F0CFEFC80F8C2F90E0A0E021
:10088000B0E08093FC049093FD04A093FE04B09329
:10089000FF041092E2098091EB09C81714F4C09389
:1008A000EB098091EB09082E000C990B04962C2F74
:1008B0000C2E000C330B8217930724F48CEF8C0F53
:1008C0008093EB091091EB09D0E0FF24F394111110
:1008D0001DC08091F00D811106C080911202882305
:1008E00009F471C109C0C111F8CF0E941759809154
:1008F000E209882391F36FC181E0C11180E024E017
:100900004FEC5CE16D2F0E94ACC65DC1113051F51A
:100910008091F00D811106C080911202882309F4A4
:1009200052C111C0C130C1F727EE33E04AE050E0B8
:1009300064E272E089EC9CE10E94D7778091E20941
:10094000882351F348C180912402909125020E948E
:1009500099C59C0181E0C13009F080E000E043ECE2
:100960005CE12EC11230A1F58091F00D811106C01D
:1009700080911202882309F426C11BC0C230C1F73E
:10098000F092E90D1092E50D1092E60D1092E70D30
:100990001092E80D24E034E842E251E06BE07AE0A6
:1009A0008AEB9CE10E9424638091E209882301F391
:1009B00012C180910B0A90910C0A0E9499C59C016A
:1009C00081E0C23009F080E000E041EB5CE1F8C07A
:1009D0001330A1F58091F00D811106C080911202B3
:1009E000882309F4F0C01BC0C330C1F7F092E90DB1
:1009F0001092E50D1092E60D1092E70D1092E80DA1
:100A000027E034E842E251E06DE07AE088EA9CE1D8
:100A10000E9424638091E209882301F3DCC0809165
:100A20000D0A90910E0A0E9499C59C0181E0C33085
:100A300009F080E000E04FE95CE1C2C01430A1F5AC
:100A40008091F00D811106C080911202882309F473
:100A5000BAC01BC0C430C1F7F092E90D1092E50D89
:100A60001092E60D1092E70D1092E80D2AE034E89E
:100A700047E850E069E07AE08BE99CE10E9424635A
:100A80008091E209882301F3A6C08091090A909120
:100A90000A0A0E9499C59C0181E0C43009F080E0F7
:100AA00000E047E95CE18CC01530A1F58091F00DC4
:100AB000811106C080911202882309F484C01BC0F2
:100AC000C530C1F7F092E90D1092E50D1092E60DD8
:100AD0001092E70D1092E80D2FEF30E040E050E06B
:100AE00065E07AE08BE89CE10E94D7778091E2098B
:100AF000882301F370C08091050A9091060A0E9434
:100B000099C59C0181E0C53009F080E000E04FE725
:100B10005CE156C0163051F58091F00D811106C090
:100B200080911202882309F44EC011C0C630C1F76B
:100B300027EE33E04AE050E060E272E088E79CE1B3
:100B40000E94D7778091E209882351F344C08091B5
:100B50002002909121020E9499C59C0181E0C6303B
:100B600009F080E000E041E75CE12AC0173059F568
:100B70008091F00D811105C080911202882319F136
:100B800011C0C730C9F727EE33E04AE050E062E217
:100B900072E08AE69CE10E94D7778091E20988237F
:100BA00059F319C080912202909123020E9499C5A5
:100BB0009C0181E0C73009F080E000E043E65CE1A1
:100BC0006D2F0E94F059DF5F1F5FD53009F07FCE97
:100BD00088E08093F109DF91CF911F910F91FF90F1
:100BE0000895CF92DF92EF92FF921F93CF93DF93FE
:100BF0001092E90D8091FC049091FD04A091FE04F7
:100C0000B091FF0481309048A105B10540F01092E9
:100C1000FC041092FD041092FE041092FF04C09197
:100C2000FC048091ED091816DCF4282F082E000C26
:100C3000330B215031094C2F0C2E000C550B421751
:100C4000530774F0CFEFC80F8C2F90E0A0E0B0E016
:100C50008093FC049093FD04A093FE04B093FF04E2
:100C60001092E2098091EB09C81714F4C093EB09C4
:100C70008091EB09082E000C990B04962C2F0C2E5A
:100C8000000C330B8217930724F48CEF8C0F8093A6
:100C9000EB091091EB09D0E087EEE82E8BE1F82EFE
:100CA00095EFC92E9BE1D92E11111AC08091F00D3C
:100CB000811106C080911202882309F472C009C014
:100CC000C111F8CF0E9417598091E209882391F34E
:100CD00070C081E0C11180E024E049EF5BE15EC0BB
:100CE0001130F9F48091F00D811106C0809112024B
:100CF000882309F456C00DC0C130C1F7D092570700
:100D0000C09256070E9451498091E209882371F3ED
:100D100050C081E0C13009F080E020E24BEE5BE1A1
:100D20003DC01230F1F48091F00D811105C0809129
:100D300012028823B1F10DC0C230C9F7F0925707F3
:100D4000E09256070E9451498091E209882379F385
:100D500030C081E0C23009F080E020E246ED5BE186
:100D60001DC01330F1F48091F00D811105C0809108
:100D700012028823B1F00BC0C330C9F784E399E9AC
:100D80000E94CDCA8091E209882389F312C081E0D4
:100D9000C33009F080E023E04CEC5BE16D2F0E9452
:100DA000ACC6DF5F1F5FD53009F07ECF84E0809353
:100DB000ED09DF91CF911F91FF90EF90DF90CF90E1
:100DC00008958091F00D882321F01092DE0D0C948F
:100DD00017590C94F0EFEF92FF921F93CF93DF938C
:100DE0001092E90D8091FC049091FD04A091FE0405
:100DF000B091FF0481309048A105B10540F01092F8
:100E0000FC041092FD041092FE041092FF04C091A5
:100E1000FC048091EE091816DCF4282F082E000C33
:100E2000330B215031094C2F0C2E000C550B42175F
:100E3000530774F0CFEFC80F8C2F90E0A0E0B0E024
:100E40008093FC049093FD04A093FE04B093FF04F0
:100E50001092E2098091EB09C81714F4C093EB09D2
:100E60008091EB09082E000C990B04962C2F0C2E68
:100E7000000C330B8217930724F48CEF8C0F8093B4
:100E8000EB091091EB09D0E08EEFE82E8BE1F82E04
:100E900011111AC08091F00D811106C080911202CB
:100EA000882309F4A6C009C0C111F8CF0E941759C0
:100EB0008091E209882391F3A3C081E0C11180E011
:100EC00024E048E45CE192C01130E9F48091F00D37
:100ED000811106C080911202882309F48AC00BC0D8
:100EE000C130C1F78BEC96EB0E94CDCA8091E2092C
:100EF000882381F385C081E0C13009F080E023E0E0
:100F000046E35CE173C0123041F58091F00D811130
:100F100006C080911202882309F46BC016C0C2304B
:100F2000C1F70E9485DA882319F00E949CC608C088
:100F300048EB51E064E170E080E090E00E9442FC08
:100F40008091E209882329F35BC081E0C23009F077
:100F500080E020E247E25CE149C0133041F5809136
:100F6000F00D811106C080911202882309F441C05E
:100F700016C0C330C1F70E9466D5882319F00E94BD
:100F80009CC608C048EB51E064E170E080E090E06E
:100F90000E9442FC8091E209882329F331C081E05C
:100FA000C33009F080E020E248E05CE11FC014306B
:100FB00001F58091F00D811105C080911202882306
:100FC000C1F00DC0C430C9F7F0925707E092560740
:100FD0000E9451498091E209882379F311C081E090
:100FE000C43009F080E020E246E15CE16D2F0E9410
:100FF000ACC6DF5F1F5FD53009F04ACFD093EE0952
:10100000DF91CF911F91FF90EF9008950F931F9361
:10101000CF93DF93082F7093F8096093F70910922C
:10102000E90D8091FC049091FD04A091FE04B09123
:10103000FF0481309048A105B10540F01092FC04F6
:101040001092FD041092FE041092FF04C091FC0463
:101050008091F6091816DCF4282F082E000C330BAB
:10106000215031094C2F0C2E000C550B4217530701
:1010700074F0CFEFC80F8C2F90E0A0E0B0E0809329
:10108000FC049093FD04A093FE04B093FF0410921F
:10109000E2098091EB09C81714F4C093EB09209181
:1010A000EB09022E000C330B2C5F3F4F8C2F0C2EC4
:1010B000000C990B2817390724F48CEF8C0F8093C0
:1010C000EB091091EB09D0E091E0013049F10230D9
:1010D00009F44AC001116CC0111191C09923B1F0FB
:1010E0001C16A4F08091FC049091FD04A091FE04D4
:1010F000B091FF040196A11DB11D8093FC04909353
:10110000FD04A093FE04B093FF04CF5F8091120210
:10111000882309F4EEC021E041E06CE37DE16BC07F
:1011200011116DC09923B1F01C16A4F08091FC043C
:101130009091FD04A091FE04B091FF040196A11DC1
:10114000B11D8093FC049093FD04A093FE04B09322
:10115000FF04CF5F80911202882309F4CAC021E006
:1011600041E065E37DE147C0111149C09923B1F029
:101170001C16A4F08091FC049091FD04A091FE0443
:10118000B091FF040196A11DB11D8093FC049093C2
:10119000FD04A093FE04B093FF04CF5F8091120280
:1011A000882309F4A6C021E041E06EE27DE123C07E
:1011B000111125C09923B1F01C16A4F08091FC04F4
:1011C0009091FD04A091FE04B091FF040196A11D31
:1011D000B11D8093FC049093FD04A093FE04B09392
:1011E000FF04CF5F80911202882309F482C021E0BE
:1011F00041E065E27DE18D2F0E94C7627AC0113027
:10120000D9F48091F00D811106C0809112028823DB
:1012100009F46FC009C0C130C1F70E94175980910D
:10122000E209882391F36DC081E0C13009F080E0CC
:1012300024E04BE15DE15AC01230E9F48091F00DF9
:10124000811106C080911202882309F452C00BC09C
:10125000C230C1F789EB91E80E94CDCA8091E209C2
:10126000882381F34EC081E0C23009F080E023E0A2
:1012700041E15DE13BC01330E1F48091F00D81115B
:1012800005C0809112028823A1F10BC0C330C9F7B9
:101290008EEB91E80E94CDCA8091E209882389F300
:1012A00030C081E0C33009F080E023E048E05DE138
:1012B0001DC01430F1F48091F00D811105C08091B2
:1012C00012028823B1F00BC0C430C9F783EC91E857
:1012D0000E94CDCA8091E209882389F312C081E07F
:1012E000C43009F080E023E04DEF5CE16D2F0E94F7
:1012F000ACC6DF5F1F5F90E0D53009F0E6CED0933B
:10130000F609DF91CF911F910F910895CF93C82FC8
:101310008091F00983FD1EC08091EF0981111AC0F0
:10132000E0914605F0E0EE0FFF1FE55FF54F2081ED
:10133000318180911E0290911F022817390754F4C1
:101340000E94B65340E050E0BA0188EE93EBCF9193
:101350000C94D65381E08093DE0D40E050E0BA015A
:1013600082E096E70E94D653CC2319F08DE49CE1ED
:1013700002C088E59CE19093570780935607CF9170
:101380000C945149EF92FF920F931F93CF937C01DE
:101390008B01C42F80E20E940669CF3F11F084E5E3
:1013A00001C082E40E940669C7FD04C080E38C0F7F
:1013B0000E9406698AE30E940669F70160817181D3
:1013C0008281938142E00E94DF69F801408151816E
:1013D0006281738186E39EE10E948DC262E070E0CB
:1013E00080E090E0CF911F910F91FF90EF900C94CF
:1013F000D052CF92EF92FF920F931F93E09087020B
:10140000F09088020091890210918A02C0904605EE
:101410002DE235E049E255E065E275E081E295E0D4
:101420000E94C2A41F910F91FF90EF90CF9008955A
:101430000F931F93CF93DF93CDB7DEB728970FB6E7
:10144000F894DEBF0FBECDBF00912E0410E0F8016E
:10145000EE0FFF1FE55FF54F60817181072E000CD5
:10146000880B990B0F9497026D837E838F839887E7
:10147000000F111F000F111FF801E452FB4F808174
:101480009181A281B38189839A83AB83BC834EEF20
:10149000BE016B5F7F4FCE01019674DF6091090A38
:1014A00070910A0A072E000C880B990B0F94970273
:1014B0006D837E838F8398878091E4049091E50407
:1014C000A091E604B091E70489839A83AB83BC833F
:1014D0004FEFBE016B5F7F4FCE01019653DF6091EE
:1014E0000B0A70910C0A072E000C880B990B0F94B5
:1014F00097026D837E838F8398878091DC0490911F
:10150000DD04A091DE04B091DF0489839A83AB836C
:10151000BC8340E0BE016B5F7F4FCE01019632DF9E
:1015200060910D0A70910E0A072E000C880B990B22
:101530000F9497026D837E838F8398878091E00458
:101540009091E104A091E204B091E30489839A832D
:10155000AB83BC8341E0BE016B5F7F4FCE01019640
:1015600011DFE1E4FEE184918F010F5F1F4F8823BB
:1015700021F00E940669F801F6CFE0912E04F0E018
:10158000EB56F14F608170E080E090E00E94C56909
:10159000ECE3FEE184918F010F5F1F4F882321F060
:1015A0000E940669F801F6CF6091920E70E080E02B
:1015B00090E00E94C56960E070E089E39EE10E94CE
:1015C000D1C28AE30E9406696091950E70E080E0C6
:1015D00090E00E94C56961E070E089E39EE10E94AD
:1015E000D1C28AE30E9406696091960E70E080E0A5
:1015F00090E00E94C56928960FB6F894DEBF0FBE32
:10160000CDBFDF91CF911F910F9108950F931F933D
:10161000CF93DF9383E50E94E04C882309F452C006
:101620000E945E4C082F80E50E94E04C882309F45C
:1016300049C080E50E94E04C882331F00E944E4C66
:10164000EB0177FD3FC002C0CDE0D0E09C2FE7EF7B
:10165000FDE180E38E0F2491921721F031968E13D5
:10166000FACF16C0E6ECF7E18491EF0121968823CA
:1016700021F00E940669FE01F7CFE7E2FEE18491C6
:10168000EF0121968823F1F00E940669FE01F7CF51
:101690008C2F0E940BBD602F8C2F0E94D95110E01F
:1016A000B8018C2F0E940952C630D10529F410933D
:1016B000060A0093050A06C0289721F41093080A29
:1016C0000093070ADF91CF911F910F9108950F9317
:1016D0001F93CF9380911F0B81110E94CCF9009131
:1016E0002C0410912D0480E50E94B14CC82F882352
:1016F00019F00E946F4CC82F8091200B882341F174
:101700004C2F61E0C8010E94885C83E50E94E04C98
:10171000882381F00E944E4CAB01BC014093C20D66
:101720005093C30D6093C40D7093C50D81E19DE08E
:101730000E9490798091200B882319F081E080939A
:101740001F0BC11105C0CF911F910F910C944D61DA
:10175000CF911F910F9108956F927F928F929F92D8
:10176000AF92BF92CF92DF92EF92FF920F931F93AF
:10177000CF93DF93CDB7DEB765970FB6F894DEBF92
:101780000FBECDBF0E947BC02CE3C22ED12CE12C1A
:10179000F12CA70196010F946C06762E672ECA01D4
:1017A000B901A70196010F946C066B017C01CA0177
:1017B000B90128E130E040E050E00F946C064B01A5
:1017C0005C01C9016DE671E00F948E098E010F5F17
:1017D0001F4F6115710599F06F927F92DF92CF9242
:1017E0009F928F929F938F937F936F9386ED9DE14E
:1017F0009F938F931F930F930F942A0212C0009709
:10180000B1F06F927F92DF92CF929F928F929F93CF
:101810008F9386EC9DE19F938F931F930F930F946B
:101820002A020FB6F894DEBF0FBECDBF36C08114BA
:101830009104A104B10479F06F927F92DF92CF926C
:101840009F928F928AEB9DE19F938F931F930F93AB
:101850000F942A02E6CFC114D104E104F10469F027
:101860006F927F92DF92CF9282EB9DE19F938F9355
:101870001F930F930F942A02D4CF6F927F928EEA18
:101880009DE19F938F931F930F930F942A020F90C4
:101890000F900F900F900F900F9060E0C8010E9482
:1018A00086C7E4EFF2E284917F019FEFE91AF90A1B
:1018B000882321F00E940669F701F5CFB8018AEE6E
:1018C0009DE10E94EAC28AE00E94066965960FB611
:1018D000F894DEBF0FBECDBFDF91CF911F910F9166
:1018E000FF90EF90DF90CF90BF90AF909F908F9040
:1018F0007F906F900895BF92CF92DF92EF92FF9208
:101900000F931F93CF93DF9381E080939A02BB24C0
:10191000B39481E090919A02992309F44FC08823EF
:1019200009F44CC080E00E945EEA0BE01AE0CCEDC6
:10193000D4E0F801619171918F0161157105B1F1E8
:10194000072E000C880B990B0F9497029B01AC019A
:10195000688179818A819B810F94C9066B017C0122
:1019600020E030E0A9010F94F00818165CF420E0A4
:1019700030E040E251E4C701B6010F94F0081816B8
:10198000ACF40AC020E030E040E251ECC701B601FF
:101990000F94910287FF0AC0B092DE0D40E050E044
:1019A000BA0180EE94E70E94D653B3CF249680E02C
:1019B000FAE00F301F0709F4ADCFBBCFDF91CF9115
:1019C0001F910F91FF90EF90DF90CF90BF900C94FC
:1019D0001159CF92DF92EF92FF920F931F93CF9303
:1019E000DF9300D01F92CDB7DEB7182F662351F0DA
:1019F0001092030A1092FF091092000A1092010A35
:101A00001092020A0E940A53C090FF09D090000A67
:101A1000E090010AF090020A9B01AC012C193D09EB
:101A20004E095F0957FD3EC017FD16C04091030ADD
:101A3000212F012E000C330B2C5F3F4FE42F042E7F
:101A4000000CFF0B2E173F076CF141172CF000E93B
:101A500011E020E030E004C004EC19E020E030E0C8
:101A6000DC01CB01800F911FA21FB31F8093FF09E0
:101A70009093000AA093010AB093020A80ED97E0C8
:101A80009C838B838CE291E09A838983BE016D5F96
:101A90007F4FCE0101960E94FE608091030A8F5F06
:101AA0008093030A0F900F900F900F90DF91CF91CA
:101AB0001F910F91FF90EF90DF90CF900895BF920C
:101AC000CF92DF92EF92FF920F931F93CF93DF930A
:101AD0008AE1E82E89E0F82E01E215E09BE3C92EA9
:101AE00094E0D92EC3E4D3E0BC2E84E0B80E8991F3
:101AF0000E94B14C8823D9F00E947E4CF6012081CF
:101B0000211104C020913F04222331F0F8012081EB
:101B100031814281538103C020E030E0A9010F945C
:101B2000CA06F70160837183828393830AC0F80138
:101B300080819181A281B381F70180839183A28307
:101B4000B383F4E0EF0EF11C0C5F1F4F8FEFC81A48
:101B5000D80ABC12CCCF86E40E94E04C8823C9F09E
:101B60000E947E4C20E030E0A9010F94F008181686
:101B700084F40E947E4C20E030E040E752E40F9471
:101B8000A6076093870270938802809389029093DE
:101B90008A02DF91CF911F910F91FF90EF90DF901C
:101BA000CF90BF9008959F92AF92BF92CF92DF9255
:101BB000EF92FF920F931F93CF93DF9300D01F926A
:101BC000CDB7DEB7902EA12EB22ED32E94E089028F
:101BD0007001112487010F5D1A4FF80110821182E4
:101BE0001282138249835A836B837C830E94344C14
:101BF00049815A816B817C81F801408351836283E2
:101C00007383C090460520E030E0A901692D7A2D4C
